Component: ARM Compiler 5.06 update 2 (build 183) Tool: armlink [4d35b7]

==============================================================================

Section Cross References

    main.o(i.app_error_fault_handler) refers to main.o(i.on_error) for on_error
    main.o(i.app_error_handler) refers to main.o(i.on_error) for on_error
    main.o(i.app_error_handler_bare) refers to main.o(i.on_error) for on_error
    main.o(i.dfu_observer) refers to boards.o(i.bsp_board_init) for bsp_board_init
    main.o(i.dfu_observer) refers to boards.o(i.bsp_board_led_on) for bsp_board_led_on
    main.o(i.dfu_observer) refers to boards.o(i.bsp_board_led_off) for bsp_board_led_off
    main.o(i.main) refers to nrf_bootloader_info.o(i.nrf_bootloader_mbr_addrs_populate) for nrf_bootloader_mbr_addrs_populate
    main.o(i.main) refers to nrf_bootloader_app_start_final.o(i.nrf_bootloader_flash_protect) for nrf_bootloader_flash_protect
    main.o(i.main) refers to nrf_bootloader.o(i.nrf_bootloader_init) for nrf_bootloader_init
    main.o(i.main) refers to main.o(i.on_error) for on_error
    main.o(i.main) refers to main.o(i.dfu_observer) for dfu_observer
    boards.o(i.bsp_board_button_idx_to_pin) refers to boards.o(.constdata) for .constdata
    boards.o(i.bsp_board_button_state_get) refers to boards.o(.constdata) for .constdata
    boards.o(i.bsp_board_init) refers to boards.o(i.nrf_gpio_cfg) for nrf_gpio_cfg
    boards.o(i.bsp_board_init) refers to boards.o(i.bsp_board_leds_off) for bsp_board_leds_off
    boards.o(i.bsp_board_init) refers to boards.o(.constdata) for .constdata
    boards.o(i.bsp_board_led_idx_to_pin) refers to boards.o(.constdata) for .constdata
    boards.o(i.bsp_board_led_invert) refers to boards.o(.constdata) for .constdata
    boards.o(i.bsp_board_led_off) refers to boards.o(i.nrf_gpio_pin_write) for nrf_gpio_pin_write
    boards.o(i.bsp_board_led_off) refers to boards.o(.constdata) for .constdata
    boards.o(i.bsp_board_led_on) refers to boards.o(i.nrf_gpio_pin_write) for nrf_gpio_pin_write
    boards.o(i.bsp_board_led_on) refers to boards.o(.constdata) for .constdata
    boards.o(i.bsp_board_led_state_get) refers to boards.o(.constdata) for .constdata
    boards.o(i.bsp_board_leds_off) refers to boards.o(i.bsp_board_led_off) for bsp_board_led_off
    boards.o(i.bsp_board_leds_on) refers to boards.o(i.bsp_board_led_on) for bsp_board_led_on
    boards.o(i.bsp_board_pin_to_button_idx) refers to boards.o(.constdata) for .constdata
    boards.o(i.bsp_board_pin_to_led_idx) refers to boards.o(.constdata) for .constdata
    nrf_bootloader.o(i.boot_validate) refers to nrf_dfu_validation.o(i.nrf_dfu_validation_boot_validate) for nrf_dfu_validation_boot_validate
    nrf_bootloader.o(i.bootloader_reset) refers to nrf_dfu_settings.o(i.nrf_dfu_settings_backup) for nrf_dfu_settings_backup
    nrf_bootloader.o(i.bootloader_reset) refers to nrf_bootloader.o(i.do_reset) for do_reset
    nrf_bootloader.o(i.bootloader_reset) refers to nrf_bootloader.o(.data) for .data
    nrf_bootloader.o(i.dfu_enter_check) refers to nrf_bootloader.o(i.boot_validate) for boot_validate
    nrf_bootloader.o(i.dfu_enter_check) refers to nrf_dfu_utils.o(i.nrf_dfu_bank0_start_addr) for nrf_dfu_bank0_start_addr
    nrf_bootloader.o(i.dfu_enter_check) refers to nrf_dfu_settings.o(.bss) for s_dfu_settings
    nrf_bootloader.o(i.dfu_observer) refers to nrf_bootloader_dfu_timers.o(i.nrf_bootloader_dfu_inactivity_timer_restart) for nrf_bootloader_dfu_inactivity_timer_restart
    nrf_bootloader.o(i.dfu_observer) refers to nrf_bootloader.o(i.bootloader_reset) for bootloader_reset
    nrf_bootloader.o(i.dfu_observer) refers to nrf_dfu_settings.o(i.nrf_dfu_settings_reinit) for nrf_dfu_settings_reinit
    nrf_bootloader.o(i.dfu_observer) refers to nrf_bootloader.o(i.inactivity_timeout) for inactivity_timeout
    nrf_bootloader.o(i.dfu_observer) refers to nrf_bootloader.o(.data) for .data
    nrf_bootloader.o(i.flash_write_callback) refers to nrf_bootloader.o(.data) for .data
    nrf_bootloader.o(i.inactivity_timeout) refers to nrf_bootloader.o(i.bootloader_reset) for bootloader_reset
    nrf_bootloader.o(i.nrf_bootloader_init) refers to nrf_dfu_settings.o(i.nrf_dfu_settings_init) for nrf_dfu_settings_init
    nrf_bootloader.o(i.nrf_bootloader_init) refers to nrf_bootloader_fw_activation.o(i.nrf_bootloader_fw_activate) for nrf_bootloader_fw_activate
    nrf_bootloader.o(i.nrf_bootloader_init) refers to nrf_bootloader.o(i.dfu_enter_check) for dfu_enter_check
    nrf_bootloader.o(i.nrf_bootloader_init) refers to main.o(i.led_test) for led_test
    nrf_bootloader.o(i.nrf_bootloader_init) refers to nrf_bootloader_wdt.o(i.nrf_bootloader_wdt_init) for nrf_bootloader_wdt_init
    nrf_bootloader.o(i.nrf_bootloader_init) refers to app_scheduler.o(i.app_sched_init) for app_sched_init
    nrf_bootloader.o(i.nrf_bootloader_init) refers to main.o(i.app_error_handler_bare) for app_error_handler_bare
    nrf_bootloader.o(i.nrf_bootloader_init) refers to nrf_bootloader.o(i.bootloader_reset) for bootloader_reset
    nrf_bootloader.o(i.nrf_bootloader_init) refers to nrf_bootloader.o(i.nrf_dfu_init_user) for nrf_dfu_init_user
    nrf_bootloader.o(i.nrf_bootloader_init) refers to nrf_bootloader_dfu_timers.o(i.nrf_bootloader_dfu_inactivity_timer_restart) for nrf_bootloader_dfu_inactivity_timer_restart
    nrf_bootloader.o(i.nrf_bootloader_init) refers to nrf_dfu.o(i.nrf_dfu_init) for nrf_dfu_init
    nrf_bootloader.o(i.nrf_bootloader_init) refers to nrf_bootloader_wdt.o(i.nrf_bootloader_wdt_feed) for nrf_bootloader_wdt_feed
    nrf_bootloader.o(i.nrf_bootloader_init) refers to app_scheduler.o(i.app_sched_execute) for app_sched_execute
    nrf_bootloader.o(i.nrf_bootloader_init) refers to nrf_dfu_settings.o(i.nrf_dfu_settings_additional_erase) for nrf_dfu_settings_additional_erase
    nrf_bootloader.o(i.nrf_bootloader_init) refers to nrf_dfu_settings.o(i.nrf_dfu_settings_backup) for nrf_dfu_settings_backup
    nrf_bootloader.o(i.nrf_bootloader_init) refers to nrf_bootloader_app_start.o(i.nrf_bootloader_app_start) for nrf_bootloader_app_start
    nrf_bootloader.o(i.nrf_bootloader_init) refers to nrf_bootloader.o(.data) for .data
    nrf_bootloader.o(i.nrf_bootloader_init) refers to nrf_bootloader.o(.bss) for .bss
    nrf_bootloader.o(i.nrf_bootloader_init) refers to nrf_bootloader.o(i.inactivity_timeout) for inactivity_timeout
    nrf_bootloader.o(i.nrf_bootloader_init) refers to nrf_bootloader.o(i.dfu_observer) for dfu_observer
    nrf_bootloader.o(i.nrf_bootloader_init) refers to nrf_bootloader.o(i.flash_write_callback) for flash_write_callback
    nrf_bootloader_app_start.o(i.nrf_bootloader_app_start) refers to nrf_dfu_mbr.o(i.nrf_dfu_mbr_irq_forward_address_set) for nrf_dfu_mbr_irq_forward_address_set
    nrf_bootloader_app_start.o(i.nrf_bootloader_app_start) refers to nrf_bootloader_app_start_final.o(i.nrf_bootloader_app_start_final) for nrf_bootloader_app_start_final
    nrf_bootloader_app_start_final.o(i.nrf_bootloader_app_start_final) refers to nrf_bootloader_app_start_final.o(i.nrf_bootloader_flash_protect) for nrf_bootloader_flash_protect
    nrf_bootloader_app_start_final.o(i.nrf_bootloader_app_start_final) refers to main.o(i.app_error_handler_bare) for app_error_handler_bare
    nrf_bootloader_app_start_final.o(i.nrf_bootloader_app_start_final) refers to nrf_dfu_utils.o(i.nrf_dfu_bank0_start_addr) for nrf_dfu_bank0_start_addr
    nrf_bootloader_app_start_final.o(i.nrf_bootloader_app_start_final) refers to nrf_dfu_settings.o(.bss) for s_dfu_settings
    nrf_bootloader_app_start_final.o(i.nrf_bootloader_flash_protect) refers to nrf_bootloader_app_start_final.o(.data) for .data
    nrf_bootloader_dfu_timers.o(i.RTC1_IRQHandler) refers to nrf_bootloader_dfu_timers.o(i.nrf_rtc_event_clear) for nrf_rtc_event_clear
    nrf_bootloader_dfu_timers.o(i.RTC1_IRQHandler) refers to nrf_bootloader_dfu_timers.o(i.timer_stop) for timer_stop
    nrf_bootloader_dfu_timers.o(i.RTC1_IRQHandler) refers to nrf_bootloader_dfu_timers.o(i.timer_activate) for timer_activate
    nrf_bootloader_dfu_timers.o(i.RTC1_IRQHandler) refers to nrf_bootloader_dfu_timers.o(.data) for .data
    nrf_bootloader_dfu_timers.o(i.nrf_bootloader_dfu_inactivity_timer_restart) refers to nrf_bootloader_dfu_timers.o(i.timer_stop) for timer_stop
    nrf_bootloader_dfu_timers.o(i.nrf_bootloader_dfu_inactivity_timer_restart) refers to nrf_bootloader_dfu_timers.o(i.timer_start) for timer_start
    nrf_bootloader_dfu_timers.o(i.nrf_bootloader_dfu_inactivity_timer_restart) refers to nrf_bootloader_dfu_timers.o(.data) for .data
    nrf_bootloader_dfu_timers.o(i.nrf_bootloader_dfu_timer_counter_get) refers to nrf_bootloader_dfu_timers.o(.data) for .data
    nrf_bootloader_dfu_timers.o(i.nrf_bootloader_wdt_feed_timer_start) refers to nrf_bootloader_dfu_timers.o(i.timer_start) for timer_start
    nrf_bootloader_dfu_timers.o(i.nrf_bootloader_wdt_feed_timer_start) refers to nrf_bootloader_dfu_timers.o(.data) for .data
    nrf_bootloader_dfu_timers.o(i.timer_activate) refers to nrf_bootloader_dfu_timers.o(i.nrf_rtc_event_clear) for nrf_rtc_event_clear
    nrf_bootloader_dfu_timers.o(i.timer_activate) refers to nrf_bootloader_dfu_timers.o(.constdata) for .constdata
    nrf_bootloader_dfu_timers.o(i.timer_init) refers to nrf_bootloader_dfu_timers.o(i.nrf_rtc_event_clear) for nrf_rtc_event_clear
    nrf_bootloader_dfu_timers.o(i.timer_init) refers to nrf_bootloader_dfu_timers.o(.data) for .data
    nrf_bootloader_dfu_timers.o(i.timer_start) refers to nrf_bootloader_dfu_timers.o(i.timer_init) for timer_init
    nrf_bootloader_dfu_timers.o(i.timer_start) refers to nrf_bootloader_dfu_timers.o(i.timer_activate) for timer_activate
    nrf_bootloader_fw_activation.o(i.app_activate) refers to nrf_dfu_utils.o(i.nrf_dfu_bank0_start_addr) for nrf_dfu_bank0_start_addr
    nrf_bootloader_fw_activation.o(i.app_activate) refers to nrf_bootloader_fw_activation.o(i.image_copy) for image_copy
    nrf_bootloader_fw_activation.o(i.app_activate) refers to crc32.o(i.crc32_compute) for crc32_compute
    nrf_bootloader_fw_activation.o(i.app_activate) refers to nrf_dfu_settings.o(.bss) for s_dfu_settings
    nrf_bootloader_fw_activation.o(i.bl_activate) refers to nrf_dfu_utils.o(i.nrf_dfu_bank1_start_addr) for nrf_dfu_bank1_start_addr
    nrf_bootloader_fw_activation.o(i.bl_activate) refers to memcmp.o(.text) for memcmp
    nrf_bootloader_fw_activation.o(i.bl_activate) refers to nrf_bootloader_wdt.o(i.nrf_bootloader_wdt_feed) for nrf_bootloader_wdt_feed
    nrf_bootloader_fw_activation.o(i.bl_activate) refers to nrf_dfu_mbr.o(i.nrf_dfu_mbr_copy_bl) for nrf_dfu_mbr_copy_bl
    nrf_bootloader_fw_activation.o(i.bl_activate) refers to nrf_dfu_settings.o(.bss) for s_dfu_settings
    nrf_bootloader_fw_activation.o(i.flash_write_callback) refers to nrf_bootloader_fw_activation.o(.data) for .data
    nrf_bootloader_fw_activation.o(i.image_copy) refers to nrf_bootloader_wdt.o(i.nrf_bootloader_wdt_init) for nrf_bootloader_wdt_init
    nrf_bootloader_fw_activation.o(i.image_copy) refers to nrf_dfu_flash.o(i.nrf_dfu_flash_erase) for nrf_dfu_flash_erase
    nrf_bootloader_fw_activation.o(i.image_copy) refers to nrf_dfu_flash.o(i.nrf_dfu_flash_store) for nrf_dfu_flash_store
    nrf_bootloader_fw_activation.o(i.image_copy) refers to nrf_dfu_settings.o(i.nrf_dfu_settings_write_and_backup) for nrf_dfu_settings_write_and_backup
    nrf_bootloader_fw_activation.o(i.image_copy) refers to nrf_dfu_settings.o(.bss) for s_dfu_settings
    nrf_bootloader_fw_activation.o(i.nrf_bootloader_fw_activate) refers to nrf_bootloader_fw_activation.o(i.app_activate) for app_activate
    nrf_bootloader_fw_activation.o(i.nrf_bootloader_fw_activate) refers to nrf_bootloader_fw_activation.o(i.sd_activate) for sd_activate
    nrf_bootloader_fw_activation.o(i.nrf_bootloader_fw_activate) refers to nrf_bootloader_fw_activation.o(i.bl_activate) for bl_activate
    nrf_bootloader_fw_activation.o(i.nrf_bootloader_fw_activate) refers to nrf_dfu_utils.o(i.nrf_dfu_bank_invalidate) for nrf_dfu_bank_invalidate
    nrf_bootloader_fw_activation.o(i.nrf_bootloader_fw_activate) refers to nrf_dfu_settings.o(i.nrf_dfu_settings_write_and_backup) for nrf_dfu_settings_write_and_backup
    nrf_bootloader_fw_activation.o(i.nrf_bootloader_fw_activate) refers to nrf_dfu_settings.o(.bss) for s_dfu_settings
    nrf_bootloader_fw_activation.o(i.nrf_bootloader_fw_activate) refers to nrf_bootloader_fw_activation.o(.data) for .data
    nrf_bootloader_fw_activation.o(i.nrf_bootloader_fw_activate) refers to nrf_bootloader_fw_activation.o(i.flash_write_callback) for flash_write_callback
    nrf_bootloader_fw_activation.o(i.sd_activate) refers to nrf_dfu_utils.o(i.nrf_dfu_softdevice_start_address) for nrf_dfu_softdevice_start_address
    nrf_bootloader_fw_activation.o(i.sd_activate) refers to nrf_bootloader_fw_activation.o(i.image_copy) for image_copy
    nrf_bootloader_fw_activation.o(i.sd_activate) refers to nrf_dfu_settings.o(i.nrf_dfu_settings_write_and_backup) for nrf_dfu_settings_write_and_backup
    nrf_bootloader_fw_activation.o(i.sd_activate) refers to nrf_dfu_settings.o(.bss) for s_dfu_settings
    nrf_bootloader_info.o(i.nrf_bootloader_debug_port_disable) refers to nrf_nvmc.o(i.nrf_nvmc_write_word) for nrf_nvmc_write_word
    nrf_bootloader_info.o(i.nrf_bootloader_debug_port_disable) refers to nrf_bootloader_info.o(i.__NVIC_SystemReset) for __NVIC_SystemReset
    nrf_bootloader_info.o(i.nrf_bootloader_mbr_addrs_populate) refers to nrf_nvmc.o(i.nrf_nvmc_write_word) for nrf_nvmc_write_word
    nrf_bootloader_wdt.o(i.nrf_bootloader_wdt_feed) refers to nrf_bootloader_wdt.o(i.nrf_wdt_started) for nrf_wdt_started
    nrf_bootloader_wdt.o(i.nrf_bootloader_wdt_feed) refers to nrf_bootloader_wdt.o(i.wdt_feed) for wdt_feed
    nrf_bootloader_wdt.o(i.nrf_bootloader_wdt_init) refers to nrf_bootloader_wdt.o(i.nrf_wdt_started) for nrf_wdt_started
    nrf_bootloader_wdt.o(i.nrf_bootloader_wdt_init) refers to nrf_bootloader_wdt.o(i.wdt_feed) for wdt_feed
    nrf_bootloader_wdt.o(i.nrf_bootloader_wdt_init) refers to nrf_bootloader_dfu_timers.o(i.nrf_bootloader_wdt_feed_timer_start) for nrf_bootloader_wdt_feed_timer_start
    nrf_bootloader_wdt.o(i.nrf_bootloader_wdt_init) refers to nrf_bootloader_wdt.o(.data) for .data
    nrf_bootloader_wdt.o(i.nrf_bootloader_wdt_init) refers to nrf_bootloader_wdt.o(i.wdt_feed_timer_handler) for wdt_feed_timer_handler
    nrf_bootloader_wdt.o(i.wdt_feed) refers to nrf_bootloader_wdt.o(i.nrf_wdt_started) for nrf_wdt_started
    nrf_bootloader_wdt.o(i.wdt_feed_timer_handler) refers to nrf_bootloader_wdt.o(i.wdt_feed) for wdt_feed
    nrf_crypto_ecc.o(i.nrf_crypto_ecc_curve_info_get) refers to nrf_crypto_ecc.o(i.nrf_crypto_internal_ecc_key_input_check) for nrf_crypto_internal_ecc_key_input_check
    nrf_crypto_ecc.o(i.nrf_crypto_ecc_key_pair_generate) refers to nrf_crypto_ecc.o(i.nrf_crypto_internal_ecc_key_output_prepare) for nrf_crypto_internal_ecc_key_output_prepare
    nrf_crypto_ecc.o(i.nrf_crypto_ecc_key_pair_generate) refers to micro_ecc_backend_ecc.o(i.nrf_crypto_backend_micro_ecc_key_pair_generate) for nrf_crypto_backend_micro_ecc_key_pair_generate
    nrf_crypto_ecc.o(i.nrf_crypto_ecc_private_key_free) refers to nrf_crypto_ecc.o(i.nrf_crypto_internal_ecc_key_input_check) for nrf_crypto_internal_ecc_key_input_check
    nrf_crypto_ecc.o(i.nrf_crypto_ecc_private_key_from_raw) refers to nrf_crypto_ecc.o(i.nrf_crypto_internal_ecc_key_output_prepare) for nrf_crypto_internal_ecc_key_output_prepare
    nrf_crypto_ecc.o(i.nrf_crypto_ecc_private_key_from_raw) refers to nrf_crypto_ecc.o(i.nrf_crypto_internal_ecc_raw_input_check) for nrf_crypto_internal_ecc_raw_input_check
    nrf_crypto_ecc.o(i.nrf_crypto_ecc_private_key_from_raw) refers to micro_ecc_backend_ecc.o(i.nrf_crypto_backend_micro_ecc_private_key_from_raw) for nrf_crypto_backend_micro_ecc_private_key_from_raw
    nrf_crypto_ecc.o(i.nrf_crypto_ecc_private_key_to_raw) refers to nrf_crypto_ecc.o(i.nrf_crypto_internal_ecc_key_input_check) for nrf_crypto_internal_ecc_key_input_check
    nrf_crypto_ecc.o(i.nrf_crypto_ecc_private_key_to_raw) refers to nrf_crypto_ecc.o(i.nrf_crypto_internal_ecc_raw_output_prepare) for nrf_crypto_internal_ecc_raw_output_prepare
    nrf_crypto_ecc.o(i.nrf_crypto_ecc_private_key_to_raw) refers to micro_ecc_backend_ecc.o(i.nrf_crypto_backend_micro_ecc_private_key_to_raw) for nrf_crypto_backend_micro_ecc_private_key_to_raw
    nrf_crypto_ecc.o(i.nrf_crypto_ecc_public_key_calculate) refers to nrf_crypto_ecc.o(i.nrf_crypto_internal_ecc_key_input_check) for nrf_crypto_internal_ecc_key_input_check
    nrf_crypto_ecc.o(i.nrf_crypto_ecc_public_key_calculate) refers to nrf_crypto_ecc.o(i.nrf_crypto_internal_ecc_key_output_prepare) for nrf_crypto_internal_ecc_key_output_prepare
    nrf_crypto_ecc.o(i.nrf_crypto_ecc_public_key_calculate) refers to micro_ecc_backend_ecc.o(i.nrf_crypto_backend_micro_ecc_public_key_calculate) for nrf_crypto_backend_micro_ecc_public_key_calculate
    nrf_crypto_ecc.o(i.nrf_crypto_ecc_public_key_free) refers to nrf_crypto_ecc.o(i.nrf_crypto_internal_ecc_key_input_check) for nrf_crypto_internal_ecc_key_input_check
    nrf_crypto_ecc.o(i.nrf_crypto_ecc_public_key_from_raw) refers to nrf_crypto_ecc.o(i.nrf_crypto_internal_ecc_key_output_prepare) for nrf_crypto_internal_ecc_key_output_prepare
    nrf_crypto_ecc.o(i.nrf_crypto_ecc_public_key_from_raw) refers to nrf_crypto_ecc.o(i.nrf_crypto_internal_ecc_raw_input_check) for nrf_crypto_internal_ecc_raw_input_check
    nrf_crypto_ecc.o(i.nrf_crypto_ecc_public_key_from_raw) refers to micro_ecc_backend_ecc.o(i.nrf_crypto_backend_micro_ecc_public_key_from_raw) for nrf_crypto_backend_micro_ecc_public_key_from_raw
    nrf_crypto_ecc.o(i.nrf_crypto_ecc_public_key_to_raw) refers to nrf_crypto_ecc.o(i.nrf_crypto_internal_ecc_key_input_check) for nrf_crypto_internal_ecc_key_input_check
    nrf_crypto_ecc.o(i.nrf_crypto_ecc_public_key_to_raw) refers to nrf_crypto_ecc.o(i.nrf_crypto_internal_ecc_raw_output_prepare) for nrf_crypto_internal_ecc_raw_output_prepare
    nrf_crypto_ecc.o(i.nrf_crypto_ecc_public_key_to_raw) refers to micro_ecc_backend_ecc.o(i.nrf_crypto_backend_micro_ecc_public_key_to_raw) for nrf_crypto_backend_micro_ecc_public_key_to_raw
    nrf_crypto_ecdsa.o(i.nrf_crypto_ecdsa_sign) refers to nrf_crypto_ecc.o(i.nrf_crypto_internal_ecc_key_input_check) for nrf_crypto_internal_ecc_key_input_check
    nrf_crypto_ecdsa.o(i.nrf_crypto_ecdsa_sign) refers to nrf_crypto_ecc.o(i.nrf_crypto_internal_ecc_raw_output_prepare) for nrf_crypto_internal_ecc_raw_output_prepare
    nrf_crypto_ecdsa.o(i.nrf_crypto_ecdsa_sign) refers to micro_ecc_backend_ecdsa.o(i.nrf_crypto_backend_micro_ecc_sign) for nrf_crypto_backend_micro_ecc_sign
    nrf_crypto_ecdsa.o(i.nrf_crypto_ecdsa_verify) refers to nrf_crypto_ecc.o(i.nrf_crypto_internal_ecc_key_input_check) for nrf_crypto_internal_ecc_key_input_check
    nrf_crypto_ecdsa.o(i.nrf_crypto_ecdsa_verify) refers to nrf_crypto_ecc.o(i.nrf_crypto_internal_ecc_raw_input_check) for nrf_crypto_internal_ecc_raw_input_check
    nrf_crypto_ecdsa.o(i.nrf_crypto_ecdsa_verify) refers to micro_ecc_backend_ecdsa.o(i.nrf_crypto_backend_micro_ecc_verify) for nrf_crypto_backend_micro_ecc_verify
    nrf_crypto_hash.o(i.nrf_crypto_hash_calculate) refers to nrf_crypto_hash.o(i.nrf_crypto_hash_init) for nrf_crypto_hash_init
    nrf_crypto_hash.o(i.nrf_crypto_hash_calculate) refers to nrf_crypto_hash.o(i.nrf_crypto_hash_update) for nrf_crypto_hash_update
    nrf_crypto_hash.o(i.nrf_crypto_hash_calculate) refers to nrf_crypto_hash.o(i.nrf_crypto_hash_finalize) for nrf_crypto_hash_finalize
    nrf_crypto_hash.o(i.nrf_crypto_hash_finalize) refers to nrf_crypto_hash.o(i.verify_context) for verify_context
    nrf_crypto_hash.o(i.nrf_crypto_hash_update) refers to nrf_crypto_hash.o(i.verify_context) for verify_context
    nrf_crypto_init.o(i.nrf_crypto_init) refers to nrf_crypto_init.o(.data) for .data
    nrf_crypto_init.o(i.nrf_crypto_is_initialized) refers to nrf_crypto_init.o(.data) for .data
    nrf_crypto_init.o(i.nrf_crypto_is_initializing) refers to nrf_crypto_init.o(.data) for .data
    nrf_crypto_init.o(i.nrf_crypto_uninit) refers to nrf_crypto_init.o(.data) for .data
    nrf_crypto_shared.o(i.nrf_crypto_internal_double_swap_endian) refers to nrf_crypto_shared.o(i.nrf_crypto_internal_swap_endian) for nrf_crypto_internal_swap_endian
    nrf_crypto_shared.o(i.nrf_crypto_internal_double_swap_endian_in_place) refers to nrf_crypto_shared.o(i.nrf_crypto_internal_swap_endian_in_place) for nrf_crypto_internal_swap_endian_in_place
    nrf_sw_backend_hash.o(i.nrf_sw_backend_hash_sha256_finalize) refers to sha256.o(i.sha256_final) for sha256_final
    nrf_sw_backend_hash.o(i.nrf_sw_backend_hash_sha256_init) refers to sha256.o(i.sha256_init) for sha256_init
    nrf_sw_backend_hash.o(i.nrf_sw_backend_hash_sha256_update) refers to sha256.o(i.sha256_update) for sha256_update
    nrf_sw_backend_hash.o(.constdata) refers to nrf_sw_backend_hash.o(i.nrf_sw_backend_hash_sha256_init) for nrf_sw_backend_hash_sha256_init
    nrf_sw_backend_hash.o(.constdata) refers to nrf_sw_backend_hash.o(i.nrf_sw_backend_hash_sha256_update) for nrf_sw_backend_hash_sha256_update
    nrf_sw_backend_hash.o(.constdata) refers to nrf_sw_backend_hash.o(i.nrf_sw_backend_hash_sha256_finalize) for nrf_sw_backend_hash_sha256_finalize
    micro_ecc_backend_ecc.o(i.nrf_crypto_backend_micro_ecc_key_pair_generate) refers to micro_ecc_backend_ecc.o(i.nrf_crypto_backend_micro_ecc_curve_get) for nrf_crypto_backend_micro_ecc_curve_get
    micro_ecc_backend_ecc.o(i.nrf_crypto_backend_micro_ecc_key_pair_generate) refers to uECC.c.o(.text.uECC_set_rng) for uECC_set_rng
    micro_ecc_backend_ecc.o(i.nrf_crypto_backend_micro_ecc_key_pair_generate) refers to uECC.c.o(.text.uECC_make_key) for uECC_make_key
    micro_ecc_backend_ecc.o(i.nrf_crypto_backend_micro_ecc_key_pair_generate) refers to micro_ecc_backend_ecc.o(i.nrf_crypto_backend_micro_ecc_rng_callback) for nrf_crypto_backend_micro_ecc_rng_callback
    micro_ecc_backend_ecc.o(i.nrf_crypto_backend_micro_ecc_private_key_from_raw) refers to nrf_crypto_shared.o(i.nrf_crypto_internal_swap_endian) for nrf_crypto_internal_swap_endian
    micro_ecc_backend_ecc.o(i.nrf_crypto_backend_micro_ecc_private_key_to_raw) refers to nrf_crypto_shared.o(i.nrf_crypto_internal_swap_endian) for nrf_crypto_internal_swap_endian
    micro_ecc_backend_ecc.o(i.nrf_crypto_backend_micro_ecc_public_key_calculate) refers to micro_ecc_backend_ecc.o(i.nrf_crypto_backend_micro_ecc_curve_get) for nrf_crypto_backend_micro_ecc_curve_get
    micro_ecc_backend_ecc.o(i.nrf_crypto_backend_micro_ecc_public_key_calculate) refers to uECC.c.o(.text.uECC_compute_public_key) for uECC_compute_public_key
    micro_ecc_backend_ecc.o(i.nrf_crypto_backend_micro_ecc_public_key_from_raw) refers to nrf_crypto_shared.o(i.nrf_crypto_internal_double_swap_endian) for nrf_crypto_internal_double_swap_endian
    micro_ecc_backend_ecc.o(i.nrf_crypto_backend_micro_ecc_public_key_to_raw) refers to nrf_crypto_shared.o(i.nrf_crypto_internal_double_swap_endian) for nrf_crypto_internal_double_swap_endian
    micro_ecc_backend_ecc.o(.constdata) refers to uECC.c.o(.text.uECC_secp256r1) for uECC_secp256r1
    micro_ecc_backend_ecdh.o(i.nrf_crypto_backend_micro_ecc_ecdh_compute) refers to micro_ecc_backend_ecc.o(i.nrf_crypto_backend_micro_ecc_curve_get) for nrf_crypto_backend_micro_ecc_curve_get
    micro_ecc_backend_ecdh.o(i.nrf_crypto_backend_micro_ecc_ecdh_compute) refers to uECC.c.o(.text.uECC_valid_public_key) for uECC_valid_public_key
    micro_ecc_backend_ecdh.o(i.nrf_crypto_backend_micro_ecc_ecdh_compute) refers to uECC.c.o(.text.uECC_shared_secret) for uECC_shared_secret
    micro_ecc_backend_ecdh.o(i.nrf_crypto_backend_micro_ecc_ecdh_compute) refers to nrf_crypto_shared.o(i.nrf_crypto_internal_swap_endian_in_place) for nrf_crypto_internal_swap_endian_in_place
    micro_ecc_backend_ecdsa.o(i.nrf_crypto_backend_micro_ecc_sign) refers to micro_ecc_backend_ecc.o(i.nrf_crypto_backend_micro_ecc_curve_get) for nrf_crypto_backend_micro_ecc_curve_get
    micro_ecc_backend_ecdsa.o(i.nrf_crypto_backend_micro_ecc_sign) refers to nrf_crypto_shared.o(i.nrf_crypto_internal_swap_endian) for nrf_crypto_internal_swap_endian
    micro_ecc_backend_ecdsa.o(i.nrf_crypto_backend_micro_ecc_sign) refers to uECC.c.o(.text.uECC_set_rng) for uECC_set_rng
    micro_ecc_backend_ecdsa.o(i.nrf_crypto_backend_micro_ecc_sign) refers to uECC.c.o(.text.uECC_sign) for uECC_sign
    micro_ecc_backend_ecdsa.o(i.nrf_crypto_backend_micro_ecc_sign) refers to nrf_crypto_shared.o(i.nrf_crypto_internal_double_swap_endian_in_place) for nrf_crypto_internal_double_swap_endian_in_place
    micro_ecc_backend_ecdsa.o(i.nrf_crypto_backend_micro_ecc_sign) refers to micro_ecc_backend_ecc.o(i.nrf_crypto_backend_micro_ecc_rng_callback) for nrf_crypto_backend_micro_ecc_rng_callback
    micro_ecc_backend_ecdsa.o(i.nrf_crypto_backend_micro_ecc_verify) refers to micro_ecc_backend_ecc.o(i.nrf_crypto_backend_micro_ecc_curve_get) for nrf_crypto_backend_micro_ecc_curve_get
    micro_ecc_backend_ecdsa.o(i.nrf_crypto_backend_micro_ecc_verify) refers to nrf_crypto_shared.o(i.nrf_crypto_internal_swap_endian) for nrf_crypto_internal_swap_endian
    micro_ecc_backend_ecdsa.o(i.nrf_crypto_backend_micro_ecc_verify) refers to nrf_crypto_shared.o(i.nrf_crypto_internal_double_swap_endian) for nrf_crypto_internal_double_swap_endian
    micro_ecc_backend_ecdsa.o(i.nrf_crypto_backend_micro_ecc_verify) refers to uECC.c.o(.text.uECC_verify) for uECC_verify
    dfu-cc.pb.o(.constdata) refers to dfu-cc.pb.o(.constdata) for dfu_hash_fields
    dfu-cc.pb.o(.constdata) refers to dfu-cc.pb.o(.constdata) for dfu_init_command_is_debug_default
    dfu-cc.pb.o(.constdata) refers to dfu-cc.pb.o(.constdata) for dfu_boot_validation_fields
    dfu-cc.pb.o(.constdata) refers to dfu-cc.pb.o(.constdata) for dfu_init_command_fields
    dfu-cc.pb.o(.constdata) refers to dfu-cc.pb.o(.constdata) for dfu_command_fields
    dfu-cc.pb.o(.constdata) refers to dfu-cc.pb.o(.constdata) for dfu_command_fields
    dfu-cc.pb.o(.constdata) refers to dfu-cc.pb.o(.constdata) for dfu_signed_command_fields
    nrf_dfu.o(i.dfu_observer) refers to nrf_dfu_transport.o(i.nrf_dfu_transports_close) for nrf_dfu_transports_close
    nrf_dfu.o(i.dfu_observer) refers to nrf_dfu.o(.data) for .data
    nrf_dfu.o(i.nrf_dfu_init) refers to nrf_dfu.o(i.dfu_observer) for dfu_observer
    nrf_dfu.o(i.nrf_dfu_init) refers to nrf_dfu_transport.o(i.nrf_dfu_transports_init) for nrf_dfu_transports_init
    nrf_dfu.o(i.nrf_dfu_init) refers to nrf_dfu_req_handler.o(i.nrf_dfu_req_handler_init) for nrf_dfu_req_handler_init
    nrf_dfu.o(i.nrf_dfu_init) refers to nrf_dfu.o(.data) for .data
    nrf_dfu_flash.o(i.nrf_dfu_flash_erase) refers to nrf_fstorage.o(i.nrf_fstorage_erase) for nrf_fstorage_erase
    nrf_dfu_flash.o(i.nrf_dfu_flash_erase) refers to nrf_dfu_flash.o(fs_data) for fs_data
    nrf_dfu_flash.o(i.nrf_dfu_flash_init) refers to nrf_fstorage.o(i.nrf_fstorage_init) for nrf_fstorage_init
    nrf_dfu_flash.o(i.nrf_dfu_flash_init) refers to nrf_fstorage_nvmc.o(.constdata) for nrf_fstorage_nvmc
    nrf_dfu_flash.o(i.nrf_dfu_flash_init) refers to nrf_dfu_flash.o(fs_data) for fs_data
    nrf_dfu_flash.o(i.nrf_dfu_flash_store) refers to nrf_fstorage.o(i.nrf_fstorage_write) for nrf_fstorage_write
    nrf_dfu_flash.o(i.nrf_dfu_flash_store) refers to nrf_dfu_flash.o(fs_data) for fs_data
    nrf_dfu_flash.o(fs_data) refers to nrf_dfu_flash.o(i.dfu_fstorage_evt_handler) for dfu_fstorage_evt_handler
    nrf_dfu_handling_error.o(i.ext_error_get) refers to nrf_dfu_handling_error.o(.data) for .data
    nrf_dfu_handling_error.o(i.ext_error_set) refers to nrf_dfu_handling_error.o(.data) for .data
    nrf_dfu_mbr.o(i.nrf_dfu_mbr_init_sd) refers to nrf_dfu_mbr.o(.constdata) for .constdata
    nrf_dfu_mbr.o(i.nrf_dfu_mbr_irq_forward_address_set) refers to nrf_dfu_mbr.o(.constdata) for .constdata
    nrf_dfu_req_handler.o(i.cmd_response_offset_and_crc_set) refers to nrf_dfu_settings.o(.bss) for s_dfu_settings
    nrf_dfu_req_handler.o(i.ext_err_code_handle) refers to nrf_dfu_handling_error.o(i.ext_error_set) for ext_error_set
    nrf_dfu_req_handler.o(i.nrf_dfu_command_req) refers to nrf_dfu_validation.o(i.nrf_dfu_validation_init_cmd_create) for nrf_dfu_validation_init_cmd_create
    nrf_dfu_req_handler.o(i.nrf_dfu_command_req) refers to nrf_dfu_req_handler.o(i.ext_err_code_handle) for ext_err_code_handle
    nrf_dfu_req_handler.o(i.nrf_dfu_command_req) refers to nrf_dfu_validation.o(i.nrf_dfu_validation_init_cmd_append) for nrf_dfu_validation_init_cmd_append
    nrf_dfu_req_handler.o(i.nrf_dfu_command_req) refers to nrf_dfu_req_handler.o(i.cmd_response_offset_and_crc_set) for cmd_response_offset_and_crc_set
    nrf_dfu_req_handler.o(i.nrf_dfu_command_req) refers to nrf_dfu_validation.o(i.nrf_dfu_validation_init_cmd_execute) for nrf_dfu_validation_init_cmd_execute
    nrf_dfu_req_handler.o(i.nrf_dfu_command_req) refers to nrf_dfu_settings.o(i.nrf_dfu_settings_write_and_backup) for nrf_dfu_settings_write_and_backup
    nrf_dfu_req_handler.o(i.nrf_dfu_command_req) refers to nrf_dfu_req_handler.o(.data) for .data
    nrf_dfu_req_handler.o(i.nrf_dfu_data_req) refers to nrf_dfu_req_handler.o(i.on_data_obj_create_request) for on_data_obj_create_request
    nrf_dfu_req_handler.o(i.nrf_dfu_data_req) refers to nrf_dfu_req_handler.o(i.on_data_obj_write_request) for on_data_obj_write_request
    nrf_dfu_req_handler.o(i.nrf_dfu_data_req) refers to nrf_dfu_req_handler.o(i.on_data_obj_execute_request_sched) for on_data_obj_execute_request_sched
    nrf_dfu_req_handler.o(i.nrf_dfu_data_req) refers to nrf_dfu_settings.o(.bss) for s_dfu_settings
    nrf_dfu_req_handler.o(i.nrf_dfu_data_req) refers to nrf_dfu_req_handler.o(.data) for .data
    nrf_dfu_req_handler.o(i.nrf_dfu_req_handler_init) refers to nrf_dfu_flash.o(i.nrf_dfu_flash_init) for nrf_dfu_flash_init
    nrf_dfu_req_handler.o(i.nrf_dfu_req_handler_init) refers to nrf_dfu_validation.o(i.nrf_dfu_validation_init) for nrf_dfu_validation_init
    nrf_dfu_req_handler.o(i.nrf_dfu_req_handler_init) refers to nrf_dfu_validation.o(i.nrf_dfu_validation_init_cmd_present) for nrf_dfu_validation_init_cmd_present
    nrf_dfu_req_handler.o(i.nrf_dfu_req_handler_init) refers to nrf_dfu_validation.o(i.nrf_dfu_validation_init_cmd_execute) for nrf_dfu_validation_init_cmd_execute
    nrf_dfu_req_handler.o(i.nrf_dfu_req_handler_init) refers to nrf_dfu_handling_error.o(i.ext_error_set) for ext_error_set
    nrf_dfu_req_handler.o(i.nrf_dfu_req_handler_init) refers to nrf_dfu_req_handler.o(.data) for .data
    nrf_dfu_req_handler.o(i.nrf_dfu_req_handler_on_req) refers to app_scheduler.o(i.app_sched_event_put) for app_sched_event_put
    nrf_dfu_req_handler.o(i.nrf_dfu_req_handler_on_req) refers to nrf_dfu_req_handler.o(i.nrf_dfu_req_handler_req) for nrf_dfu_req_handler_req
    nrf_dfu_req_handler.o(i.nrf_dfu_req_handler_req) refers to nrf_dfu_req_handler.o(i.nrf_dfu_req_handler_req_process) for nrf_dfu_req_handler_req_process
    nrf_dfu_req_handler.o(i.nrf_dfu_req_handler_req_process) refers to memcpya.o(.text) for __aeabi_memcpy4
    nrf_dfu_req_handler.o(i.nrf_dfu_req_handler_req_process) refers to nrf_dfu_req_handler.o(i.on_fw_version_request) for on_fw_version_request
    nrf_dfu_req_handler.o(i.nrf_dfu_req_handler_req_process) refers to nrf_dfu_req_handler.o(i.nrf_dfu_command_req) for nrf_dfu_command_req
    nrf_dfu_req_handler.o(i.nrf_dfu_req_handler_req_process) refers to nrf_dfu_req_handler.o(i.nrf_dfu_data_req) for nrf_dfu_data_req
    nrf_dfu_req_handler.o(i.nrf_dfu_req_handler_req_process) refers to nrf_dfu_req_handler.o(.constdata) for .constdata
    nrf_dfu_req_handler.o(i.nrf_dfu_req_handler_req_process) refers to nrf_dfu_req_handler.o(.data) for .data
    nrf_dfu_req_handler.o(i.on_data_obj_create_request) refers to nrf_dfu_validation.o(i.nrf_dfu_validation_init_cmd_present) for nrf_dfu_validation_init_cmd_present
    nrf_dfu_req_handler.o(i.on_data_obj_create_request) refers to nrf_dfu_flash.o(i.nrf_dfu_flash_erase) for nrf_dfu_flash_erase
    nrf_dfu_req_handler.o(i.on_data_obj_create_request) refers to nrf_dfu_settings.o(.bss) for s_dfu_settings
    nrf_dfu_req_handler.o(i.on_data_obj_create_request) refers to nrf_dfu_req_handler.o(.data) for .data
    nrf_dfu_req_handler.o(i.on_data_obj_execute_request_sched) refers to nrf_fstorage.o(i.nrf_fstorage_is_busy) for nrf_fstorage_is_busy
    nrf_dfu_req_handler.o(i.on_data_obj_execute_request_sched) refers to app_scheduler.o(i.app_sched_event_put) for app_sched_event_put
    nrf_dfu_req_handler.o(i.on_data_obj_execute_request_sched) refers to memcpya.o(.text) for __aeabi_memcpy4
    nrf_dfu_req_handler.o(i.on_data_obj_execute_request_sched) refers to nrf_dfu_validation.o(i.nrf_dfu_validation_activation_prepare) for nrf_dfu_validation_activation_prepare
    nrf_dfu_req_handler.o(i.on_data_obj_execute_request_sched) refers to nrf_dfu_req_handler.o(i.ext_err_code_handle) for ext_err_code_handle
    nrf_dfu_req_handler.o(i.on_data_obj_execute_request_sched) refers to nrf_dfu_settings.o(i.nrf_dfu_settings_write_and_backup) for nrf_dfu_settings_write_and_backup
    nrf_dfu_req_handler.o(i.on_data_obj_execute_request_sched) refers to nrf_dfu_req_handler.o(.constdata) for .constdata
    nrf_dfu_req_handler.o(i.on_data_obj_execute_request_sched) refers to nrf_dfu_settings.o(.bss) for s_dfu_settings
    nrf_dfu_req_handler.o(i.on_data_obj_execute_request_sched) refers to nrf_dfu_req_handler.o(.data) for .data
    nrf_dfu_req_handler.o(i.on_data_obj_execute_request_sched) refers to nrf_dfu_req_handler.o(i.on_dfu_complete) for on_dfu_complete
    nrf_dfu_req_handler.o(i.on_data_obj_write_request) refers to nrf_dfu_validation.o(i.nrf_dfu_validation_init_cmd_present) for nrf_dfu_validation_init_cmd_present
    nrf_dfu_req_handler.o(i.on_data_obj_write_request) refers to crc32.o(i.crc32_compute) for crc32_compute
    nrf_dfu_req_handler.o(i.on_data_obj_write_request) refers to nrf_dfu_flash.o(i.nrf_dfu_flash_store) for nrf_dfu_flash_store
    nrf_dfu_req_handler.o(i.on_data_obj_write_request) refers to nrf_dfu_settings.o(.bss) for s_dfu_settings
    nrf_dfu_req_handler.o(i.on_data_obj_write_request) refers to nrf_dfu_req_handler.o(.data) for .data
    nrf_dfu_req_handler.o(i.on_dfu_complete) refers to nrf_dfu_req_handler.o(.data) for .data
    nrf_dfu_req_handler.o(i.on_fw_version_request) refers to nrf_dfu_utils.o(i.nrf_dfu_app_start_address) for nrf_dfu_app_start_address
    nrf_dfu_req_handler.o(i.on_fw_version_request) refers to nrf_dfu_settings.o(.bss) for s_dfu_settings
    nrf_dfu_serial_uart.o(i.nrf_drv_uart_rx) refers to nrfx_uarte.o(i.nrfx_uarte_rx) for nrfx_uarte_rx
    nrf_dfu_serial_uart.o(i.payload_free) refers to nrf_balloc.o(i.nrf_balloc_free) for nrf_balloc_free
    nrf_dfu_serial_uart.o(i.payload_free) refers to nrf_dfu_serial_uart.o(nrf_balloc) for nrf_balloc
    nrf_dfu_serial_uart.o(i.rsp_send) refers to slip.o(i.slip_encode) for slip_encode
    nrf_dfu_serial_uart.o(i.rsp_send) refers to nrfx_uarte.o(i.nrfx_uarte_tx) for nrfx_uarte_tx
    nrf_dfu_serial_uart.o(i.rsp_send) refers to nrf_dfu_serial_uart.o(.bss) for .bss
    nrf_dfu_serial_uart.o(i.rsp_send) refers to nrf_dfu_serial_uart.o(.data) for .data
    nrf_dfu_serial_uart.o(i.uart_dfu_transport_close) refers to nrfx_uarte.o(i.nrfx_uarte_uninit) for nrfx_uarte_uninit
    nrf_dfu_serial_uart.o(i.uart_dfu_transport_close) refers to nrf_dfu_serial_uart.o(.data) for .data
    nrf_dfu_serial_uart.o(i.uart_dfu_transport_close) refers to nrf_dfu_serial_uart.o(dfu_trans) for dfu_trans
    nrf_dfu_serial_uart.o(i.uart_dfu_transport_init) refers to nrf_balloc.o(i.nrf_balloc_init) for nrf_balloc_init
    nrf_dfu_serial_uart.o(i.uart_dfu_transport_init) refers to nrf_balloc.o(i.nrf_balloc_alloc) for nrf_balloc_alloc
    nrf_dfu_serial_uart.o(i.uart_dfu_transport_init) refers to memcpya.o(.text) for __aeabi_memcpy4
    nrf_dfu_serial_uart.o(i.uart_dfu_transport_init) refers to nrf_drv_uart.o(i.nrf_drv_uart_init) for nrf_drv_uart_init
    nrf_dfu_serial_uart.o(i.uart_dfu_transport_init) refers to nrf_dfu_serial_uart.o(i.nrf_drv_uart_rx) for nrf_drv_uart_rx
    nrf_dfu_serial_uart.o(i.uart_dfu_transport_init) refers to nrf_dfu_serial_uart.o(.data) for .data
    nrf_dfu_serial_uart.o(i.uart_dfu_transport_init) refers to nrf_dfu_serial_uart.o(nrf_balloc) for nrf_balloc
    nrf_dfu_serial_uart.o(i.uart_dfu_transport_init) refers to nrf_dfu_serial_uart.o(.bss) for .bss
    nrf_dfu_serial_uart.o(i.uart_dfu_transport_init) refers to nrf_dfu_serial_uart.o(i.rsp_send) for rsp_send
    nrf_dfu_serial_uart.o(i.uart_dfu_transport_init) refers to nrf_dfu_serial_uart.o(i.payload_free) for payload_free
    nrf_dfu_serial_uart.o(i.uart_dfu_transport_init) refers to nrf_dfu_serial_uart.o(dfu_trans) for dfu_trans
    nrf_dfu_serial_uart.o(i.uart_dfu_transport_init) refers to nrf_dfu_serial_uart.o(.constdata) for .constdata
    nrf_dfu_serial_uart.o(i.uart_dfu_transport_init) refers to nrf_dfu_serial_uart.o(i.uart_event_handler) for uart_event_handler
    nrf_dfu_serial_uart.o(i.uart_event_handler) refers to main.o(i.app_error_handler_bare) for app_error_handler_bare
    nrf_dfu_serial_uart.o(i.uart_event_handler) refers to slip.o(i.slip_decode_add_byte) for slip_decode_add_byte
    nrf_dfu_serial_uart.o(i.uart_event_handler) refers to nrf_dfu_serial_uart.o(i.nrf_drv_uart_rx) for nrf_drv_uart_rx
    nrf_dfu_serial_uart.o(i.uart_event_handler) refers to nrf_dfu_serial.o(i.nrf_dfu_serial_on_packet_received) for nrf_dfu_serial_on_packet_received
    nrf_dfu_serial_uart.o(i.uart_event_handler) refers to nrf_balloc.o(i.nrf_balloc_alloc) for nrf_balloc_alloc
    nrf_dfu_serial_uart.o(i.uart_event_handler) refers to nrf_dfu_serial_uart.o(.bss) for .bss
    nrf_dfu_serial_uart.o(i.uart_event_handler) refers to nrf_dfu_serial_uart.o(.data) for .data
    nrf_dfu_serial_uart.o(i.uart_event_handler) refers to nrf_dfu_serial_uart.o(nrf_balloc) for nrf_balloc
    nrf_dfu_serial_uart.o(dfu_trans) refers to nrf_dfu_serial_uart.o(i.uart_dfu_transport_init) for uart_dfu_transport_init
    nrf_dfu_serial_uart.o(dfu_trans) refers to nrf_dfu_serial_uart.o(i.uart_dfu_transport_close) for uart_dfu_transport_close
    nrf_dfu_serial_uart.o(nrf_balloc) refers to nrf_dfu_serial_uart.o(.data) for m_payload_pool_nrf_balloc_cb
    nrf_dfu_serial_uart.o(nrf_balloc) refers to nrf_dfu_serial_uart.o(.data) for m_payload_pool_nrf_balloc_pool_stack
    nrf_dfu_serial_uart.o(nrf_balloc) refers to nrf_dfu_serial_uart.o(.bss) for m_payload_pool_nrf_balloc_pool_mem
    nrf_dfu_settings.o(i.boot_validation_crc) refers to crc32.o(i.crc32_compute) for crc32_compute
    nrf_dfu_settings.o(i.crc_ok) refers to nrf_dfu_settings.o(i.settings_crc_get) for settings_crc_get
    nrf_dfu_settings.o(i.nrf_dfu_settings_backup) refers to nrf_dfu_settings.o(i.settings_backup) for settings_backup
    nrf_dfu_settings.o(i.nrf_dfu_settings_backup) refers to nrf_dfu_settings.o(.ARM.__AT_0x0003F000) for .ARM.__AT_0x0003F000
    nrf_dfu_settings.o(i.nrf_dfu_settings_init) refers to nrf_dfu_flash.o(i.nrf_dfu_flash_init) for nrf_dfu_flash_init
    nrf_dfu_settings.o(i.nrf_dfu_settings_init) refers to nrf_dfu_settings.o(i.nrf_dfu_settings_reinit) for nrf_dfu_settings_reinit
    nrf_dfu_settings.o(i.nrf_dfu_settings_init) refers to nrf_dfu_settings.o(i.nrf_dfu_settings_write_and_backup) for nrf_dfu_settings_write_and_backup
    nrf_dfu_settings.o(i.nrf_dfu_settings_progress_reset) refers to memseta.o(.text) for __aeabi_memset
    nrf_dfu_settings.o(i.nrf_dfu_settings_progress_reset) refers to nrf_dfu_settings.o(.bss) for .bss
    nrf_dfu_settings.o(i.nrf_dfu_settings_reinit) refers to nrf_dfu_settings.o(i.crc_ok) for crc_ok
    nrf_dfu_settings.o(i.nrf_dfu_settings_reinit) refers to nrf_dfu_settings.o(i.boot_validation_crc) for boot_validation_crc
    nrf_dfu_settings.o(i.nrf_dfu_settings_reinit) refers to memcpya.o(.text) for __aeabi_memcpy
    nrf_dfu_settings.o(i.nrf_dfu_settings_reinit) refers to memseta.o(.text) for __aeabi_memclr4
    nrf_dfu_settings.o(i.nrf_dfu_settings_reinit) refers to nrf_dfu_settings.o(.ARM.__AT_0x0003F000) for .ARM.__AT_0x0003F000
    nrf_dfu_settings.o(i.nrf_dfu_settings_reinit) refers to nrf_dfu_settings.o(.data) for .data
    nrf_dfu_settings.o(i.nrf_dfu_settings_reinit) refers to nrf_dfu_settings.o(.bss) for .bss
    nrf_dfu_settings.o(i.nrf_dfu_settings_write) refers to nrf_dfu_settings.o(i.settings_crc_get) for settings_crc_get
    nrf_dfu_settings.o(i.nrf_dfu_settings_write) refers to nrf_dfu_settings.o(i.boot_validation_crc) for boot_validation_crc
    nrf_dfu_settings.o(i.nrf_dfu_settings_write) refers to nrf_dfu_settings.o(i.settings_write) for settings_write
    nrf_dfu_settings.o(i.nrf_dfu_settings_write) refers to nrf_dfu_settings.o(.bss) for .bss
    nrf_dfu_settings.o(i.nrf_dfu_settings_write) refers to nrf_dfu_settings.o(.ARM.__AT_0x0003F000) for .ARM.__AT_0x0003F000
    nrf_dfu_settings.o(i.nrf_dfu_settings_write_and_backup) refers to nrf_dfu_settings.o(i.nrf_dfu_settings_write) for nrf_dfu_settings_write
    nrf_dfu_settings.o(i.nrf_dfu_settings_write_and_backup) refers to nrf_dfu_settings.o(i.settings_backup) for settings_backup
    nrf_dfu_settings.o(i.nrf_dfu_settings_write_and_backup) refers to nrf_dfu_settings.o(.bss) for .bss
    nrf_dfu_settings.o(i.settings_backup) refers to nrf_dfu_settings.o(i.settings_write) for settings_write
    nrf_dfu_settings.o(i.settings_backup) refers to nrf_dfu_settings.o(.bss) for .bss
    nrf_dfu_settings.o(i.settings_backup) refers to nrf_dfu_settings.o(.data) for .data
    nrf_dfu_settings.o(i.settings_crc_get) refers to crc32.o(i.crc32_compute) for crc32_compute
    nrf_dfu_settings.o(i.settings_write) refers to memcmp.o(.text) for memcmp
    nrf_dfu_settings.o(i.settings_write) refers to nrf_dfu_flash.o(i.nrf_dfu_flash_erase) for nrf_dfu_flash_erase
    nrf_dfu_settings.o(i.settings_write) refers to memcpya.o(.text) for __aeabi_memcpy
    nrf_dfu_settings.o(i.settings_write) refers to nrf_dfu_flash.o(i.nrf_dfu_flash_store) for nrf_dfu_flash_store
    nrf_dfu_settings.o(.data) refers to nrf_dfu_settings.o(.ARM.__AT_0x0003E000) for m_mbr_params_page
    nrf_dfu_utils.o(i.nrf_dfu_app_start_address) refers to nrf_dfu_utils.o(i.nrf_dfu_bank0_start_addr) for nrf_dfu_bank0_start_addr
    nrf_dfu_utils.o(i.nrf_dfu_bank1_start_addr) refers to nrf_dfu_utils.o(i.nrf_dfu_bank0_start_addr) for nrf_dfu_bank0_start_addr
    nrf_dfu_utils.o(i.nrf_dfu_bank1_start_addr) refers to nrf_dfu_settings.o(.bss) for s_dfu_settings
    nrf_dfu_utils.o(i.nrf_dfu_bank_invalidate) refers to nrf_dfu_settings.o(.bss) for s_dfu_settings
    nrf_dfu_utils.o(i.nrf_dfu_cache_prepare) refers to nrf_dfu_utils.o(i.nrf_dfu_bank1_start_addr) for nrf_dfu_bank1_start_addr
    nrf_dfu_utils.o(i.nrf_dfu_cache_prepare) refers to nrf_dfu_utils.o(i.nrf_dfu_bank0_start_addr) for nrf_dfu_bank0_start_addr
    nrf_dfu_utils.o(i.nrf_dfu_cache_prepare) refers to nrf_dfu_utils.o(i.nrf_dfu_softdevice_invalidate) for nrf_dfu_softdevice_invalidate
    nrf_dfu_utils.o(i.nrf_dfu_cache_prepare) refers to nrf_dfu_utils.o(i.nrf_dfu_bank_invalidate) for nrf_dfu_bank_invalidate
    nrf_dfu_utils.o(i.nrf_dfu_cache_prepare) refers to nrf_dfu_settings.o(.bss) for s_dfu_settings
    nrf_dfu_utils.o(i.nrf_dfu_softdevice_invalidate) refers to nrf_dfu_flash.o(i.nrf_dfu_flash_store) for nrf_dfu_flash_store
    nrf_dfu_utils.o(i.nrf_dfu_softdevice_invalidate) refers to nrf_dfu_utils.o(.constdata) for .constdata
    nrf_dfu_utils.o(i.nrf_dfu_softdevice_invalidate) refers to nrf_dfu_settings.o(.bss) for s_dfu_settings
    nrf_dfu_validation.o(i.boot_validation_extract) refers to memseta.o(.text) for __aeabi_memclr4
    nrf_dfu_validation.o(i.boot_validation_extract) refers to crc32.o(i.crc32_compute) for crc32_compute
    nrf_dfu_validation.o(i.boot_validation_extract) refers to nrf_crypto_hash.o(i.nrf_crypto_hash_calculate) for nrf_crypto_hash_calculate
    nrf_dfu_validation.o(i.boot_validation_extract) refers to memcpya.o(.text) for __aeabi_memcpy
    nrf_dfu_validation.o(i.boot_validation_extract) refers to nrf_dfu_validation.o(i.nrf_dfu_validation_boot_validate) for nrf_dfu_validation_boot_validate
    nrf_dfu_validation.o(i.boot_validation_extract) refers to nrf_sw_backend_hash.o(.constdata) for g_nrf_crypto_hash_sha256_info
    nrf_dfu_validation.o(i.crypto_init) refers to nrf_crypto_init.o(i.nrf_crypto_init) for nrf_crypto_init
    nrf_dfu_validation.o(i.crypto_init) refers to nrf_crypto_shared.o(i.nrf_crypto_internal_double_swap_endian) for nrf_crypto_internal_double_swap_endian
    nrf_dfu_validation.o(i.crypto_init) refers to nrf_crypto_ecc.o(i.nrf_crypto_ecc_public_key_from_raw) for nrf_crypto_ecc_public_key_from_raw
    nrf_dfu_validation.o(i.crypto_init) refers to nrf_dfu_validation.o(.data) for .data
    nrf_dfu_validation.o(i.crypto_init) refers to dfu_public_key.o(.constdata) for pk
    nrf_dfu_validation.o(i.crypto_init) refers to nrf_dfu_validation.o(.bss) for .bss
    nrf_dfu_validation.o(i.crypto_init) refers to micro_ecc_backend_ecc.o(.constdata) for g_nrf_crypto_ecc_secp256r1_curve_info
    nrf_dfu_validation.o(i.fw_hash_ok) refers to nrf_dfu_validation.o(i.nrf_dfu_validation_hash_ok) for nrf_dfu_validation_hash_ok
    nrf_dfu_validation.o(i.nrf_dfu_validation_activation_prepare) refers to nrf_dfu_validation.o(i.postvalidate) for postvalidate
    nrf_dfu_validation.o(i.nrf_dfu_validation_boot_validate) refers to crc32.o(i.crc32_compute) for crc32_compute
    nrf_dfu_validation.o(i.nrf_dfu_validation_boot_validate) refers to nrf_dfu_validation.o(i.nrf_dfu_validation_hash_ok) for nrf_dfu_validation_hash_ok
    nrf_dfu_validation.o(i.nrf_dfu_validation_boot_validate) refers to nrf_dfu_validation.o(i.nrf_dfu_validation_signature_check) for nrf_dfu_validation_signature_check
    nrf_dfu_validation.o(i.nrf_dfu_validation_hash_ok) refers to memseta.o(.text) for __aeabi_memclr4
    nrf_dfu_validation.o(i.nrf_dfu_validation_hash_ok) refers to nrf_dfu_validation.o(i.crypto_init) for crypto_init
    nrf_dfu_validation.o(i.nrf_dfu_validation_hash_ok) refers to nrf_crypto_shared.o(i.nrf_crypto_internal_swap_endian) for nrf_crypto_internal_swap_endian
    nrf_dfu_validation.o(i.nrf_dfu_validation_hash_ok) refers to nrf_crypto_hash.o(i.nrf_crypto_hash_calculate) for nrf_crypto_hash_calculate
    nrf_dfu_validation.o(i.nrf_dfu_validation_hash_ok) refers to memcmp.o(.text) for memcmp
    nrf_dfu_validation.o(i.nrf_dfu_validation_hash_ok) refers to nrf_dfu_validation.o(.bss) for .bss
    nrf_dfu_validation.o(i.nrf_dfu_validation_hash_ok) refers to nrf_sw_backend_hash.o(.constdata) for g_nrf_crypto_hash_sha256_info
    nrf_dfu_validation.o(i.nrf_dfu_validation_init) refers to nrf_dfu_validation.o(i.stored_init_cmd_decode) for stored_init_cmd_decode
    nrf_dfu_validation.o(i.nrf_dfu_validation_init) refers to nrf_dfu_settings.o(.bss) for s_dfu_settings
    nrf_dfu_validation.o(i.nrf_dfu_validation_init) refers to nrf_dfu_validation.o(.data) for .data
    nrf_dfu_validation.o(i.nrf_dfu_validation_init_cmd_append) refers to memcpya.o(.text) for __aeabi_memcpy
    nrf_dfu_validation.o(i.nrf_dfu_validation_init_cmd_append) refers to crc32.o(i.crc32_compute) for crc32_compute
    nrf_dfu_validation.o(i.nrf_dfu_validation_init_cmd_append) refers to nrf_dfu_settings.o(.bss) for s_dfu_settings
    nrf_dfu_validation.o(i.nrf_dfu_validation_init_cmd_create) refers to nrf_dfu_settings.o(i.nrf_dfu_settings_progress_reset) for nrf_dfu_settings_progress_reset
    nrf_dfu_validation.o(i.nrf_dfu_validation_init_cmd_create) refers to nrf_dfu_validation.o(.data) for .data
    nrf_dfu_validation.o(i.nrf_dfu_validation_init_cmd_create) refers to nrf_dfu_settings.o(.bss) for s_dfu_settings
    nrf_dfu_validation.o(i.nrf_dfu_validation_init_cmd_execute) refers to nrf_dfu_utils.o(i.nrf_dfu_bank1_start_addr) for nrf_dfu_bank1_start_addr
    nrf_dfu_validation.o(i.nrf_dfu_validation_init_cmd_execute) refers to nrf_dfu_validation.o(i.update_data_size_get) for update_data_size_get
    nrf_dfu_validation.o(i.nrf_dfu_validation_init_cmd_execute) refers to nrf_dfu_validation.o(i.stored_init_cmd_decode) for stored_init_cmd_decode
    nrf_dfu_validation.o(i.nrf_dfu_validation_init_cmd_execute) refers to nrf_dfu_validation.o(i.nrf_dfu_validation_prevalidate) for nrf_dfu_validation_prevalidate
    nrf_dfu_validation.o(i.nrf_dfu_validation_init_cmd_execute) refers to nrf_dfu_validation.o(i.update_requires_softdevice) for update_requires_softdevice
    nrf_dfu_validation.o(i.nrf_dfu_validation_init_cmd_execute) refers to nrf_dfu_utils.o(i.nrf_dfu_cache_prepare) for nrf_dfu_cache_prepare
    nrf_dfu_validation.o(i.nrf_dfu_validation_init_cmd_execute) refers to nrf_dfu_settings.o(i.nrf_dfu_settings_progress_reset) for nrf_dfu_settings_progress_reset
    nrf_dfu_validation.o(i.nrf_dfu_validation_init_cmd_execute) refers to nrf_dfu_settings.o(.bss) for s_dfu_settings
    nrf_dfu_validation.o(i.nrf_dfu_validation_init_cmd_execute) refers to nrf_dfu_validation.o(.data) for .data
    nrf_dfu_validation.o(i.nrf_dfu_validation_init_cmd_present) refers to nrf_dfu_validation.o(.data) for .data
    nrf_dfu_validation.o(i.nrf_dfu_validation_init_cmd_status_get) refers to nrf_dfu_settings.o(.bss) for s_dfu_settings
    nrf_dfu_validation.o(i.nrf_dfu_validation_post_data_execute) refers to nrf_dfu_validation.o(i.postvalidate) for postvalidate
    nrf_dfu_validation.o(i.nrf_dfu_validation_prevalidate) refers to nrf_dfu_validation.o(i.nrf_dfu_validation_signature_check) for nrf_dfu_validation_signature_check
    nrf_dfu_validation.o(i.nrf_dfu_validation_prevalidate) refers to nrf_dfu_ver_validation.o(i.nrf_dfu_ver_validation_check) for nrf_dfu_ver_validation_check
    nrf_dfu_validation.o(i.nrf_dfu_validation_prevalidate) refers to nrf_dfu_validation.o(.bss) for .bss
    nrf_dfu_validation.o(i.nrf_dfu_validation_prevalidate) refers to nrf_dfu_validation.o(.data) for .data
    nrf_dfu_validation.o(i.nrf_dfu_validation_signature_check) refers to memseta.o(.text) for __aeabi_memclr4
    nrf_dfu_validation.o(i.nrf_dfu_validation_signature_check) refers to nrf_dfu_validation.o(i.crypto_init) for crypto_init
    nrf_dfu_validation.o(i.nrf_dfu_validation_signature_check) refers to nrf_crypto_hash.o(i.nrf_crypto_hash_calculate) for nrf_crypto_hash_calculate
    nrf_dfu_validation.o(i.nrf_dfu_validation_signature_check) refers to memcpya.o(.text) for __aeabi_memcpy
    nrf_dfu_validation.o(i.nrf_dfu_validation_signature_check) refers to nrf_crypto_shared.o(i.nrf_crypto_internal_double_swap_endian_in_place) for nrf_crypto_internal_double_swap_endian_in_place
    nrf_dfu_validation.o(i.nrf_dfu_validation_signature_check) refers to nrf_crypto_ecdsa.o(i.nrf_crypto_ecdsa_verify) for nrf_crypto_ecdsa_verify
    nrf_dfu_validation.o(i.nrf_dfu_validation_signature_check) refers to nrf_dfu_validation.o(.bss) for .bss
    nrf_dfu_validation.o(i.nrf_dfu_validation_signature_check) refers to nrf_sw_backend_hash.o(.constdata) for g_nrf_crypto_hash_sha256_info
    nrf_dfu_validation.o(i.nrf_dfu_validation_valid_external_app) refers to nrf_dfu_settings.o(.bss) for s_dfu_settings
    nrf_dfu_validation.o(i.pb_decoding_callback) refers to dfu-cc.pb.o(.constdata) for dfu_init_command_fields
    nrf_dfu_validation.o(i.pb_decoding_callback) refers to nrf_dfu_validation.o(.data) for .data
    nrf_dfu_validation.o(i.postvalidate) refers to nrf_dfu_validation.o(i.fw_hash_ok) for fw_hash_ok
    nrf_dfu_validation.o(i.postvalidate) refers to nrf_dfu_validation.o(i.postvalidate_sd_bl) for postvalidate_sd_bl
    nrf_dfu_validation.o(i.postvalidate) refers to nrf_dfu_validation.o(i.boot_validation_extract) for boot_validation_extract
    nrf_dfu_validation.o(i.postvalidate) refers to memcpya.o(.text) for __aeabi_memcpy
    nrf_dfu_validation.o(i.postvalidate) refers to nrf_dfu_validation.o(i.update_requires_softdevice) for update_requires_softdevice
    nrf_dfu_validation.o(i.postvalidate) refers to nrf_dfu_utils.o(i.nrf_dfu_softdevice_invalidate) for nrf_dfu_softdevice_invalidate
    nrf_dfu_validation.o(i.postvalidate) refers to nrf_dfu_utils.o(i.nrf_dfu_softdevice_start_address) for nrf_dfu_softdevice_start_address
    nrf_dfu_validation.o(i.postvalidate) refers to nrf_dfu_utils.o(i.nrf_dfu_bank_invalidate) for nrf_dfu_bank_invalidate
    nrf_dfu_validation.o(i.postvalidate) refers to nrf_dfu_settings.o(i.nrf_dfu_settings_progress_reset) for nrf_dfu_settings_progress_reset
    nrf_dfu_validation.o(i.postvalidate) refers to crc32.o(i.crc32_compute) for crc32_compute
    nrf_dfu_validation.o(i.postvalidate) refers to nrf_dfu_validation.o(.data) for .data
    nrf_dfu_validation.o(i.postvalidate) refers to nrf_dfu_settings.o(.bss) for s_dfu_settings
    nrf_dfu_validation.o(i.postvalidate_sd_bl) refers to memseta.o(.text) for __aeabi_memclr4
    nrf_dfu_validation.o(i.postvalidate_sd_bl) refers to nrf_dfu_validation.o(i.is_major_softdevice_update) for is_major_softdevice_update
    nrf_dfu_validation.o(i.postvalidate_sd_bl) refers to nrf_dfu_validation.o(i.boot_validation_extract) for boot_validation_extract
    nrf_dfu_validation.o(i.postvalidate_sd_bl) refers to nrf_dfu_utils.o(i.nrf_dfu_bank_invalidate) for nrf_dfu_bank_invalidate
    nrf_dfu_validation.o(i.postvalidate_sd_bl) refers to memcpya.o(.text) for __aeabi_memcpy4
    nrf_dfu_validation.o(i.postvalidate_sd_bl) refers to nrf_dfu_settings.o(.bss) for s_dfu_settings
    nrf_dfu_validation.o(i.stored_init_cmd_decode) refers to pb_decode.o(i.pb_istream_from_buffer) for pb_istream_from_buffer
    nrf_dfu_validation.o(i.stored_init_cmd_decode) refers to memseta.o(.text) for __aeabi_memclr4
    nrf_dfu_validation.o(i.stored_init_cmd_decode) refers to pb_decode.o(i.pb_decode) for pb_decode
    nrf_dfu_validation.o(i.stored_init_cmd_decode) refers to nrf_dfu_settings.o(.bss) for s_dfu_settings
    nrf_dfu_validation.o(i.stored_init_cmd_decode) refers to nrf_dfu_validation.o(.bss) for .bss
    nrf_dfu_validation.o(i.stored_init_cmd_decode) refers to nrf_dfu_validation.o(i.pb_decoding_callback) for pb_decoding_callback
    nrf_dfu_validation.o(i.stored_init_cmd_decode) refers to nrf_dfu_validation.o(.data) for .data
    nrf_dfu_validation.o(i.stored_init_cmd_decode) refers to dfu-cc.pb.o(.constdata) for dfu_packet_fields
    nrf_dfu_validation.o(i.stored_init_cmd_decode) refers to dfu-cc.pb.o(.constdata) for dfu_init_command_fields
    nrf_dfu_ver_validation.o(i.nrf_dfu_ver_validation_check) refers to nrf_dfu_ver_validation.o(i.sd_req_ok) for sd_req_ok
    nrf_dfu_ver_validation.o(i.nrf_dfu_ver_validation_check) refers to nrf_dfu_settings.o(.bss) for s_dfu_settings
    nrf_dfu_ver_validation.o(i.sd_req_ok) refers to nrf_dfu_ver_validation.o(i.sd_req_check) for sd_req_check
    nrf_drv_uart.o(i.nrf_drv_uart_init) refers to memcpya.o(.text) for __aeabi_memcpy4
    nrf_drv_uart.o(i.nrf_drv_uart_init) refers to nrfx_uarte.o(i.nrfx_uarte_init) for nrfx_uarte_init
    nrf_drv_uart.o(i.nrf_drv_uart_init) refers to nrf_drv_uart.o(.data) for .data
    nrf_drv_uart.o(i.nrf_drv_uart_init) refers to nrf_drv_uart.o(i.uarte_evt_handler) for uarte_evt_handler
    nrf_drv_uart.o(i.uarte_evt_handler) refers to nrf_drv_uart.o(.data) for .data
    nrf_nvic.o(i.sd_nvic_critical_region_enter) refers to nrf_nvic.o(.data) for .data
    nrf_nvic.o(i.sd_nvic_critical_region_exit) refers to nrf_nvic.o(.data) for .data
    nrf_nvmc.o(i.nrf_nvmc_write_bytes) refers to nrf_nvmc.o(i.nrf_nvmc_write_byte) for nrf_nvmc_write_byte
    nrfx_atomic.o(i.nrfx_atomic_flag_clear) refers to nrfx_atomic.o(i.nrfx_atomic_u32_and) for nrfx_atomic_u32_and
    nrfx_atomic.o(i.nrfx_atomic_flag_clear_fetch) refers to nrfx_atomic.o(i.nrfx_atomic_u32_fetch_and) for nrfx_atomic_u32_fetch_and
    nrfx_atomic.o(i.nrfx_atomic_flag_set) refers to nrfx_atomic.o(i.nrfx_atomic_u32_or) for nrfx_atomic_u32_or
    nrfx_atomic.o(i.nrfx_atomic_flag_set_fetch) refers to nrfx_atomic.o(i.nrfx_atomic_u32_fetch_or) for nrfx_atomic_u32_fetch_or
    nrfx_atomic.o(i.nrfx_atomic_u32_add) refers to nrfx_atomic.o(.emb_text) for __asm___13_nrfx_atomic_c_3bd32246__nrfx_atomic_internal_add
    nrfx_atomic.o(i.nrfx_atomic_u32_and) refers to nrfx_atomic.o(.emb_text) for __asm___13_nrfx_atomic_c_3bd32246__nrfx_atomic_internal_and
    nrfx_atomic.o(i.nrfx_atomic_u32_cmp_exch) refers to nrfx_atomic.o(.emb_text) for __asm___13_nrfx_atomic_c_3bd32246__nrfx_atomic_internal_cmp_exch
    nrfx_atomic.o(i.nrfx_atomic_u32_fetch_add) refers to nrfx_atomic.o(.emb_text) for __asm___13_nrfx_atomic_c_3bd32246__nrfx_atomic_internal_add
    nrfx_atomic.o(i.nrfx_atomic_u32_fetch_and) refers to nrfx_atomic.o(.emb_text) for __asm___13_nrfx_atomic_c_3bd32246__nrfx_atomic_internal_and
    nrfx_atomic.o(i.nrfx_atomic_u32_fetch_or) refers to nrfx_atomic.o(.emb_text) for __asm___13_nrfx_atomic_c_3bd32246__nrfx_atomic_internal_orr
    nrfx_atomic.o(i.nrfx_atomic_u32_fetch_store) refers to nrfx_atomic.o(.emb_text) for __asm___13_nrfx_atomic_c_3bd32246__nrfx_atomic_internal_mov
    nrfx_atomic.o(i.nrfx_atomic_u32_fetch_sub) refers to nrfx_atomic.o(.emb_text) for __asm___13_nrfx_atomic_c_3bd32246__nrfx_atomic_internal_sub
    nrfx_atomic.o(i.nrfx_atomic_u32_fetch_sub_hs) refers to nrfx_atomic.o(.emb_text) for __asm___13_nrfx_atomic_c_3bd32246__nrfx_atomic_internal_sub_hs
    nrfx_atomic.o(i.nrfx_atomic_u32_fetch_xor) refers to nrfx_atomic.o(.emb_text) for __asm___13_nrfx_atomic_c_3bd32246__nrfx_atomic_internal_eor
    nrfx_atomic.o(i.nrfx_atomic_u32_or) refers to nrfx_atomic.o(.emb_text) for __asm___13_nrfx_atomic_c_3bd32246__nrfx_atomic_internal_orr
    nrfx_atomic.o(i.nrfx_atomic_u32_store) refers to nrfx_atomic.o(.emb_text) for __asm___13_nrfx_atomic_c_3bd32246__nrfx_atomic_internal_mov
    nrfx_atomic.o(i.nrfx_atomic_u32_sub) refers to nrfx_atomic.o(.emb_text) for __asm___13_nrfx_atomic_c_3bd32246__nrfx_atomic_internal_sub
    nrfx_atomic.o(i.nrfx_atomic_u32_sub_hs) refers to nrfx_atomic.o(.emb_text) for __asm___13_nrfx_atomic_c_3bd32246__nrfx_atomic_internal_sub_hs
    nrfx_atomic.o(i.nrfx_atomic_u32_xor) refers to nrfx_atomic.o(.emb_text) for __asm___13_nrfx_atomic_c_3bd32246__nrfx_atomic_internal_eor
    nrfx_uarte.o(i.UARTE0_UART0_IRQHandler) refers to nrfx_uarte.o(i.uarte_irq_handler) for uarte_irq_handler
    nrfx_uarte.o(i.UARTE0_UART0_IRQHandler) refers to nrfx_uarte.o(.bss) for .bss
    nrfx_uarte.o(i.apply_config) refers to nrfx_uarte.o(i.nrf_gpio_cfg_output) for nrf_gpio_cfg_output
    nrfx_uarte.o(i.apply_config) refers to nrfx_uarte.o(i.nrf_gpio_cfg_input) for nrf_gpio_cfg_input
    nrfx_uarte.o(i.interrupts_enable) refers to nrfx_uarte.o(i.nrf_uarte_event_clear) for nrf_uarte_event_clear
    nrfx_uarte.o(i.nrf_gpio_cfg_default) refers to nrfx_uarte.o(i.nrf_gpio_cfg) for nrf_gpio_cfg
    nrfx_uarte.o(i.nrf_gpio_cfg_input) refers to nrfx_uarte.o(i.nrf_gpio_cfg) for nrf_gpio_cfg
    nrfx_uarte.o(i.nrf_gpio_cfg_output) refers to nrfx_uarte.o(i.nrf_gpio_cfg) for nrf_gpio_cfg
    nrfx_uarte.o(i.nrfx_uarte_errorsrc_get) refers to nrfx_uarte.o(i.nrf_uarte_event_clear) for nrf_uarte_event_clear
    nrfx_uarte.o(i.nrfx_uarte_init) refers to nrfx_prs.o(i.nrfx_prs_acquire) for nrfx_prs_acquire
    nrfx_uarte.o(i.nrfx_uarte_init) refers to nrfx_uarte.o(i.apply_config) for apply_config
    nrfx_uarte.o(i.nrfx_uarte_init) refers to nrfx_uarte.o(i.interrupts_enable) for interrupts_enable
    nrfx_uarte.o(i.nrfx_uarte_init) refers to nrfx_uarte.o(.bss) for .bss
    nrfx_uarte.o(i.nrfx_uarte_init) refers to nrfx_uarte.o(.constdata) for .constdata
    nrfx_uarte.o(i.nrfx_uarte_rx) refers to nrfx_uarte.o(i.nrfx_is_in_ram) for nrfx_is_in_ram
    nrfx_uarte.o(i.nrfx_uarte_rx) refers to nrfx_uarte.o(i.nrf_uarte_event_clear) for nrf_uarte_event_clear
    nrfx_uarte.o(i.nrfx_uarte_rx) refers to nrfx_uarte.o(i.nrf_uarte_event_check) for nrf_uarte_event_check
    nrfx_uarte.o(i.nrfx_uarte_rx) refers to nrfx_uarte.o(.bss) for .bss
    nrfx_uarte.o(i.nrfx_uarte_rx_abort) refers to nrfx_uarte.o(.bss) for .bss
    nrfx_uarte.o(i.nrfx_uarte_tx) refers to nrfx_uarte.o(i.nrfx_is_in_ram) for nrfx_is_in_ram
    nrfx_uarte.o(i.nrfx_uarte_tx) refers to nrfx_uarte.o(i.nrfx_uarte_tx_in_progress) for nrfx_uarte_tx_in_progress
    nrfx_uarte.o(i.nrfx_uarte_tx) refers to nrfx_uarte.o(i.nrf_uarte_event_clear) for nrf_uarte_event_clear
    nrfx_uarte.o(i.nrfx_uarte_tx) refers to nrfx_uarte.o(i.nrf_uarte_event_check) for nrf_uarte_event_check
    nrfx_uarte.o(i.nrfx_uarte_tx) refers to nrfx_uarte.o(.bss) for .bss
    nrfx_uarte.o(i.nrfx_uarte_tx_abort) refers to nrfx_uarte.o(i.nrf_uarte_event_clear) for nrf_uarte_event_clear
    nrfx_uarte.o(i.nrfx_uarte_tx_abort) refers to nrfx_uarte.o(i.nrf_uarte_event_check) for nrf_uarte_event_check
    nrfx_uarte.o(i.nrfx_uarte_tx_abort) refers to nrfx_uarte.o(.bss) for .bss
    nrfx_uarte.o(i.nrfx_uarte_tx_in_progress) refers to nrfx_uarte.o(.bss) for .bss
    nrfx_uarte.o(i.nrfx_uarte_uninit) refers to nrfx_uarte.o(i.nrf_uarte_event_clear) for nrf_uarte_event_clear
    nrfx_uarte.o(i.nrfx_uarte_uninit) refers to nrfx_uarte.o(i.nrf_uarte_event_check) for nrf_uarte_event_check
    nrfx_uarte.o(i.nrfx_uarte_uninit) refers to nrfx_uarte.o(i.nrf_gpio_cfg_default) for nrf_gpio_cfg_default
    nrfx_uarte.o(i.nrfx_uarte_uninit) refers to nrfx_prs.o(i.nrfx_prs_release) for nrfx_prs_release
    nrfx_uarte.o(i.nrfx_uarte_uninit) refers to nrfx_uarte.o(.bss) for .bss
    nrfx_uarte.o(i.uarte_irq_handler) refers to nrfx_uarte.o(i.nrf_uarte_event_check) for nrf_uarte_event_check
    nrfx_uarte.o(i.uarte_irq_handler) refers to nrfx_uarte.o(i.nrf_uarte_event_clear) for nrf_uarte_event_clear
    nrfx_uarte.o(i.uarte_irq_handler) refers to nrfx_uarte.o(i.rx_done_event) for rx_done_event
    nrfx_uarte.o(i.uarte_irq_handler) refers to nrfx_uarte.o(i.tx_done_event) for tx_done_event
    nrfx_uarte.o(.constdata) refers to nrfx_uarte.o(i.UARTE0_UART0_IRQHandler) for UARTE0_UART0_IRQHandler
    app_scheduler.o(i.app_sched_event_put) refers to app_util_platform.o(i.app_util_critical_region_enter) for app_util_critical_region_enter
    app_scheduler.o(i.app_sched_event_put) refers to app_util_platform.o(i.app_util_critical_region_exit) for app_util_critical_region_exit
    app_scheduler.o(i.app_sched_event_put) refers to memcpya.o(.text) for __aeabi_memcpy
    app_scheduler.o(i.app_sched_event_put) refers to app_scheduler.o(.data) for .data
    app_scheduler.o(i.app_sched_execute) refers to app_scheduler.o(.data) for .data
    app_scheduler.o(i.app_sched_init) refers to app_scheduler.o(.data) for .data
    app_scheduler.o(i.app_sched_queue_space_get) refers to app_scheduler.o(.data) for .data
    app_util_platform.o(i.app_util_critical_region_enter) refers to app_util_platform.o(i.app_util_disable_irq) for app_util_disable_irq
    app_util_platform.o(i.app_util_critical_region_exit) refers to app_util_platform.o(i.app_util_enable_irq) for app_util_enable_irq
    app_util_platform.o(i.app_util_disable_irq) refers to app_util_platform.o(.data) for .data
    app_util_platform.o(i.app_util_enable_irq) refers to app_util_platform.o(.data) for .data
    mem_manager.o(i.block_init) refers to mem_manager.o(.data) for .data
    mem_manager.o(i.get_block_cat) refers to mem_manager.o(.constdata) for .constdata
    mem_manager.o(i.get_block_size) refers to mem_manager.o(i.get_block_cat) for get_block_cat
    mem_manager.o(i.get_block_size) refers to mem_manager.o(.constdata) for .constdata
    mem_manager.o(i.nrf_calloc) refers to mem_manager.o(i.nrf_mem_reserve) for nrf_mem_reserve
    mem_manager.o(i.nrf_calloc) refers to memseta.o(.text) for __aeabi_memclr
    mem_manager.o(i.nrf_free) refers to mem_manager.o(i.block_init) for block_init
    mem_manager.o(i.nrf_free) refers to mem_manager.o(i.get_block_size) for get_block_size
    mem_manager.o(i.nrf_free) refers to mem_manager.o(.data) for .data
    mem_manager.o(i.nrf_free) refers to mem_manager.o(.bss) for .bss
    mem_manager.o(i.nrf_malloc) refers to mem_manager.o(i.nrf_mem_reserve) for nrf_mem_reserve
    mem_manager.o(i.nrf_mem_init) refers to mem_manager.o(i.block_init) for block_init
    mem_manager.o(i.nrf_mem_init) refers to mem_manager.o(.data) for .data
    mem_manager.o(i.nrf_mem_reserve) refers to mem_manager.o(i.get_block_cat) for get_block_cat
    mem_manager.o(i.nrf_mem_reserve) refers to mem_manager.o(i.get_block_size) for get_block_size
    mem_manager.o(i.nrf_mem_reserve) refers to mem_manager.o(.data) for .data
    mem_manager.o(i.nrf_mem_reserve) refers to mem_manager.o(.constdata) for .constdata
    mem_manager.o(i.nrf_mem_reserve) refers to mem_manager.o(.bss) for .bss
    nrf_assert.o(i.assert_nrf_callback) refers to main.o(i.app_error_fault_handler) for app_error_fault_handler
    nrf_atomic.o(i.nrf_atomic_flag_clear) refers to nrf_atomic.o(i.nrf_atomic_u32_and) for nrf_atomic_u32_and
    nrf_atomic.o(i.nrf_atomic_flag_clear_fetch) refers to nrf_atomic.o(i.nrf_atomic_u32_fetch_and) for nrf_atomic_u32_fetch_and
    nrf_atomic.o(i.nrf_atomic_flag_set) refers to nrf_atomic.o(i.nrf_atomic_u32_or) for nrf_atomic_u32_or
    nrf_atomic.o(i.nrf_atomic_flag_set_fetch) refers to nrf_atomic.o(i.nrf_atomic_u32_fetch_or) for nrf_atomic_u32_fetch_or
    nrf_atomic.o(i.nrf_atomic_u32_add) refers to nrf_atomic.o(.emb_text) for __asm___12_nrf_atomic_c_85ca2469__nrf_atomic_internal_add
    nrf_atomic.o(i.nrf_atomic_u32_and) refers to nrf_atomic.o(.emb_text) for __asm___12_nrf_atomic_c_85ca2469__nrf_atomic_internal_and
    nrf_atomic.o(i.nrf_atomic_u32_cmp_exch) refers to nrf_atomic.o(.emb_text) for __asm___12_nrf_atomic_c_85ca2469__nrf_atomic_internal_cmp_exch
    nrf_atomic.o(i.nrf_atomic_u32_fetch_add) refers to nrf_atomic.o(.emb_text) for __asm___12_nrf_atomic_c_85ca2469__nrf_atomic_internal_add
    nrf_atomic.o(i.nrf_atomic_u32_fetch_and) refers to nrf_atomic.o(.emb_text) for __asm___12_nrf_atomic_c_85ca2469__nrf_atomic_internal_and
    nrf_atomic.o(i.nrf_atomic_u32_fetch_or) refers to nrf_atomic.o(.emb_text) for __asm___12_nrf_atomic_c_85ca2469__nrf_atomic_internal_orr
    nrf_atomic.o(i.nrf_atomic_u32_fetch_store) refers to nrf_atomic.o(.emb_text) for __asm___12_nrf_atomic_c_85ca2469__nrf_atomic_internal_mov
    nrf_atomic.o(i.nrf_atomic_u32_fetch_sub) refers to nrf_atomic.o(.emb_text) for __asm___12_nrf_atomic_c_85ca2469__nrf_atomic_internal_sub
    nrf_atomic.o(i.nrf_atomic_u32_fetch_sub_hs) refers to nrf_atomic.o(.emb_text) for __asm___12_nrf_atomic_c_85ca2469__nrf_atomic_internal_sub_hs
    nrf_atomic.o(i.nrf_atomic_u32_fetch_xor) refers to nrf_atomic.o(.emb_text) for __asm___12_nrf_atomic_c_85ca2469__nrf_atomic_internal_eor
    nrf_atomic.o(i.nrf_atomic_u32_or) refers to nrf_atomic.o(.emb_text) for __asm___12_nrf_atomic_c_85ca2469__nrf_atomic_internal_orr
    nrf_atomic.o(i.nrf_atomic_u32_store) refers to nrf_atomic.o(.emb_text) for __asm___12_nrf_atomic_c_85ca2469__nrf_atomic_internal_mov
    nrf_atomic.o(i.nrf_atomic_u32_sub) refers to nrf_atomic.o(.emb_text) for __asm___12_nrf_atomic_c_85ca2469__nrf_atomic_internal_sub
    nrf_atomic.o(i.nrf_atomic_u32_sub_hs) refers to nrf_atomic.o(.emb_text) for __asm___12_nrf_atomic_c_85ca2469__nrf_atomic_internal_sub_hs
    nrf_atomic.o(i.nrf_atomic_u32_xor) refers to nrf_atomic.o(.emb_text) for __asm___12_nrf_atomic_c_85ca2469__nrf_atomic_internal_eor
    nrf_balloc.o(i.nrf_balloc_alloc) refers to app_util_platform.o(i.app_util_critical_region_enter) for app_util_critical_region_enter
    nrf_balloc.o(i.nrf_balloc_alloc) refers to app_util_platform.o(i.app_util_critical_region_exit) for app_util_critical_region_exit
    nrf_balloc.o(i.nrf_balloc_free) refers to app_util_platform.o(i.app_util_critical_region_enter) for app_util_critical_region_enter
    nrf_balloc.o(i.nrf_balloc_free) refers to app_util_platform.o(i.app_util_critical_region_exit) for app_util_critical_region_exit
    nrf_fprintf.o(i.nrf_fprintf) refers to nrf_fprintf_format.o(i.nrf_fprintf_fmt) for nrf_fprintf_fmt
    nrf_fprintf_format.o(i.buffer_add) refers to nrf_fprintf.o(i.nrf_fprintf_buffer_flush) for nrf_fprintf_buffer_flush
    nrf_fprintf_format.o(i.int_print) refers to nrf_fprintf_format.o(i.buffer_add) for buffer_add
    nrf_fprintf_format.o(i.int_print) refers to nrf_fprintf_format.o(i.unsigned_print) for unsigned_print
    nrf_fprintf_format.o(i.nrf_fprintf_fmt) refers to nrf_fprintf_format.o(i.buffer_add) for buffer_add
    nrf_fprintf_format.o(i.nrf_fprintf_fmt) refers to nrf_fprintf.o(i.nrf_fprintf_buffer_flush) for nrf_fprintf_buffer_flush
    nrf_fprintf_format.o(i.nrf_fprintf_fmt) refers to nrf_fprintf_format.o(i.int_print) for int_print
    nrf_fprintf_format.o(i.nrf_fprintf_fmt) refers to nrf_fprintf_format.o(i.unsigned_print) for unsigned_print
    nrf_fprintf_format.o(i.nrf_fprintf_fmt) refers to strlen.o(.text) for strlen
    nrf_fprintf_format.o(i.unsigned_print) refers to nrf_fprintf_format.o(i.buffer_add) for buffer_add
    nrf_fprintf_format.o(i.unsigned_print) refers to nrf_fprintf_format.o(.constdata) for .constdata
    nrf_fstorage.o(i.nrf_fstorage_erase) refers to nrf_fstorage.o(i.addr_is_within_bounds) for addr_is_within_bounds
    nrf_fstorage.o(i.nrf_fstorage_read) refers to nrf_fstorage.o(i.addr_is_aligned32) for addr_is_aligned32
    nrf_fstorage.o(i.nrf_fstorage_read) refers to nrf_fstorage.o(i.addr_is_within_bounds) for addr_is_within_bounds
    nrf_fstorage.o(i.nrf_fstorage_write) refers to nrf_fstorage.o(i.addr_is_aligned32) for addr_is_aligned32
    nrf_fstorage.o(i.nrf_fstorage_write) refers to nrf_fstorage.o(i.addr_is_within_bounds) for addr_is_within_bounds
    nrf_fstorage_nvmc.o(i.erase) refers to nrf_atomic.o(i.nrf_atomic_flag_set_fetch) for nrf_atomic_flag_set_fetch
    nrf_fstorage_nvmc.o(i.erase) refers to nrf_nvmc.o(i.nrf_nvmc_page_erase) for nrf_nvmc_page_erase
    nrf_fstorage_nvmc.o(i.erase) refers to nrf_atomic.o(i.nrf_atomic_flag_clear) for nrf_atomic_flag_clear
    nrf_fstorage_nvmc.o(i.erase) refers to nrf_fstorage_nvmc.o(i.event_send) for event_send
    nrf_fstorage_nvmc.o(i.erase) refers to nrf_fstorage_nvmc.o(.data) for .data
    nrf_fstorage_nvmc.o(i.event_send) refers to memseta.o(.text) for __aeabi_memclr4
    nrf_fstorage_nvmc.o(i.init) refers to nrf_fstorage_nvmc.o(.constdata) for .constdata
    nrf_fstorage_nvmc.o(i.is_busy) refers to nrf_fstorage_nvmc.o(.data) for .data
    nrf_fstorage_nvmc.o(i.read) refers to memcpya.o(.text) for __aeabi_memcpy
    nrf_fstorage_nvmc.o(i.uninit) refers to nrf_atomic.o(i.nrf_atomic_flag_clear) for nrf_atomic_flag_clear
    nrf_fstorage_nvmc.o(i.uninit) refers to nrf_fstorage_nvmc.o(.data) for .data
    nrf_fstorage_nvmc.o(i.write) refers to nrf_atomic.o(i.nrf_atomic_flag_set_fetch) for nrf_atomic_flag_set_fetch
    nrf_fstorage_nvmc.o(i.write) refers to nrf_nvmc.o(i.nrf_nvmc_write_words) for nrf_nvmc_write_words
    nrf_fstorage_nvmc.o(i.write) refers to nrf_atomic.o(i.nrf_atomic_flag_clear) for nrf_atomic_flag_clear
    nrf_fstorage_nvmc.o(i.write) refers to nrf_fstorage_nvmc.o(i.event_send) for event_send
    nrf_fstorage_nvmc.o(i.write) refers to nrf_fstorage_nvmc.o(.data) for .data
    nrf_fstorage_nvmc.o(.constdata) refers to nrf_fstorage_nvmc.o(i.init) for init
    nrf_fstorage_nvmc.o(.constdata) refers to nrf_fstorage_nvmc.o(i.uninit) for uninit
    nrf_fstorage_nvmc.o(.constdata) refers to nrf_fstorage_nvmc.o(i.read) for read
    nrf_fstorage_nvmc.o(.constdata) refers to nrf_fstorage_nvmc.o(i.write) for write
    nrf_fstorage_nvmc.o(.constdata) refers to nrf_fstorage_nvmc.o(i.erase) for erase
    nrf_fstorage_nvmc.o(.constdata) refers to nrf_fstorage_nvmc.o(i.rmap) for rmap
    nrf_fstorage_nvmc.o(.constdata) refers to nrf_fstorage_nvmc.o(i.wmap) for wmap
    nrf_fstorage_nvmc.o(.constdata) refers to nrf_fstorage_nvmc.o(i.is_busy) for is_busy
    nrf_memobj.o(i.memobj_op) refers to memcpya.o(.text) for __aeabi_memcpy
    nrf_memobj.o(i.nrf_memobj_alloc) refers to nrf_balloc.o(i.nrf_balloc_alloc) for nrf_balloc_alloc
    nrf_memobj.o(i.nrf_memobj_alloc) refers to nrf_memobj.o(i.nrf_memobj_free) for nrf_memobj_free
    nrf_memobj.o(i.nrf_memobj_free) refers to nrf_balloc.o(i.nrf_balloc_free) for nrf_balloc_free
    nrf_memobj.o(i.nrf_memobj_get) refers to nrf_atomic.o(i.nrf_atomic_u32_add) for nrf_atomic_u32_add
    nrf_memobj.o(i.nrf_memobj_pool_init) refers to nrf_balloc.o(i.nrf_balloc_init) for nrf_balloc_init
    nrf_memobj.o(i.nrf_memobj_put) refers to nrf_atomic.o(i.nrf_atomic_u32_sub) for nrf_atomic_u32_sub
    nrf_memobj.o(i.nrf_memobj_put) refers to nrf_memobj.o(i.nrf_memobj_free) for nrf_memobj_free
    nrf_memobj.o(i.nrf_memobj_read) refers to nrf_memobj.o(i.memobj_op) for memobj_op
    nrf_memobj.o(i.nrf_memobj_write) refers to nrf_memobj.o(i.memobj_op) for memobj_op
    nrf_ringbuf.o(i.nrf_ringbuf_alloc) refers to nrf_atomic.o(i.nrf_atomic_flag_set_fetch) for nrf_atomic_flag_set_fetch
    nrf_ringbuf.o(i.nrf_ringbuf_alloc) refers to nrf_atomic.o(i.nrf_atomic_flag_clear) for nrf_atomic_flag_clear
    nrf_ringbuf.o(i.nrf_ringbuf_cpy_get) refers to nrf_atomic.o(i.nrf_atomic_flag_set_fetch) for nrf_atomic_flag_set_fetch
    nrf_ringbuf.o(i.nrf_ringbuf_cpy_get) refers to memcpya.o(.text) for __aeabi_memcpy
    nrf_ringbuf.o(i.nrf_ringbuf_cpy_get) refers to nrf_atomic.o(i.nrf_atomic_flag_clear) for nrf_atomic_flag_clear
    nrf_ringbuf.o(i.nrf_ringbuf_cpy_put) refers to nrf_atomic.o(i.nrf_atomic_flag_set_fetch) for nrf_atomic_flag_set_fetch
    nrf_ringbuf.o(i.nrf_ringbuf_cpy_put) refers to memcpya.o(.text) for __aeabi_memcpy
    nrf_ringbuf.o(i.nrf_ringbuf_cpy_put) refers to nrf_atomic.o(i.nrf_atomic_flag_clear) for nrf_atomic_flag_clear
    nrf_ringbuf.o(i.nrf_ringbuf_free) refers to nrf_atomic.o(i.nrf_atomic_flag_clear) for nrf_atomic_flag_clear
    nrf_ringbuf.o(i.nrf_ringbuf_get) refers to nrf_atomic.o(i.nrf_atomic_flag_set_fetch) for nrf_atomic_flag_set_fetch
    nrf_ringbuf.o(i.nrf_ringbuf_get) refers to nrf_atomic.o(i.nrf_atomic_flag_clear) for nrf_atomic_flag_clear
    nrf_ringbuf.o(i.nrf_ringbuf_put) refers to nrf_atomic.o(i.nrf_atomic_flag_clear_fetch) for nrf_atomic_flag_clear_fetch
    nrf_strerror.o(i.nrf_strerror_find) refers to nrf_strerror.o(.constdata) for .constdata
    nrf_strerror.o(i.nrf_strerror_get) refers to nrf_strerror.o(i.nrf_strerror_find) for nrf_strerror_find
    nrf_strerror.o(i.nrf_strerror_get) refers to nrf_strerror.o(.constdata) for .constdata
    nrf_strerror.o(.constdata) refers to nrf_strerror.o(.conststring) for .conststring
    sha256.o(i.sha256_final) refers to sha256.o(i.sha256_transform) for sha256_transform
    sha256.o(i.sha256_final) refers to memseta.o(.text) for __aeabi_memclr4
    sha256.o(i.sha256_transform) refers to sha256.o(.constdata) for .constdata
    sha256.o(i.sha256_update) refers to sha256.o(i.sha256_transform) for sha256_transform
    nrf_dfu_serial.o(i.dfu_req_handler_rsp_clbk) refers to nrf_dfu_serial.o(i.response_send) for response_send
    nrf_dfu_serial.o(i.nrf_dfu_serial_on_packet_received) refers to memcpya.o(.text) for __aeabi_memcpy4
    nrf_dfu_serial.o(i.nrf_dfu_serial_on_packet_received) refers to nrf_dfu_transport.o(i.nrf_dfu_transports_close) for nrf_dfu_transports_close
    nrf_dfu_serial.o(i.nrf_dfu_serial_on_packet_received) refers to nrf_dfu_req_handler.o(i.nrf_dfu_req_handler_on_req) for nrf_dfu_req_handler_on_req
    nrf_dfu_serial.o(i.nrf_dfu_serial_on_packet_received) refers to nrf_dfu_serial.o(.constdata) for .constdata
    nrf_dfu_serial.o(i.response_send) refers to nrf_dfu_serial.o(i.uint32_encode) for uint32_encode
    nrf_dfu_serial.o(i.response_send) refers to nrf_dfu_handling_error.o(i.ext_error_get) for ext_error_get
    nrf_dfu_serial.o(i.response_send) refers to nrf_dfu_handling_error.o(i.ext_error_set) for ext_error_set
    nrf_dfu_serial.o(.constdata) refers to nrf_dfu_serial.o(i.dfu_req_handler_rsp_clbk) for dfu_req_handler_rsp_clbk
    pb_common.o(i.pb_field_iter_find) refers to pb_common.o(i.pb_field_iter_next) for pb_field_iter_next
    pb_common.o(i.pb_field_iter_next) refers to pb_common.o(i.pb_field_iter_begin) for pb_field_iter_begin
    pb_decode.o(i.decode_callback_field) refers to pb_decode.o(i.read_raw_value) for read_raw_value
    pb_decode.o(i.decode_callback_field) refers to pb_decode.o(i.pb_istream_from_buffer) for pb_istream_from_buffer
    pb_decode.o(i.decode_callback_field) refers to pb_decode.o(i.pb_skip_field) for pb_skip_field
    pb_decode.o(i.decode_callback_field) refers to pb_decode.o(i.pb_make_string_substream) for pb_make_string_substream
    pb_decode.o(i.decode_field) refers to pb_decode.o(i.decode_static_field) for decode_static_field
    pb_decode.o(i.decode_field) refers to pb_decode.o(i.decode_callback_field) for decode_callback_field
    pb_decode.o(i.decode_static_field) refers to pb_decode.o(i.pb_make_string_substream) for pb_make_string_substream
    pb_decode.o(i.decode_static_field) refers to memseta.o(.text) for __aeabi_memclr
    pb_decode.o(i.decode_static_field) refers to pb_decode.o(i.pb_message_set_to_defaults) for pb_message_set_to_defaults
    pb_decode.o(i.decode_static_field) refers to pb_decode.o(.constdata) for .constdata
    pb_decode.o(i.iter_from_extension) refers to pb_common.o(i.pb_field_iter_begin) for pb_field_iter_begin
    pb_decode.o(i.pb_dec_bytes) refers to pb_decode.o(i.pb_decode_varint32) for pb_decode_varint32
    pb_decode.o(i.pb_dec_bytes) refers to pb_decode.o(i.pb_read) for pb_read
    pb_decode.o(i.pb_dec_fixed32) refers to pb_decode.o(i.pb_decode_fixed32) for pb_decode_fixed32
    pb_decode.o(i.pb_dec_fixed64) refers to pb_decode.o(i.pb_decode_fixed64) for pb_decode_fixed64
    pb_decode.o(i.pb_dec_string) refers to pb_decode.o(i.pb_decode_varint32) for pb_decode_varint32
    pb_decode.o(i.pb_dec_string) refers to pb_decode.o(i.pb_read) for pb_read
    pb_decode.o(i.pb_dec_submessage) refers to pb_decode.o(i.pb_make_string_substream) for pb_make_string_substream
    pb_decode.o(i.pb_dec_submessage) refers to pb_decode.o(i.pb_decode_noinit) for pb_decode_noinit
    pb_decode.o(i.pb_dec_submessage) refers to pb_decode.o(i.pb_decode) for pb_decode
    pb_decode.o(i.pb_dec_svarint) refers to pb_decode.o(i.pb_decode_svarint) for pb_decode_svarint
    pb_decode.o(i.pb_dec_uvarint) refers to pb_decode.o(i.pb_decode_varint) for pb_decode_varint
    pb_decode.o(i.pb_dec_varint) refers to pb_decode.o(i.pb_decode_varint) for pb_decode_varint
    pb_decode.o(i.pb_decode) refers to pb_decode.o(i.pb_message_set_to_defaults) for pb_message_set_to_defaults
    pb_decode.o(i.pb_decode) refers to pb_decode.o(i.pb_decode_noinit) for pb_decode_noinit
    pb_decode.o(i.pb_decode_delimited) refers to pb_decode.o(i.pb_make_string_substream) for pb_make_string_substream
    pb_decode.o(i.pb_decode_delimited) refers to pb_decode.o(i.pb_decode) for pb_decode
    pb_decode.o(i.pb_decode_fixed32) refers to pb_decode.o(i.pb_read) for pb_read
    pb_decode.o(i.pb_decode_fixed64) refers to pb_decode.o(i.pb_read) for pb_read
    pb_decode.o(i.pb_decode_noinit) refers to pb_common.o(i.pb_field_iter_begin) for pb_field_iter_begin
    pb_decode.o(i.pb_decode_noinit) refers to pb_decode.o(i.pb_decode_tag) for pb_decode_tag
    pb_decode.o(i.pb_decode_noinit) refers to pb_common.o(i.pb_field_iter_find) for pb_field_iter_find
    pb_decode.o(i.pb_decode_noinit) refers to pb_common.o(i.pb_field_iter_next) for pb_field_iter_next
    pb_decode.o(i.pb_decode_noinit) refers to pb_decode.o(i.iter_from_extension) for iter_from_extension
    pb_decode.o(i.pb_decode_noinit) refers to pb_decode.o(i.decode_field) for decode_field
    pb_decode.o(i.pb_decode_noinit) refers to pb_decode.o(i.pb_skip_field) for pb_skip_field
    pb_decode.o(i.pb_decode_svarint) refers to pb_decode.o(i.pb_decode_varint) for pb_decode_varint
    pb_decode.o(i.pb_decode_tag) refers to pb_decode.o(i.pb_decode_varint32) for pb_decode_varint32
    pb_decode.o(i.pb_decode_varint) refers to pb_decode.o(i.pb_readbyte) for pb_readbyte
    pb_decode.o(i.pb_decode_varint) refers to llshl.o(.text) for __aeabi_llsl
    pb_decode.o(i.pb_decode_varint32) refers to pb_decode.o(i.pb_readbyte) for pb_readbyte
    pb_decode.o(i.pb_field_set_to_default) refers to pb_decode.o(i.iter_from_extension) for iter_from_extension
    pb_decode.o(i.pb_field_set_to_default) refers to memcpya.o(.text) for __aeabi_memcpy
    pb_decode.o(i.pb_field_set_to_default) refers to pb_decode.o(i.pb_message_set_to_defaults) for pb_message_set_to_defaults
    pb_decode.o(i.pb_field_set_to_default) refers to memseta.o(.text) for __aeabi_memclr
    pb_decode.o(i.pb_istream_from_buffer) refers to pb_decode.o(i.buf_read) for buf_read
    pb_decode.o(i.pb_make_string_substream) refers to pb_decode.o(i.pb_decode_varint32) for pb_decode_varint32
    pb_decode.o(i.pb_message_set_to_defaults) refers to pb_common.o(i.pb_field_iter_begin) for pb_field_iter_begin
    pb_decode.o(i.pb_message_set_to_defaults) refers to pb_decode.o(i.pb_field_set_to_default) for pb_field_set_to_default
    pb_decode.o(i.pb_message_set_to_defaults) refers to pb_common.o(i.pb_field_iter_next) for pb_field_iter_next
    pb_decode.o(i.pb_read) refers to pb_decode.o(i.buf_read) for buf_read
    pb_decode.o(i.pb_skip_field) refers to pb_decode.o(i.pb_read) for pb_read
    pb_decode.o(i.pb_skip_field) refers to pb_decode.o(i.pb_decode_varint32) for pb_decode_varint32
    pb_decode.o(i.read_raw_value) refers to pb_decode.o(i.pb_read) for pb_read
    pb_decode.o(.constdata) refers to pb_decode.o(i.pb_dec_varint) for pb_dec_varint
    pb_decode.o(.constdata) refers to pb_decode.o(i.pb_dec_uvarint) for pb_dec_uvarint
    pb_decode.o(.constdata) refers to pb_decode.o(i.pb_dec_svarint) for pb_dec_svarint
    pb_decode.o(.constdata) refers to pb_decode.o(i.pb_dec_fixed32) for pb_dec_fixed32
    pb_decode.o(.constdata) refers to pb_decode.o(i.pb_dec_fixed64) for pb_dec_fixed64
    pb_decode.o(.constdata) refers to pb_decode.o(i.pb_dec_bytes) for pb_dec_bytes
    pb_decode.o(.constdata) refers to pb_decode.o(i.pb_dec_string) for pb_dec_string
    pb_decode.o(.constdata) refers to pb_decode.o(i.pb_dec_submessage) for pb_dec_submessage
    arm_startup_nrf52820.o(RESET) refers to arm_startup_nrf52820.o(STACK) for __initial_sp
    arm_startup_nrf52820.o(RESET) refers to arm_startup_nrf52820.o(.text) for Reset_Handler
    arm_startup_nrf52820.o(RESET) refers to nrfx_uarte.o(i.UARTE0_UART0_IRQHandler) for UARTE0_UART0_IRQHandler
    arm_startup_nrf52820.o(RESET) refers to nrf_bootloader_wdt.o(i.WDT_IRQHandler) for WDT_IRQHandler
    arm_startup_nrf52820.o(RESET) refers to nrf_bootloader_dfu_timers.o(i.RTC1_IRQHandler) for RTC1_IRQHandler
    arm_startup_nrf52820.o(.text) refers to system_nrf52.o(i.SystemInit) for SystemInit
    arm_startup_nrf52820.o(.text) refers to entry.o(.ARM.Collect$$$$00000000) for __main
    system_nrf52.o(i.SystemCoreClockUpdate) refers to system_nrf52.o(.data) for .data
    system_nrf52.o(i.SystemInit) refers to system_nrf52.o(i.nvmc_config) for nvmc_config
    system_nrf52.o(i.SystemInit) refers to system_nrf52.o(.data) for .data
    uECC.c.o(.text.uECC_vli_cmp) refers to uECC.c.o(.text.uECC_vli_sub) for uECC_vli_sub
    uECC.c.o(.text.uECC_vli_cmp) refers to uECC.c.o(.text.uECC_vli_isZero) for uECC_vli_isZero
    uECC.c.o(.text.uECC_vli_modAdd) refers to uECC.c.o(.text.uECC_vli_add) for uECC_vli_add
    uECC.c.o(.text.uECC_vli_modAdd) refers to uECC.c.o(.text.uECC_vli_cmp_unsafe) for uECC_vli_cmp_unsafe
    uECC.c.o(.text.uECC_vli_modAdd) refers to uECC.c.o(.text.uECC_vli_sub) for uECC_vli_sub
    uECC.c.o(.text.uECC_vli_modSub) refers to uECC.c.o(.text.uECC_vli_sub) for uECC_vli_sub
    uECC.c.o(.text.uECC_vli_modSub) refers to uECC.c.o(.text.uECC_vli_add) for uECC_vli_add
    uECC.c.o(.text.uECC_vli_modMult) refers to uECC.c.o(.text.uECC_vli_mult) for uECC_vli_mult
    uECC.c.o(.text.uECC_vli_modMult) refers to uECC.c.o(.text.uECC_vli_numBits) for uECC_vli_numBits
    uECC.c.o(.text.uECC_vli_modMult) refers to uECC.c.o(.text.uECC_vli_clear) for uECC_vli_clear
    uECC.c.o(.text.uECC_vli_modMult) refers to uECC.c.o(.text.uECC_vli_set) for uECC_vli_set
    uECC.c.o(.text.uECC_vli_modMult) refers to uECC.c.o(.text.uECC_vli_rshift1) for uECC_vli_rshift1
    uECC.c.o(.text.uECC_vli_modMult_fast) refers to uECC.c.o(.text.uECC_vli_mult) for uECC_vli_mult
    uECC.c.o(.text.uECC_vli_modSquare_fast) refers to uECC.c.o(.text.uECC_vli_modMult_fast) for uECC_vli_modMult_fast
    uECC.c.o(.text.double_jacobian_default) refers to uECC.c.o(.text.uECC_vli_isZero) for uECC_vli_isZero
    uECC.c.o(.text.double_jacobian_default) refers to uECC.c.o(.text.uECC_vli_modSquare_fast) for uECC_vli_modSquare_fast
    uECC.c.o(.text.double_jacobian_default) refers to uECC.c.o(.text.uECC_vli_modMult_fast) for uECC_vli_modMult_fast
    uECC.c.o(.text.double_jacobian_default) refers to uECC.c.o(.text.uECC_vli_modAdd) for uECC_vli_modAdd
    uECC.c.o(.text.double_jacobian_default) refers to uECC.c.o(.text.uECC_vli_modSub) for uECC_vli_modSub
    uECC.c.o(.text.double_jacobian_default) refers to uECC.c.o(.text.uECC_vli_add) for uECC_vli_add
    uECC.c.o(.text.double_jacobian_default) refers to uECC.c.o(.text.uECC_vli_rshift1) for uECC_vli_rshift1
    uECC.c.o(.text.double_jacobian_default) refers to uECC.c.o(.text.uECC_vli_set) for uECC_vli_set
    uECC.c.o(.text.x_side_default) refers to memseta.o(.text) for memset
    uECC.c.o(.text.x_side_default) refers to uECC.c.o(.text.uECC_vli_modSquare_fast) for uECC_vli_modSquare_fast
    uECC.c.o(.text.x_side_default) refers to uECC.c.o(.text.uECC_vli_modSub) for uECC_vli_modSub
    uECC.c.o(.text.x_side_default) refers to uECC.c.o(.text.uECC_vli_modMult_fast) for uECC_vli_modMult_fast
    uECC.c.o(.text.x_side_default) refers to uECC.c.o(.text.uECC_vli_modAdd) for uECC_vli_modAdd
    uECC.c.o(.text.omega_mult_secp160r1) refers to uECC.c.o(.text.uECC_vli_set) for uECC_vli_set
    uECC.c.o(.text.omega_mult_secp160r1) refers to uECC.c.o(.text.uECC_vli_rshift1) for uECC_vli_rshift1
    uECC.c.o(.text.omega_mult_secp160r1) refers to uECC.c.o(.text.uECC_vli_add) for uECC_vli_add
    uECC.c.o(.text.vli_mmod_fast_secp160r1) refers to uECC.c.o(.text.uECC_vli_clear) for uECC_vli_clear
    uECC.c.o(.text.vli_mmod_fast_secp160r1) refers to uECC.c.o(.text.omega_mult_secp160r1) for omega_mult_secp160r1
    uECC.c.o(.text.vli_mmod_fast_secp160r1) refers to uECC.c.o(.text.uECC_vli_add) for uECC_vli_add
    uECC.c.o(.text.vli_mmod_fast_secp160r1) refers to uECC.c.o(.text.uECC_vli_cmp_unsafe) for uECC_vli_cmp_unsafe
    uECC.c.o(.text.vli_mmod_fast_secp160r1) refers to uECC.c.o(.text.uECC_vli_sub) for uECC_vli_sub
    uECC.c.o(.text.vli_mmod_fast_secp160r1) refers to uECC.c.o(.rodata.curve_secp160r1) for [Anonymous Symbol]
    uECC.c.o(.text.vli_mmod_fast_secp192r1) refers to uECC.c.o(.text.uECC_vli_set) for uECC_vli_set
    uECC.c.o(.text.vli_mmod_fast_secp192r1) refers to uECC.c.o(.text.uECC_vli_add) for uECC_vli_add
    uECC.c.o(.text.vli_mmod_fast_secp192r1) refers to uECC.c.o(.text.uECC_vli_cmp_unsafe) for uECC_vli_cmp_unsafe
    uECC.c.o(.text.vli_mmod_fast_secp192r1) refers to uECC.c.o(.text.uECC_vli_sub) for uECC_vli_sub
    uECC.c.o(.text.vli_mmod_fast_secp192r1) refers to uECC.c.o(.rodata.curve_secp192r1) for [Anonymous Symbol]
    uECC.c.o(.text.vli_mmod_fast_secp224r1) refers to uECC.c.o(.text.uECC_vli_set) for uECC_vli_set
    uECC.c.o(.text.vli_mmod_fast_secp224r1) refers to uECC.c.o(.text.uECC_vli_add) for uECC_vli_add
    uECC.c.o(.text.vli_mmod_fast_secp224r1) refers to uECC.c.o(.text.uECC_vli_sub) for uECC_vli_sub
    uECC.c.o(.text.vli_mmod_fast_secp224r1) refers to uECC.c.o(.text.uECC_vli_cmp_unsafe) for uECC_vli_cmp_unsafe
    uECC.c.o(.text.vli_mmod_fast_secp224r1) refers to uECC.c.o(.rodata.curve_secp224r1) for [Anonymous Symbol]
    uECC.c.o(.text.vli_mmod_fast_secp256r1) refers to uECC.c.o(.text.uECC_vli_set) for uECC_vli_set
    uECC.c.o(.text.vli_mmod_fast_secp256r1) refers to uECC.c.o(.text.uECC_vli_add) for uECC_vli_add
    uECC.c.o(.text.vli_mmod_fast_secp256r1) refers to uECC.c.o(.text.uECC_vli_sub) for uECC_vli_sub
    uECC.c.o(.text.vli_mmod_fast_secp256r1) refers to uECC.c.o(.text.uECC_vli_cmp_unsafe) for uECC_vli_cmp_unsafe
    uECC.c.o(.text.vli_mmod_fast_secp256r1) refers to uECC.c.o(.rodata.curve_secp256r1) for [Anonymous Symbol]
    uECC.c.o(.text.x_side_secp256k1) refers to uECC.c.o(.text.uECC_vli_modSquare_fast) for uECC_vli_modSquare_fast
    uECC.c.o(.text.x_side_secp256k1) refers to uECC.c.o(.text.uECC_vli_modMult_fast) for uECC_vli_modMult_fast
    uECC.c.o(.text.x_side_secp256k1) refers to uECC.c.o(.text.uECC_vli_modAdd) for uECC_vli_modAdd
    uECC.c.o(.text.omega_mult_secp256k1) refers to uECC.c.o(.text.uECC_vli_add) for uECC_vli_add
    uECC.c.o(.text.vli_mmod_fast_secp256k1) refers to uECC.c.o(.text.uECC_vli_clear) for uECC_vli_clear
    uECC.c.o(.text.vli_mmod_fast_secp256k1) refers to uECC.c.o(.text.omega_mult_secp256k1) for omega_mult_secp256k1
    uECC.c.o(.text.vli_mmod_fast_secp256k1) refers to uECC.c.o(.text.uECC_vli_add) for uECC_vli_add
    uECC.c.o(.text.vli_mmod_fast_secp256k1) refers to uECC.c.o(.text.uECC_vli_cmp_unsafe) for uECC_vli_cmp_unsafe
    uECC.c.o(.text.vli_mmod_fast_secp256k1) refers to uECC.c.o(.text.uECC_vli_sub) for uECC_vli_sub
    uECC.c.o(.text.vli_mmod_fast_secp256k1) refers to uECC.c.o(.rodata.curve_secp256k1) for [Anonymous Symbol]
    uECC.c.o(.text.apply_z) refers to uECC.c.o(.text.uECC_vli_modSquare_fast) for uECC_vli_modSquare_fast
    uECC.c.o(.text.apply_z) refers to uECC.c.o(.text.uECC_vli_modMult_fast) for uECC_vli_modMult_fast
    uECC.c.o(.text.XYcZ_add) refers to uECC.c.o(.text.uECC_vli_modSub) for uECC_vli_modSub
    uECC.c.o(.text.XYcZ_add) refers to uECC.c.o(.text.uECC_vli_modSquare_fast) for uECC_vli_modSquare_fast
    uECC.c.o(.text.XYcZ_add) refers to uECC.c.o(.text.uECC_vli_modMult_fast) for uECC_vli_modMult_fast
    uECC.c.o(.text.XYcZ_add) refers to uECC.c.o(.text.uECC_vli_set) for uECC_vli_set
    uECC.c.o(.text.XYcZ_addC) refers to uECC.c.o(.text.uECC_vli_modSub) for uECC_vli_modSub
    uECC.c.o(.text.XYcZ_addC) refers to uECC.c.o(.text.uECC_vli_modSquare_fast) for uECC_vli_modSquare_fast
    uECC.c.o(.text.XYcZ_addC) refers to uECC.c.o(.text.uECC_vli_modMult_fast) for uECC_vli_modMult_fast
    uECC.c.o(.text.XYcZ_addC) refers to uECC.c.o(.text.uECC_vli_modAdd) for uECC_vli_modAdd
    uECC.c.o(.text.XYcZ_addC) refers to uECC.c.o(.text.uECC_vli_set) for uECC_vli_set
    uECC.c.o(.text.regularize_k) refers to uECC.c.o(.text.uECC_vli_add) for uECC_vli_add
    uECC.c.o(.text.regularize_k) refers to uECC.c.o(.text.uECC_vli_testBit) for uECC_vli_testBit
    uECC.c.o(.text.uECC_generate_random_int) refers to uECC.c.o(.text.uECC_vli_numBits) for uECC_vli_numBits
    uECC.c.o(.text.uECC_generate_random_int) refers to uECC.c.o(.text.uECC_vli_isZero) for uECC_vli_isZero
    uECC.c.o(.text.uECC_generate_random_int) refers to uECC.c.o(.text.uECC_vli_cmp) for uECC_vli_cmp
    uECC.c.o(.text.uECC_generate_random_int) refers to uECC.c.o(.bss.g_rng_function) for [Anonymous Symbol]
    uECC.c.o(.text.bits2int) refers to uECC.c.o(.text.uECC_vli_clear) for uECC_vli_clear
    uECC.c.o(.text.bits2int) refers to uECC.c.o(.text.bcopy) for bcopy
    uECC.c.o(.text.bits2int) refers to uECC.c.o(.text.uECC_vli_cmp_unsafe) for uECC_vli_cmp_unsafe
    uECC.c.o(.text.bits2int) refers to uECC.c.o(.text.uECC_vli_sub) for uECC_vli_sub
    uECC.c.o(.text.update_V) refers to uECC.c.o(.text.HMAC_init) for HMAC_init
    uECC.c.o(.text.update_V) refers to uECC.c.o(.text.HMAC_update) for HMAC_update
    uECC.c.o(.text.update_V) refers to uECC.c.o(.text.HMAC_finish) for HMAC_finish
    uECC.c.o(.text.vli_modInv_update) refers to uECC.c.o(.text.uECC_vli_add) for uECC_vli_add
    uECC.c.o(.text.vli_modInv_update) refers to uECC.c.o(.text.uECC_vli_rshift1) for uECC_vli_rshift1
    uECC.c.o(.text.uECC_vli_modInv) refers to uECC.c.o(.text.uECC_vli_isZero) for uECC_vli_isZero
    uECC.c.o(.text.uECC_vli_modInv) refers to uECC.c.o(.text.uECC_vli_clear) for uECC_vli_clear
    uECC.c.o(.text.uECC_vli_modInv) refers to uECC.c.o(.text.uECC_vli_set) for uECC_vli_set
    uECC.c.o(.text.uECC_vli_modInv) refers to uECC.c.o(.text.uECC_vli_cmp_unsafe) for uECC_vli_cmp_unsafe
    uECC.c.o(.text.uECC_vli_modInv) refers to uECC.c.o(.text.uECC_vli_rshift1) for uECC_vli_rshift1
    uECC.c.o(.text.uECC_vli_modInv) refers to uECC.c.o(.text.vli_modInv_update) for vli_modInv_update
    uECC.c.o(.text.uECC_vli_modInv) refers to uECC.c.o(.text.uECC_vli_sub) for uECC_vli_sub
    uECC.c.o(.text.uECC_vli_modInv) refers to uECC.c.o(.text.uECC_vli_add) for uECC_vli_add
    uECC.c.o(.text.EccPoint_mult) refers to uECC.c.o(.text.uECC_vli_set) for uECC_vli_set
    uECC.c.o(.text.EccPoint_mult) refers to uECC.c.o(.text.apply_z) for apply_z
    uECC.c.o(.text.EccPoint_mult) refers to uECC.c.o(.text.XYcZ_addC) for XYcZ_addC
    uECC.c.o(.text.EccPoint_mult) refers to uECC.c.o(.text.uECC_vli_modSub) for uECC_vli_modSub
    uECC.c.o(.text.EccPoint_mult) refers to uECC.c.o(.text.uECC_vli_modMult_fast) for uECC_vli_modMult_fast
    uECC.c.o(.text.EccPoint_mult) refers to uECC.c.o(.text.uECC_vli_modInv) for uECC_vli_modInv
    uECC.c.o(.text.EccPoint_mult) refers to uECC.c.o(.text.XYcZ_add) for XYcZ_add
    uECC.c.o(.text.EccPoint_mult) refers to uECC.c.o(.text.uECC_vli_clear) for uECC_vli_clear
    uECC.c.o(.text.EccPoint_mult) refers to uECC.c.o(.text.uECC_vli_testBit) for uECC_vli_testBit
    uECC.c.o(.text.EccPoint_compute_public_key) refers to uECC.c.o(.text.regularize_k) for regularize_k
    uECC.c.o(.text.EccPoint_compute_public_key) refers to uECC.c.o(.text.uECC_generate_random_int) for uECC_generate_random_int
    uECC.c.o(.text.EccPoint_compute_public_key) refers to uECC.c.o(.text.EccPoint_mult) for EccPoint_mult
    uECC.c.o(.text.EccPoint_compute_public_key) refers to uECC.c.o(.text.uECC_vli_isZero) for uECC_vli_isZero
    uECC.c.o(.text.EccPoint_compute_public_key) refers to uECC.c.o(.bss.g_rng_function) for [Anonymous Symbol]
    uECC.c.o(.text.uECC_sign_with_k_internal) refers to uECC.c.o(.text.uECC_vli_isZero) for uECC_vli_isZero
    uECC.c.o(.text.uECC_sign_with_k_internal) refers to uECC.c.o(.text.uECC_vli_cmp) for uECC_vli_cmp
    uECC.c.o(.text.uECC_sign_with_k_internal) refers to uECC.c.o(.text.regularize_k) for regularize_k
    uECC.c.o(.text.uECC_sign_with_k_internal) refers to uECC.c.o(.text.uECC_generate_random_int) for uECC_generate_random_int
    uECC.c.o(.text.uECC_sign_with_k_internal) refers to uECC.c.o(.text.EccPoint_mult) for EccPoint_mult
    uECC.c.o(.text.uECC_sign_with_k_internal) refers to uECC.c.o(.text.uECC_vli_clear) for uECC_vli_clear
    uECC.c.o(.text.uECC_sign_with_k_internal) refers to uECC.c.o(.text.uECC_vli_modMult) for uECC_vli_modMult
    uECC.c.o(.text.uECC_sign_with_k_internal) refers to uECC.c.o(.text.uECC_vli_modInv) for uECC_vli_modInv
    uECC.c.o(.text.uECC_sign_with_k_internal) refers to uECC.c.o(.text.bcopy) for bcopy
    uECC.c.o(.text.uECC_sign_with_k_internal) refers to uECC.c.o(.text.uECC_vli_set) for uECC_vli_set
    uECC.c.o(.text.uECC_sign_with_k_internal) refers to uECC.c.o(.text.bits2int) for bits2int
    uECC.c.o(.text.uECC_sign_with_k_internal) refers to uECC.c.o(.text.uECC_vli_modAdd) for uECC_vli_modAdd
    uECC.c.o(.text.uECC_sign_with_k_internal) refers to uECC.c.o(.text.uECC_vli_numBits) for uECC_vli_numBits
    uECC.c.o(.text.uECC_sign_with_k_internal) refers to uECC.c.o(.bss.g_rng_function) for [Anonymous Symbol]
    uECC.c.o(.text.double_jacobian_secp256k1) refers to uECC.c.o(.text.uECC_vli_isZero) for uECC_vli_isZero
    uECC.c.o(.text.double_jacobian_secp256k1) refers to uECC.c.o(.text.uECC_vli_modSquare_fast) for uECC_vli_modSquare_fast
    uECC.c.o(.text.double_jacobian_secp256k1) refers to uECC.c.o(.text.uECC_vli_modMult_fast) for uECC_vli_modMult_fast
    uECC.c.o(.text.double_jacobian_secp256k1) refers to uECC.c.o(.text.uECC_vli_modAdd) for uECC_vli_modAdd
    uECC.c.o(.text.double_jacobian_secp256k1) refers to uECC.c.o(.text.uECC_vli_add) for uECC_vli_add
    uECC.c.o(.text.double_jacobian_secp256k1) refers to uECC.c.o(.text.uECC_vli_rshift1) for uECC_vli_rshift1
    uECC.c.o(.text.double_jacobian_secp256k1) refers to uECC.c.o(.text.uECC_vli_modSub) for uECC_vli_modSub
    uECC.c.o(.text.uECC_set_rng) refers to uECC.c.o(.bss.g_rng_function) for [Anonymous Symbol]
    uECC.c.o(.text.uECC_get_rng) refers to uECC.c.o(.bss.g_rng_function) for [Anonymous Symbol]
    uECC.c.o(.text.uECC_secp160r1) refers to uECC.c.o(.rodata.curve_secp160r1) for [Anonymous Symbol]
    uECC.c.o(.text.uECC_secp192r1) refers to uECC.c.o(.rodata.curve_secp192r1) for [Anonymous Symbol]
    uECC.c.o(.text.uECC_secp224r1) refers to uECC.c.o(.rodata.curve_secp224r1) for [Anonymous Symbol]
    uECC.c.o(.text.uECC_secp256r1) refers to uECC.c.o(.rodata.curve_secp256r1) for [Anonymous Symbol]
    uECC.c.o(.text.uECC_secp256k1) refers to uECC.c.o(.rodata.curve_secp256k1) for [Anonymous Symbol]
    uECC.c.o(.text.uECC_make_key) refers to uECC.c.o(.text.uECC_generate_random_int) for uECC_generate_random_int
    uECC.c.o(.text.uECC_make_key) refers to uECC.c.o(.text.EccPoint_compute_public_key) for EccPoint_compute_public_key
    uECC.c.o(.text.uECC_shared_secret) refers to uECC.c.o(.text.bcopy) for bcopy
    uECC.c.o(.text.uECC_shared_secret) refers to uECC.c.o(.text.regularize_k) for regularize_k
    uECC.c.o(.text.uECC_shared_secret) refers to uECC.c.o(.text.uECC_generate_random_int) for uECC_generate_random_int
    uECC.c.o(.text.uECC_shared_secret) refers to uECC.c.o(.text.EccPoint_mult) for EccPoint_mult
    uECC.c.o(.text.uECC_shared_secret) refers to uECC.c.o(.text.uECC_vli_isZero) for uECC_vli_isZero
    uECC.c.o(.text.uECC_shared_secret) refers to uECC.c.o(.bss.g_rng_function) for [Anonymous Symbol]
    uECC.c.o(.text.uECC_valid_public_key) refers to uECC.c.o(.text.uECC_vli_isZero) for uECC_vli_isZero
    uECC.c.o(.text.uECC_valid_public_key) refers to uECC.c.o(.text.uECC_vli_cmp_unsafe) for uECC_vli_cmp_unsafe
    uECC.c.o(.text.uECC_valid_public_key) refers to uECC.c.o(.text.uECC_vli_modSquare_fast) for uECC_vli_modSquare_fast
    uECC.c.o(.text.uECC_compute_public_key) refers to uECC.c.o(.text.uECC_vli_isZero) for uECC_vli_isZero
    uECC.c.o(.text.uECC_compute_public_key) refers to uECC.c.o(.text.uECC_vli_cmp) for uECC_vli_cmp
    uECC.c.o(.text.uECC_compute_public_key) refers to uECC.c.o(.text.EccPoint_compute_public_key) for EccPoint_compute_public_key
    uECC.c.o(.text.uECC_sign_with_k) refers to uECC.c.o(.text.bits2int) for bits2int
    uECC.c.o(.text.uECC_sign_with_k) refers to uECC.c.o(.text.uECC_sign_with_k_internal) for uECC_sign_with_k_internal
    uECC.c.o(.text.uECC_sign) refers to uECC.c.o(.text.uECC_generate_random_int) for uECC_generate_random_int
    uECC.c.o(.text.uECC_sign) refers to uECC.c.o(.text.uECC_sign_with_k_internal) for uECC_sign_with_k_internal
    uECC.c.o(.text.uECC_sign_deterministic) refers to uECC.c.o(.text.HMAC_init) for HMAC_init
    uECC.c.o(.text.uECC_sign_deterministic) refers to uECC.c.o(.text.HMAC_update) for HMAC_update
    uECC.c.o(.text.uECC_sign_deterministic) refers to uECC.c.o(.text.HMAC_finish) for HMAC_finish
    uECC.c.o(.text.uECC_sign_deterministic) refers to uECC.c.o(.text.update_V) for update_V
    uECC.c.o(.text.uECC_sign_deterministic) refers to uECC.c.o(.text.uECC_sign_with_k_internal) for uECC_sign_with_k_internal
    uECC.c.o(.text.uECC_verify) refers to uECC.c.o(.text.bcopy) for bcopy
    uECC.c.o(.text.uECC_verify) refers to uECC.c.o(.text.uECC_vli_isZero) for uECC_vli_isZero
    uECC.c.o(.text.uECC_verify) refers to uECC.c.o(.text.uECC_vli_cmp_unsafe) for uECC_vli_cmp_unsafe
    uECC.c.o(.text.uECC_verify) refers to uECC.c.o(.text.uECC_vli_modInv) for uECC_vli_modInv
    uECC.c.o(.text.uECC_verify) refers to uECC.c.o(.text.bits2int) for bits2int
    uECC.c.o(.text.uECC_verify) refers to uECC.c.o(.text.uECC_vli_modMult) for uECC_vli_modMult
    uECC.c.o(.text.uECC_verify) refers to uECC.c.o(.text.uECC_vli_set) for uECC_vli_set
    uECC.c.o(.text.uECC_verify) refers to uECC.c.o(.text.uECC_vli_modSub) for uECC_vli_modSub
    uECC.c.o(.text.uECC_verify) refers to uECC.c.o(.text.XYcZ_add) for XYcZ_add
    uECC.c.o(.text.uECC_verify) refers to uECC.c.o(.text.apply_z) for apply_z
    uECC.c.o(.text.uECC_verify) refers to uECC.c.o(.text.uECC_vli_numBits) for uECC_vli_numBits
    uECC.c.o(.text.uECC_verify) refers to uECC.c.o(.text.uECC_vli_testBit) for uECC_vli_testBit
    uECC.c.o(.text.uECC_verify) refers to uECC.c.o(.text.uECC_vli_clear) for uECC_vli_clear
    uECC.c.o(.text.uECC_verify) refers to uECC.c.o(.text.uECC_vli_sub) for uECC_vli_sub
    uECC.c.o(.text.uECC_verify) refers to uECC.c.o(.text.uECC_vli_modMult_fast) for uECC_vli_modMult_fast
    uECC.c.o(.rodata.curve_secp160r1) refers to uECC.c.o(.text.double_jacobian_default) for double_jacobian_default
    uECC.c.o(.rodata.curve_secp160r1) refers to uECC.c.o(.text.x_side_default) for x_side_default
    uECC.c.o(.rodata.curve_secp160r1) refers to uECC.c.o(.text.vli_mmod_fast_secp160r1) for vli_mmod_fast_secp160r1
    uECC.c.o(.rodata.curve_secp192r1) refers to uECC.c.o(.text.double_jacobian_default) for double_jacobian_default
    uECC.c.o(.rodata.curve_secp192r1) refers to uECC.c.o(.text.x_side_default) for x_side_default
    uECC.c.o(.rodata.curve_secp192r1) refers to uECC.c.o(.text.vli_mmod_fast_secp192r1) for vli_mmod_fast_secp192r1
    uECC.c.o(.rodata.curve_secp224r1) refers to uECC.c.o(.text.double_jacobian_default) for double_jacobian_default
    uECC.c.o(.rodata.curve_secp224r1) refers to uECC.c.o(.text.x_side_default) for x_side_default
    uECC.c.o(.rodata.curve_secp224r1) refers to uECC.c.o(.text.vli_mmod_fast_secp224r1) for vli_mmod_fast_secp224r1
    uECC.c.o(.rodata.curve_secp256k1) refers to uECC.c.o(.text.double_jacobian_secp256k1) for double_jacobian_secp256k1
    uECC.c.o(.rodata.curve_secp256k1) refers to uECC.c.o(.text.x_side_secp256k1) for x_side_secp256k1
    uECC.c.o(.rodata.curve_secp256k1) refers to uECC.c.o(.text.vli_mmod_fast_secp256k1) for vli_mmod_fast_secp256k1
    uECC.c.o(.rodata.curve_secp256r1) refers to uECC.c.o(.text.double_jacobian_default) for double_jacobian_default
    uECC.c.o(.rodata.curve_secp256r1) refers to uECC.c.o(.text.x_side_default) for x_side_default
    uECC.c.o(.rodata.curve_secp256r1) refers to uECC.c.o(.text.vli_mmod_fast_secp256r1) for vli_mmod_fast_secp256r1
    entry.o(.ARM.Collect$$$$00000000) refers (Special) to entry10a.o(.ARM.Collect$$$$0000000D) for __rt_final_cpp
    entry.o(.ARM.Collect$$$$00000000) refers (Special) to entry11a.o(.ARM.Collect$$$$0000000F) for __rt_final_exit
    entry.o(.ARM.Collect$$$$00000000) refers (Special) to entry7b.o(.ARM.Collect$$$$00000008) for _main_clock
    entry.o(.ARM.Collect$$$$00000000) refers (Special) to entry8b.o(.ARM.Collect$$$$0000000A) for _main_cpp_init
    entry.o(.ARM.Collect$$$$00000000) refers (Special) to entry9a.o(.ARM.Collect$$$$0000000B) for _main_init
    entry.o(.ARM.Collect$$$$00000000) refers (Special) to entry5.o(.ARM.Collect$$$$00000004) for _main_scatterload
    entry.o(.ARM.Collect$$$$00000000) refers (Special) to entry2.o(.ARM.Collect$$$$00000001) for _main_stk
    entry2.o(.ARM.Collect$$$$00000001) refers to entry2.o(.ARM.Collect$$$$00002712) for __lit__00000000
    entry2.o(.ARM.Collect$$$$00002712) refers to arm_startup_nrf52820.o(STACK) for __initial_sp
    entry2.o(__vectab_stack_and_reset_area) refers to arm_startup_nrf52820.o(STACK) for __initial_sp
    entry2.o(__vectab_stack_and_reset_area) refers to entry.o(.ARM.Collect$$$$00000000) for __main
    entry5.o(.ARM.Collect$$$$00000004) refers to init.o(.text) for __scatterload
    entry9a.o(.ARM.Collect$$$$0000000B) refers to main.o(i.main) for main
    entry9b.o(.ARM.Collect$$$$0000000C) refers to main.o(i.main) for main
    init.o(.text) refers to entry5.o(.ARM.Collect$$$$00000004) for __main_after_scatterload


==============================================================================

Removing Unused input sections from the image.

    Removing main.o(.rev16_text), (4 bytes).
    Removing main.o(.revsh_text), (4 bytes).
    Removing main.o(.rrx_text), (6 bytes).
    Removing main.o(i.app_error_fault_handler), (4 bytes).
    Removing main.o(i.app_error_handler), (4 bytes).
    Removing boards.o(.rev16_text), (4 bytes).
    Removing boards.o(.revsh_text), (4 bytes).
    Removing boards.o(.rrx_text), (6 bytes).
    Removing boards.o(i.bsp_board_button_idx_to_pin), (12 bytes).
    Removing boards.o(i.bsp_board_button_state_get), (32 bytes).
    Removing boards.o(i.bsp_board_led_idx_to_pin), (12 bytes).
    Removing boards.o(i.bsp_board_led_invert), (36 bytes).
    Removing boards.o(i.bsp_board_led_state_get), (32 bytes).
    Removing boards.o(i.bsp_board_leds_on), (18 bytes).
    Removing boards.o(i.bsp_board_pin_to_button_idx), (36 bytes).
    Removing boards.o(i.bsp_board_pin_to_led_idx), (36 bytes).
    Removing nrf_bootloader.o(.rev16_text), (4 bytes).
    Removing nrf_bootloader.o(.revsh_text), (4 bytes).
    Removing nrf_bootloader.o(.rrx_text), (6 bytes).
    Removing nrf_bootloader.o(i.nrf_dfu_init), (4 bytes).
    Removing nrf_bootloader.o(.constdata), (6 bytes).
    Removing nrf_bootloader_app_start.o(.rev16_text), (4 bytes).
    Removing nrf_bootloader_app_start.o(.revsh_text), (4 bytes).
    Removing nrf_bootloader_app_start.o(.rrx_text), (6 bytes).
    Removing nrf_bootloader_app_start_final.o(.rev16_text), (4 bytes).
    Removing nrf_bootloader_app_start_final.o(.revsh_text), (4 bytes).
    Removing nrf_bootloader_app_start_final.o(.rrx_text), (6 bytes).
    Removing nrf_bootloader_app_start_final.o(i.jump_to_addr), (6 bytes).
    Removing nrf_bootloader_dfu_timers.o(.rev16_text), (4 bytes).
    Removing nrf_bootloader_dfu_timers.o(.revsh_text), (4 bytes).
    Removing nrf_bootloader_dfu_timers.o(.rrx_text), (6 bytes).
    Removing nrf_bootloader_dfu_timers.o(i.nrf_bootloader_dfu_timer_counter_get), (24 bytes).
    Removing nrf_bootloader_fw_activation.o(.rev16_text), (4 bytes).
    Removing nrf_bootloader_fw_activation.o(.revsh_text), (4 bytes).
    Removing nrf_bootloader_fw_activation.o(.rrx_text), (6 bytes).
    Removing nrf_bootloader_info.o(.rev16_text), (4 bytes).
    Removing nrf_bootloader_info.o(.revsh_text), (4 bytes).
    Removing nrf_bootloader_info.o(.rrx_text), (6 bytes).
    Removing nrf_bootloader_info.o(i.__NVIC_SystemReset), (36 bytes).
    Removing nrf_bootloader_info.o(i.nrf_bootloader_debug_port_disable), (48 bytes).
    Removing nrf_bootloader_wdt.o(.rev16_text), (4 bytes).
    Removing nrf_bootloader_wdt.o(.revsh_text), (4 bytes).
    Removing nrf_bootloader_wdt.o(.rrx_text), (6 bytes).
    Removing nrf_crypto_ecc.o(.rev16_text), (4 bytes).
    Removing nrf_crypto_ecc.o(.revsh_text), (4 bytes).
    Removing nrf_crypto_ecc.o(.rrx_text), (6 bytes).
    Removing nrf_crypto_ecc.o(i.nrf_crypto_ecc_byte_order_invert), (82 bytes).
    Removing nrf_crypto_ecc.o(i.nrf_crypto_ecc_curve_info_get), (48 bytes).
    Removing nrf_crypto_ecc.o(i.nrf_crypto_ecc_key_pair_generate), (68 bytes).
    Removing nrf_crypto_ecc.o(i.nrf_crypto_ecc_private_key_free), (24 bytes).
    Removing nrf_crypto_ecc.o(i.nrf_crypto_ecc_private_key_from_raw), (52 bytes).
    Removing nrf_crypto_ecc.o(i.nrf_crypto_ecc_private_key_to_raw), (52 bytes).
    Removing nrf_crypto_ecc.o(i.nrf_crypto_ecc_public_key_calculate), (60 bytes).
    Removing nrf_crypto_ecc.o(i.nrf_crypto_ecc_public_key_free), (24 bytes).
    Removing nrf_crypto_ecc.o(i.nrf_crypto_ecc_public_key_to_raw), (52 bytes).
    Removing nrf_crypto_ecc.o(i.nrf_crypto_internal_ecc_raw_output_prepare), (28 bytes).
    Removing nrf_crypto_ecdsa.o(.rev16_text), (4 bytes).
    Removing nrf_crypto_ecdsa.o(.revsh_text), (4 bytes).
    Removing nrf_crypto_ecdsa.o(.rrx_text), (6 bytes).
    Removing nrf_crypto_ecdsa.o(i.nrf_crypto_ecdsa_sign), (76 bytes).
    Removing nrf_crypto_hash.o(.rev16_text), (4 bytes).
    Removing nrf_crypto_hash.o(.revsh_text), (4 bytes).
    Removing nrf_crypto_hash.o(.rrx_text), (6 bytes).
    Removing nrf_crypto_init.o(.rev16_text), (4 bytes).
    Removing nrf_crypto_init.o(.revsh_text), (4 bytes).
    Removing nrf_crypto_init.o(.rrx_text), (6 bytes).
    Removing nrf_crypto_init.o(i.nrf_crypto_is_initialized), (20 bytes).
    Removing nrf_crypto_init.o(i.nrf_crypto_is_initializing), (28 bytes).
    Removing nrf_crypto_init.o(i.nrf_crypto_uninit), (56 bytes).
    Removing nrf_crypto_shared.o(.rev16_text), (4 bytes).
    Removing nrf_crypto_shared.o(.revsh_text), (4 bytes).
    Removing nrf_crypto_shared.o(.rrx_text), (6 bytes).
    Removing oberon_backend_chacha_poly_aead.o(.rev16_text), (4 bytes).
    Removing oberon_backend_chacha_poly_aead.o(.revsh_text), (4 bytes).
    Removing oberon_backend_chacha_poly_aead.o(.rrx_text), (6 bytes).
    Removing oberon_backend_hash.o(.rev16_text), (4 bytes).
    Removing oberon_backend_hash.o(.revsh_text), (4 bytes).
    Removing oberon_backend_hash.o(.rrx_text), (6 bytes).
    Removing oberon_backend_hmac.o(.rev16_text), (4 bytes).
    Removing oberon_backend_hmac.o(.revsh_text), (4 bytes).
    Removing oberon_backend_hmac.o(.rrx_text), (6 bytes).
    Removing nrf_sw_backend_hash.o(.rev16_text), (4 bytes).
    Removing nrf_sw_backend_hash.o(.revsh_text), (4 bytes).
    Removing nrf_sw_backend_hash.o(.rrx_text), (6 bytes).
    Removing micro_ecc_backend_ecc.o(.rev16_text), (4 bytes).
    Removing micro_ecc_backend_ecc.o(.revsh_text), (4 bytes).
    Removing micro_ecc_backend_ecc.o(.rrx_text), (6 bytes).
    Removing micro_ecc_backend_ecc.o(i.nrf_crypto_backend_micro_ecc_key_pair_generate), (52 bytes).
    Removing micro_ecc_backend_ecc.o(i.nrf_crypto_backend_micro_ecc_private_key_from_raw), (16 bytes).
    Removing micro_ecc_backend_ecc.o(i.nrf_crypto_backend_micro_ecc_private_key_to_raw), (22 bytes).
    Removing micro_ecc_backend_ecc.o(i.nrf_crypto_backend_micro_ecc_public_key_calculate), (38 bytes).
    Removing micro_ecc_backend_ecc.o(i.nrf_crypto_backend_micro_ecc_public_key_to_raw), (22 bytes).
    Removing micro_ecc_backend_ecc.o(i.nrf_crypto_backend_micro_ecc_rng_callback), (4 bytes).
    Removing micro_ecc_backend_ecdh.o(.rev16_text), (4 bytes).
    Removing micro_ecc_backend_ecdh.o(.revsh_text), (4 bytes).
    Removing micro_ecc_backend_ecdh.o(.rrx_text), (6 bytes).
    Removing micro_ecc_backend_ecdh.o(i.nrf_crypto_backend_micro_ecc_ecdh_compute), (74 bytes).
    Removing micro_ecc_backend_ecdsa.o(.rev16_text), (4 bytes).
    Removing micro_ecc_backend_ecdsa.o(.revsh_text), (4 bytes).
    Removing micro_ecc_backend_ecdsa.o(.rrx_text), (6 bytes).
    Removing micro_ecc_backend_ecdsa.o(i.nrf_crypto_backend_micro_ecc_sign), (96 bytes).
    Removing nrf_dfu.o(.rev16_text), (4 bytes).
    Removing nrf_dfu.o(.revsh_text), (4 bytes).
    Removing nrf_dfu.o(.rrx_text), (6 bytes).
    Removing nrf_dfu_flash.o(.rev16_text), (4 bytes).
    Removing nrf_dfu_flash.o(.revsh_text), (4 bytes).
    Removing nrf_dfu_flash.o(.rrx_text), (6 bytes).
    Removing nrf_dfu_flash.o(.data), (4 bytes).
    Removing nrf_dfu_handling_error.o(.rev16_text), (4 bytes).
    Removing nrf_dfu_handling_error.o(.revsh_text), (4 bytes).
    Removing nrf_dfu_handling_error.o(.rrx_text), (6 bytes).
    Removing nrf_dfu_mbr.o(.rev16_text), (4 bytes).
    Removing nrf_dfu_mbr.o(.revsh_text), (4 bytes).
    Removing nrf_dfu_mbr.o(.rrx_text), (6 bytes).
    Removing nrf_dfu_mbr.o(i.nrf_dfu_mbr_init_sd), (24 bytes).
    Removing nrf_dfu_req_handler.o(.rev16_text), (4 bytes).
    Removing nrf_dfu_req_handler.o(.revsh_text), (4 bytes).
    Removing nrf_dfu_req_handler.o(.rrx_text), (6 bytes).
    Removing nrf_dfu_serial_uart.o(.rev16_text), (4 bytes).
    Removing nrf_dfu_serial_uart.o(.revsh_text), (4 bytes).
    Removing nrf_dfu_serial_uart.o(.rrx_text), (6 bytes).
    Removing nrf_dfu_settings.o(.rev16_text), (4 bytes).
    Removing nrf_dfu_settings.o(.revsh_text), (4 bytes).
    Removing nrf_dfu_settings.o(.rrx_text), (6 bytes).
    Removing nrf_dfu_transport.o(.rev16_text), (4 bytes).
    Removing nrf_dfu_transport.o(.revsh_text), (4 bytes).
    Removing nrf_dfu_transport.o(.rrx_text), (6 bytes).
    Removing nrf_dfu_utils.o(.rev16_text), (4 bytes).
    Removing nrf_dfu_utils.o(.revsh_text), (4 bytes).
    Removing nrf_dfu_utils.o(.rrx_text), (6 bytes).
    Removing nrf_dfu_validation.o(.rev16_text), (4 bytes).
    Removing nrf_dfu_validation.o(.revsh_text), (4 bytes).
    Removing nrf_dfu_validation.o(.rrx_text), (6 bytes).
    Removing nrf_dfu_validation.o(i.nrf_dfu_validation_init_cmd_status_get), (24 bytes).
    Removing nrf_dfu_validation.o(i.nrf_dfu_validation_post_data_execute), (6 bytes).
    Removing nrf_dfu_validation.o(i.nrf_dfu_validation_valid_external_app), (20 bytes).
    Removing nrf_dfu_ver_validation.o(.rev16_text), (4 bytes).
    Removing nrf_dfu_ver_validation.o(.revsh_text), (4 bytes).
    Removing nrf_dfu_ver_validation.o(.rrx_text), (6 bytes).
    Removing nrf_drv_uart.o(.rev16_text), (4 bytes).
    Removing nrf_drv_uart.o(.revsh_text), (4 bytes).
    Removing nrf_drv_uart.o(.rrx_text), (6 bytes).
    Removing nrf_drv_uart.o(.data), (1 bytes).
    Removing nrf_nvic.o(.rev16_text), (4 bytes).
    Removing nrf_nvic.o(.revsh_text), (4 bytes).
    Removing nrf_nvic.o(.rrx_text), (6 bytes).
    Removing nrf_nvic.o(i.sd_nvic_ClearPendingIRQ), (28 bytes).
    Removing nrf_nvic.o(i.sd_nvic_DisableIRQ), (36 bytes).
    Removing nrf_nvic.o(i.sd_nvic_EnableIRQ), (28 bytes).
    Removing nrf_nvic.o(i.sd_nvic_GetPendingIRQ), (46 bytes).
    Removing nrf_nvic.o(i.sd_nvic_GetPriority), (40 bytes).
    Removing nrf_nvic.o(i.sd_nvic_SetPendingIRQ), (28 bytes).
    Removing nrf_nvic.o(i.sd_nvic_SetPriority), (34 bytes).
    Removing nrf_nvic.o(i.sd_nvic_SystemReset), (36 bytes).
    Removing nrf_nvic.o(i.sd_nvic_critical_region_enter), (28 bytes).
    Removing nrf_nvic.o(i.sd_nvic_critical_region_exit), (24 bytes).
    Removing nrf_nvic.o(.data), (1 bytes).
    Removing nrf_nvmc.o(.rev16_text), (4 bytes).
    Removing nrf_nvmc.o(.revsh_text), (4 bytes).
    Removing nrf_nvmc.o(.rrx_text), (6 bytes).
    Removing nrf_nvmc.o(i.nrf_nvmc_write_byte), (68 bytes).
    Removing nrf_nvmc.o(i.nrf_nvmc_write_bytes), (28 bytes).
    Removing nrf_soc.o(.rev16_text), (4 bytes).
    Removing nrf_soc.o(.revsh_text), (4 bytes).
    Removing nrf_soc.o(.rrx_text), (6 bytes).
    Removing nrf_soc.o(i.sd_app_evt_wait), (6 bytes).
    Removing nrfx_atomic.o(.rev16_text), (4 bytes).
    Removing nrfx_atomic.o(.revsh_text), (4 bytes).
    Removing nrfx_atomic.o(.rrx_text), (6 bytes).
    Removing nrfx_atomic.o(.emb_text), (226 bytes).
    Removing nrfx_atomic.o(i.nrfx_atomic_flag_clear), (6 bytes).
    Removing nrfx_atomic.o(i.nrfx_atomic_flag_clear_fetch), (6 bytes).
    Removing nrfx_atomic.o(i.nrfx_atomic_flag_set), (6 bytes).
    Removing nrfx_atomic.o(i.nrfx_atomic_flag_set_fetch), (6 bytes).
    Removing nrfx_atomic.o(i.nrfx_atomic_u32_add), (12 bytes).
    Removing nrfx_atomic.o(i.nrfx_atomic_u32_and), (12 bytes).
    Removing nrfx_atomic.o(i.nrfx_atomic_u32_cmp_exch), (4 bytes).
    Removing nrfx_atomic.o(i.nrfx_atomic_u32_fetch_add), (10 bytes).
    Removing nrfx_atomic.o(i.nrfx_atomic_u32_fetch_and), (10 bytes).
    Removing nrfx_atomic.o(i.nrfx_atomic_u32_fetch_or), (10 bytes).
    Removing nrfx_atomic.o(i.nrfx_atomic_u32_fetch_store), (10 bytes).
    Removing nrfx_atomic.o(i.nrfx_atomic_u32_fetch_sub), (10 bytes).
    Removing nrfx_atomic.o(i.nrfx_atomic_u32_fetch_sub_hs), (10 bytes).
    Removing nrfx_atomic.o(i.nrfx_atomic_u32_fetch_xor), (10 bytes).
    Removing nrfx_atomic.o(i.nrfx_atomic_u32_or), (12 bytes).
    Removing nrfx_atomic.o(i.nrfx_atomic_u32_store), (12 bytes).
    Removing nrfx_atomic.o(i.nrfx_atomic_u32_sub), (12 bytes).
    Removing nrfx_atomic.o(i.nrfx_atomic_u32_sub_hs), (12 bytes).
    Removing nrfx_atomic.o(i.nrfx_atomic_u32_xor), (12 bytes).
    Removing nrfx_prs.o(.rev16_text), (4 bytes).
    Removing nrfx_prs.o(.revsh_text), (4 bytes).
    Removing nrfx_prs.o(.rrx_text), (6 bytes).
    Removing nrfx_prs.o(.constdata), (17 bytes).
    Removing nrfx_uart.o(.rev16_text), (4 bytes).
    Removing nrfx_uart.o(.revsh_text), (4 bytes).
    Removing nrfx_uart.o(.rrx_text), (6 bytes).
    Removing nrfx_uarte.o(.rev16_text), (4 bytes).
    Removing nrfx_uarte.o(.revsh_text), (4 bytes).
    Removing nrfx_uarte.o(.rrx_text), (6 bytes).
    Removing nrfx_uarte.o(i.nrfx_uarte_errorsrc_get), (26 bytes).
    Removing nrfx_uarte.o(i.nrfx_uarte_rx_abort), (44 bytes).
    Removing nrfx_uarte.o(i.nrfx_uarte_rx_ready), (14 bytes).
    Removing nrfx_uarte.o(i.nrfx_uarte_tx_abort), (56 bytes).
    Removing nrfx_uarte.o(.constdata), (16 bytes).
    Removing nrfx_uarte.o(.constdata), (14 bytes).
    Removing nrfx_uarte.o(.constdata), (14 bytes).
    Removing app_error_weak.o(.rev16_text), (4 bytes).
    Removing app_error_weak.o(.revsh_text), (4 bytes).
    Removing app_error_weak.o(.rrx_text), (6 bytes).
    Removing app_error_weak.o(i.app_error_fault_handler), (48 bytes).
    Removing app_scheduler.o(.rev16_text), (4 bytes).
    Removing app_scheduler.o(.revsh_text), (4 bytes).
    Removing app_scheduler.o(.rrx_text), (6 bytes).
    Removing app_scheduler.o(i.app_sched_queue_space_get), (36 bytes).
    Removing app_util_platform.o(.rev16_text), (4 bytes).
    Removing app_util_platform.o(.revsh_text), (4 bytes).
    Removing app_util_platform.o(.rrx_text), (6 bytes).
    Removing app_util_platform.o(i.current_int_priority_get), (48 bytes).
    Removing app_util_platform.o(i.privilege_level_get), (26 bytes).
    Removing crc32.o(.rev16_text), (4 bytes).
    Removing crc32.o(.revsh_text), (4 bytes).
    Removing crc32.o(.rrx_text), (6 bytes).
    Removing mem_manager.o(.rev16_text), (4 bytes).
    Removing mem_manager.o(.revsh_text), (4 bytes).
    Removing mem_manager.o(.rrx_text), (6 bytes).
    Removing mem_manager.o(i.block_init), (32 bytes).
    Removing mem_manager.o(i.get_block_cat), (60 bytes).
    Removing mem_manager.o(i.get_block_size), (24 bytes).
    Removing mem_manager.o(i.nrf_calloc), (36 bytes).
    Removing mem_manager.o(i.nrf_free), (40 bytes).
    Removing mem_manager.o(i.nrf_malloc), (24 bytes).
    Removing mem_manager.o(i.nrf_mem_init), (24 bytes).
    Removing mem_manager.o(i.nrf_mem_reserve), (128 bytes).
    Removing mem_manager.o(i.nrf_realloc), (2 bytes).
    Removing mem_manager.o(.bss), (32 bytes).
    Removing mem_manager.o(.constdata), (112 bytes).
    Removing mem_manager.o(.constdata), (13 bytes).
    Removing mem_manager.o(.constdata), (16 bytes).
    Removing mem_manager.o(.constdata), (11 bytes).
    Removing mem_manager.o(.constdata), (9 bytes).
    Removing mem_manager.o(.data), (8 bytes).
    Removing nrf_assert.o(.rev16_text), (4 bytes).
    Removing nrf_assert.o(.revsh_text), (4 bytes).
    Removing nrf_assert.o(.rrx_text), (6 bytes).
    Removing nrf_assert.o(i.assert_nrf_callback), (20 bytes).
    Removing nrf_atomic.o(.rev16_text), (4 bytes).
    Removing nrf_atomic.o(.revsh_text), (4 bytes).
    Removing nrf_atomic.o(.rrx_text), (6 bytes).
    Removing nrf_atomic.o(i.nrf_atomic_flag_clear_fetch), (6 bytes).
    Removing nrf_atomic.o(i.nrf_atomic_flag_set), (6 bytes).
    Removing nrf_atomic.o(i.nrf_atomic_u32_add), (12 bytes).
    Removing nrf_atomic.o(i.nrf_atomic_u32_cmp_exch), (4 bytes).
    Removing nrf_atomic.o(i.nrf_atomic_u32_fetch_add), (10 bytes).
    Removing nrf_atomic.o(i.nrf_atomic_u32_fetch_and), (10 bytes).
    Removing nrf_atomic.o(i.nrf_atomic_u32_fetch_store), (10 bytes).
    Removing nrf_atomic.o(i.nrf_atomic_u32_fetch_sub), (10 bytes).
    Removing nrf_atomic.o(i.nrf_atomic_u32_fetch_sub_hs), (10 bytes).
    Removing nrf_atomic.o(i.nrf_atomic_u32_fetch_xor), (10 bytes).
    Removing nrf_atomic.o(i.nrf_atomic_u32_or), (12 bytes).
    Removing nrf_atomic.o(i.nrf_atomic_u32_store), (12 bytes).
    Removing nrf_atomic.o(i.nrf_atomic_u32_sub), (12 bytes).
    Removing nrf_atomic.o(i.nrf_atomic_u32_sub_hs), (12 bytes).
    Removing nrf_atomic.o(i.nrf_atomic_u32_xor), (12 bytes).
    Removing nrf_balloc.o(.rev16_text), (4 bytes).
    Removing nrf_balloc.o(.revsh_text), (4 bytes).
    Removing nrf_balloc.o(.rrx_text), (6 bytes).
    Removing nrf_fprintf.o(.rev16_text), (4 bytes).
    Removing nrf_fprintf.o(.revsh_text), (4 bytes).
    Removing nrf_fprintf.o(.rrx_text), (6 bytes).
    Removing nrf_fprintf.o(i.nrf_fprintf), (26 bytes).
    Removing nrf_fprintf.o(i.nrf_fprintf_buffer_flush), (24 bytes).
    Removing nrf_fprintf_format.o(.rev16_text), (4 bytes).
    Removing nrf_fprintf_format.o(.revsh_text), (4 bytes).
    Removing nrf_fprintf_format.o(.rrx_text), (6 bytes).
    Removing nrf_fprintf_format.o(i.buffer_add), (46 bytes).
    Removing nrf_fprintf_format.o(i.int_print), (166 bytes).
    Removing nrf_fprintf_format.o(i.nrf_fprintf_fmt), (474 bytes).
    Removing nrf_fprintf_format.o(i.unsigned_print), (180 bytes).
    Removing nrf_fprintf_format.o(.constdata), (16 bytes).
    Removing nrf_fstorage.o(.rev16_text), (4 bytes).
    Removing nrf_fstorage.o(.revsh_text), (4 bytes).
    Removing nrf_fstorage.o(.rrx_text), (6 bytes).
    Removing nrf_fstorage.o(i.nrf_fstorage_read), (48 bytes).
    Removing nrf_fstorage.o(i.nrf_fstorage_rmap), (14 bytes).
    Removing nrf_fstorage.o(i.nrf_fstorage_uninit), (20 bytes).
    Removing nrf_fstorage.o(i.nrf_fstorage_wmap), (14 bytes).
    Removing nrf_fstorage.o(.constdata), (18 bytes).
    Removing nrf_fstorage.o(.constdata), (20 bytes).
    Removing nrf_fstorage.o(.constdata), (18 bytes).
    Removing nrf_fstorage.o(.constdata), (19 bytes).
    Removing nrf_fstorage.o(.constdata), (19 bytes).
    Removing nrf_fstorage_nvmc.o(.rev16_text), (4 bytes).
    Removing nrf_fstorage_nvmc.o(.revsh_text), (4 bytes).
    Removing nrf_fstorage_nvmc.o(.rrx_text), (6 bytes).
    Removing nrf_memobj.o(.rev16_text), (4 bytes).
    Removing nrf_memobj.o(.revsh_text), (4 bytes).
    Removing nrf_memobj.o(.rrx_text), (6 bytes).
    Removing nrf_memobj.o(i.memobj_op), (126 bytes).
    Removing nrf_memobj.o(i.nrf_memobj_alloc), (96 bytes).
    Removing nrf_memobj.o(i.nrf_memobj_free), (50 bytes).
    Removing nrf_memobj.o(i.nrf_memobj_get), (8 bytes).
    Removing nrf_memobj.o(i.nrf_memobj_pool_init), (4 bytes).
    Removing nrf_memobj.o(i.nrf_memobj_put), (30 bytes).
    Removing nrf_memobj.o(i.nrf_memobj_read), (16 bytes).
    Removing nrf_memobj.o(i.nrf_memobj_write), (16 bytes).
    Removing nrf_queue.o(.rev16_text), (4 bytes).
    Removing nrf_queue.o(.revsh_text), (4 bytes).
    Removing nrf_queue.o(.rrx_text), (6 bytes).
    Removing nrf_ringbuf.o(.rev16_text), (4 bytes).
    Removing nrf_ringbuf.o(.revsh_text), (4 bytes).
    Removing nrf_ringbuf.o(.rrx_text), (6 bytes).
    Removing nrf_ringbuf.o(i.nrf_ringbuf_alloc), (112 bytes).
    Removing nrf_ringbuf.o(i.nrf_ringbuf_cpy_get), (128 bytes).
    Removing nrf_ringbuf.o(i.nrf_ringbuf_cpy_put), (118 bytes).
    Removing nrf_ringbuf.o(i.nrf_ringbuf_free), (38 bytes).
    Removing nrf_ringbuf.o(i.nrf_ringbuf_get), (112 bytes).
    Removing nrf_ringbuf.o(i.nrf_ringbuf_init), (28 bytes).
    Removing nrf_ringbuf.o(i.nrf_ringbuf_put), (48 bytes).
    Removing nrf_strerror.o(.rev16_text), (4 bytes).
    Removing nrf_strerror.o(.revsh_text), (4 bytes).
    Removing nrf_strerror.o(.rrx_text), (6 bytes).
    Removing nrf_strerror.o(i.nrf_strerror_find), (56 bytes).
    Removing nrf_strerror.o(i.nrf_strerror_get), (20 bytes).
    Removing nrf_strerror.o(.constdata), (300 bytes).
    Removing nrf_strerror.o(.conststring), (957 bytes).
    Removing sha256.o(.rev16_text), (4 bytes).
    Removing sha256.o(.revsh_text), (4 bytes).
    Removing sha256.o(.rrx_text), (6 bytes).
    Removing slip.o(.rev16_text), (4 bytes).
    Removing slip.o(.revsh_text), (4 bytes).
    Removing slip.o(.rrx_text), (6 bytes).
    Removing nrf_log_frontend.o(.rev16_text), (4 bytes).
    Removing nrf_log_frontend.o(.revsh_text), (4 bytes).
    Removing nrf_log_frontend.o(.rrx_text), (6 bytes).
    Removing nrf_log_str_formatter.o(.rev16_text), (4 bytes).
    Removing nrf_log_str_formatter.o(.revsh_text), (4 bytes).
    Removing nrf_log_str_formatter.o(.rrx_text), (6 bytes).
    Removing nrf_dfu_serial.o(.rev16_text), (4 bytes).
    Removing nrf_dfu_serial.o(.revsh_text), (4 bytes).
    Removing nrf_dfu_serial.o(.rrx_text), (6 bytes).
    Removing pb_decode.o(i.pb_close_string_substream), (6 bytes).
    Removing pb_decode.o(i.pb_decode_delimited), (36 bytes).
    Removing arm_startup_nrf52820.o(HEAP), (0 bytes).
    Removing system_nrf52.o(.rev16_text), (4 bytes).
    Removing system_nrf52.o(.revsh_text), (4 bytes).
    Removing system_nrf52.o(.rrx_text), (6 bytes).
    Removing system_nrf52.o(i.SystemCoreClockUpdate), (16 bytes).
    Removing system_nrf52.o(i.nvmc_wait), (16 bytes).
    Removing uECC.c.o(.text), (0 bytes).
    Removing uECC.c.o(.data), (0 bytes).
    Removing uECC.c.o(.bss), (0 bytes).
    Removing uECC.c.o(.text.uECC_vli_cmp), (50 bytes).
    Removing uECC.c.o(.text.omega_mult_secp160r1), (64 bytes).
    Removing uECC.c.o(.text.vli_mmod_fast_secp160r1), (132 bytes).
    Removing uECC.c.o(.text.vli_mmod_fast_secp192r1), (148 bytes).
    Removing uECC.c.o(.text.vli_mmod_fast_secp224r1), (224 bytes).
    Removing uECC.c.o(.text.x_side_secp256k1), (46 bytes).
    Removing uECC.c.o(.text.omega_mult_secp256k1), (58 bytes).
    Removing uECC.c.o(.text.vli_mmod_fast_secp256k1), (132 bytes).
    Removing uECC.c.o(.text.XYcZ_addC), (284 bytes).
    Removing uECC.c.o(.text.regularize_k), (94 bytes).
    Removing uECC.c.o(.text.uECC_generate_random_int), (120 bytes).
    Removing uECC.c.o(.text.HMAC_init), (66 bytes).
    Removing uECC.c.o(.text.HMAC_update), (4 bytes).
    Removing uECC.c.o(.text.HMAC_finish), (94 bytes).
    Removing uECC.c.o(.text.update_V), (36 bytes).
    Removing uECC.c.o(.text.EccPoint_mult), (418 bytes).
    Removing uECC.c.o(.text.EccPoint_compute_public_key), (124 bytes).
    Removing uECC.c.o(.text.uECC_sign_with_k_internal), (420 bytes).
    Removing uECC.c.o(.text.double_jacobian_secp256k1), (268 bytes).
    Removing uECC.c.o(.text.uECC_set_rng), (12 bytes).
    Removing uECC.c.o(.text.uECC_get_rng), (12 bytes).
    Removing uECC.c.o(.text.uECC_curve_private_key_size), (16 bytes).
    Removing uECC.c.o(.text.uECC_curve_public_key_size), (8 bytes).
    Removing uECC.c.o(.text.uECC_secp160r1), (8 bytes).
    Removing uECC.c.o(.text.uECC_secp192r1), (8 bytes).
    Removing uECC.c.o(.text.uECC_secp224r1), (8 bytes).
    Removing uECC.c.o(.text.uECC_secp256k1), (8 bytes).
    Removing uECC.c.o(.text.uECC_make_key), (70 bytes).
    Removing uECC.c.o(.text.uECC_shared_secret), (168 bytes).
    Removing uECC.c.o(.text.uECC_valid_public_key), (132 bytes).
    Removing uECC.c.o(.text.uECC_compute_public_key), (70 bytes).
    Removing uECC.c.o(.text.uECC_sign_with_k), (58 bytes).
    Removing uECC.c.o(.text.uECC_sign), (86 bytes).
    Removing uECC.c.o(.text.uECC_sign_deterministic), (412 bytes).
    Removing uECC.c.o(.bss.g_rng_function), (4 bytes).
    Removing uECC.c.o(.rodata.curve_secp160r1), (176 bytes).
    Removing uECC.c.o(.rodata.curve_secp192r1), (176 bytes).
    Removing uECC.c.o(.rodata.curve_secp224r1), (176 bytes).
    Removing uECC.c.o(.rodata.curve_secp256k1), (176 bytes).

390 unused section(s) (total 12249 bytes) removed from the image.

==============================================================================

Image Symbol Table

    Local Symbols

    Symbol Name                              Value     Ov Type        Size  Object(Section)

    ../clib/microlib/init/entry.s            0x00000000   Number         0  entry10b.o ABSOLUTE
    ../clib/microlib/init/entry.s            0x00000000   Number         0  entry7b.o ABSOLUTE
    ../clib/microlib/init/entry.s            0x00000000   Number         0  entry8b.o ABSOLUTE
    ../clib/microlib/init/entry.s            0x00000000   Number         0  entry9a.o ABSOLUTE
    ../clib/microlib/init/entry.s            0x00000000   Number         0  entry9b.o ABSOLUTE
    ../clib/microlib/init/entry.s            0x00000000   Number         0  entry10a.o ABSOLUTE
    ../clib/microlib/init/entry.s            0x00000000   Number         0  entry11a.o ABSOLUTE
    ../clib/microlib/init/entry.s            0x00000000   Number         0  entry.o ABSOLUTE
    ../clib/microlib/init/entry.s            0x00000000   Number         0  entry2.o ABSOLUTE
    ../clib/microlib/init/entry.s            0x00000000   Number         0  entry11b.o ABSOLUTE
    ../clib/microlib/init/entry.s            0x00000000   Number         0  entry8a.o ABSOLUTE
    ../clib/microlib/init/entry.s            0x00000000   Number         0  entry5.o ABSOLUTE
    ../clib/microlib/init/entry.s            0x00000000   Number         0  entry7a.o ABSOLUTE
    ../clib/microlib/longlong.c              0x00000000   Number         0  llshl.o ABSOLUTE
    ../clib/microlib/string/memcmp.c         0x00000000   Number         0  memcmp.o ABSOLUTE
    ../clib/microlib/string/memcpy.c         0x00000000   Number         0  memcpyb.o ABSOLUTE
    ../clib/microlib/string/memcpy.c         0x00000000   Number         0  memcpya.o ABSOLUTE
    ../clib/microlib/string/memset.c         0x00000000   Number         0  memseta.o ABSOLUTE
    ../clib/microlib/string/memset.c         0x00000000   Number         0  memset.o ABSOLUTE
    ../clib/microlib/string/strlen.c         0x00000000   Number         0  strlen.o ABSOLUTE
    ..\..\..\..\..\components\boards\boards.c 0x00000000   Number         0  boards.o ABSOLUTE
    ..\..\..\..\..\components\drivers_nrf\nrf_soc_nosd\nrf_nvic.c 0x00000000   Number         0  nrf_nvic.o ABSOLUTE
    ..\..\..\..\..\components\drivers_nrf\nrf_soc_nosd\nrf_soc.c 0x00000000   Number         0  nrf_soc.o ABSOLUTE
    ..\..\..\..\..\components\libraries\atomic\nrf_atomic.c 0x00000000   Number         0  nrf_atomic.o ABSOLUTE
    ..\..\..\..\..\components\libraries\balloc\nrf_balloc.c 0x00000000   Number         0  nrf_balloc.o ABSOLUTE
    ..\..\..\..\..\components\libraries\bootloader\dfu\dfu-cc.pb.c 0x00000000   Number         0  dfu-cc.pb.o ABSOLUTE
    ..\..\..\..\..\components\libraries\bootloader\dfu\nrf_dfu.c 0x00000000   Number         0  nrf_dfu.o ABSOLUTE
    ..\..\..\..\..\components\libraries\bootloader\dfu\nrf_dfu_flash.c 0x00000000   Number         0  nrf_dfu_flash.o ABSOLUTE
    ..\..\..\..\..\components\libraries\bootloader\dfu\nrf_dfu_handling_error.c 0x00000000   Number         0  nrf_dfu_handling_error.o ABSOLUTE
    ..\..\..\..\..\components\libraries\bootloader\dfu\nrf_dfu_mbr.c 0x00000000   Number         0  nrf_dfu_mbr.o ABSOLUTE
    ..\..\..\..\..\components\libraries\bootloader\dfu\nrf_dfu_req_handler.c 0x00000000   Number         0  nrf_dfu_req_handler.o ABSOLUTE
    ..\..\..\..\..\components\libraries\bootloader\dfu\nrf_dfu_settings.c 0x00000000   Number         0  nrf_dfu_settings.o ABSOLUTE
    ..\..\..\..\..\components\libraries\bootloader\dfu\nrf_dfu_transport.c 0x00000000   Number         0  nrf_dfu_transport.o ABSOLUTE
    ..\..\..\..\..\components\libraries\bootloader\dfu\nrf_dfu_utils.c 0x00000000   Number         0  nrf_dfu_utils.o ABSOLUTE
    ..\..\..\..\..\components\libraries\bootloader\dfu\nrf_dfu_validation.c 0x00000000   Number         0  nrf_dfu_validation.o ABSOLUTE
    ..\..\..\..\..\components\libraries\bootloader\dfu\nrf_dfu_ver_validation.c 0x00000000   Number         0  nrf_dfu_ver_validation.o ABSOLUTE
    ..\..\..\..\..\components\libraries\bootloader\nrf_bootloader.c 0x00000000   Number         0  nrf_bootloader.o ABSOLUTE
    ..\..\..\..\..\components\libraries\bootloader\nrf_bootloader_app_start.c 0x00000000   Number         0  nrf_bootloader_app_start.o ABSOLUTE
    ..\..\..\..\..\components\libraries\bootloader\nrf_bootloader_app_start_final.c 0x00000000   Number         0  nrf_bootloader_app_start_final.o ABSOLUTE
    ..\..\..\..\..\components\libraries\bootloader\nrf_bootloader_dfu_timers.c 0x00000000   Number         0  nrf_bootloader_dfu_timers.o ABSOLUTE
    ..\..\..\..\..\components\libraries\bootloader\nrf_bootloader_fw_activation.c 0x00000000   Number         0  nrf_bootloader_fw_activation.o ABSOLUTE
    ..\..\..\..\..\components\libraries\bootloader\nrf_bootloader_info.c 0x00000000   Number         0  nrf_bootloader_info.o ABSOLUTE
    ..\..\..\..\..\components\libraries\bootloader\nrf_bootloader_wdt.c 0x00000000   Number         0  nrf_bootloader_wdt.o ABSOLUTE
    ..\..\..\..\..\components\libraries\bootloader\serial_dfu\nrf_dfu_serial.c 0x00000000   Number         0  nrf_dfu_serial.o ABSOLUTE
    ..\..\..\..\..\components\libraries\bootloader\serial_dfu\nrf_dfu_serial_uart.c 0x00000000   Number         0  nrf_dfu_serial_uart.o ABSOLUTE
    ..\..\..\..\..\components\libraries\crc32\crc32.c 0x00000000   Number         0  crc32.o ABSOLUTE
    ..\..\..\..\..\components\libraries\crypto\backend\micro_ecc\micro_ecc_backend_ecc.c 0x00000000   Number         0  micro_ecc_backend_ecc.o ABSOLUTE
    ..\..\..\..\..\components\libraries\crypto\backend\micro_ecc\micro_ecc_backend_ecdh.c 0x00000000   Number         0  micro_ecc_backend_ecdh.o ABSOLUTE
    ..\..\..\..\..\components\libraries\crypto\backend\micro_ecc\micro_ecc_backend_ecdsa.c 0x00000000   Number         0  micro_ecc_backend_ecdsa.o ABSOLUTE
    ..\..\..\..\..\components\libraries\crypto\backend\nrf_sw\nrf_sw_backend_hash.c 0x00000000   Number         0  nrf_sw_backend_hash.o ABSOLUTE
    ..\..\..\..\..\components\libraries\crypto\backend\oberon\oberon_backend_chacha_poly_aead.c 0x00000000   Number         0  oberon_backend_chacha_poly_aead.o ABSOLUTE
    ..\..\..\..\..\components\libraries\crypto\backend\oberon\oberon_backend_ecc.c 0x00000000   Number         0  oberon_backend_ecc.o ABSOLUTE
    ..\..\..\..\..\components\libraries\crypto\backend\oberon\oberon_backend_ecdh.c 0x00000000   Number         0  oberon_backend_ecdh.o ABSOLUTE
    ..\..\..\..\..\components\libraries\crypto\backend\oberon\oberon_backend_ecdsa.c 0x00000000   Number         0  oberon_backend_ecdsa.o ABSOLUTE
    ..\..\..\..\..\components\libraries\crypto\backend\oberon\oberon_backend_eddsa.c 0x00000000   Number         0  oberon_backend_eddsa.o ABSOLUTE
    ..\..\..\..\..\components\libraries\crypto\backend\oberon\oberon_backend_hash.c 0x00000000   Number         0  oberon_backend_hash.o ABSOLUTE
    ..\..\..\..\..\components\libraries\crypto\backend\oberon\oberon_backend_hmac.c 0x00000000   Number         0  oberon_backend_hmac.o ABSOLUTE
    ..\..\..\..\..\components\libraries\crypto\nrf_crypto_ecc.c 0x00000000   Number         0  nrf_crypto_ecc.o ABSOLUTE
    ..\..\..\..\..\components\libraries\crypto\nrf_crypto_ecdsa.c 0x00000000   Number         0  nrf_crypto_ecdsa.o ABSOLUTE
    ..\..\..\..\..\components\libraries\crypto\nrf_crypto_hash.c 0x00000000   Number         0  nrf_crypto_hash.o ABSOLUTE
    ..\..\..\..\..\components\libraries\crypto\nrf_crypto_init.c 0x00000000   Number         0  nrf_crypto_init.o ABSOLUTE
    ..\..\..\..\..\components\libraries\crypto\nrf_crypto_shared.c 0x00000000   Number         0  nrf_crypto_shared.o ABSOLUTE
    ..\..\..\..\..\components\libraries\fstorage\nrf_fstorage.c 0x00000000   Number         0  nrf_fstorage.o ABSOLUTE
    ..\..\..\..\..\components\libraries\fstorage\nrf_fstorage_nvmc.c 0x00000000   Number         0  nrf_fstorage_nvmc.o ABSOLUTE
    ..\..\..\..\..\components\libraries\log\src\nrf_log_frontend.c 0x00000000   Number         0  nrf_log_frontend.o ABSOLUTE
    ..\..\..\..\..\components\libraries\log\src\nrf_log_str_formatter.c 0x00000000   Number         0  nrf_log_str_formatter.o ABSOLUTE
    ..\..\..\..\..\components\libraries\mem_manager\mem_manager.c 0x00000000   Number         0  mem_manager.o ABSOLUTE
    ..\..\..\..\..\components\libraries\memobj\nrf_memobj.c 0x00000000   Number         0  nrf_memobj.o ABSOLUTE
    ..\..\..\..\..\components\libraries\queue\nrf_queue.c 0x00000000   Number         0  nrf_queue.o ABSOLUTE
    ..\..\..\..\..\components\libraries\ringbuf\nrf_ringbuf.c 0x00000000   Number         0  nrf_ringbuf.o ABSOLUTE
    ..\..\..\..\..\components\libraries\scheduler\app_scheduler.c 0x00000000   Number         0  app_scheduler.o ABSOLUTE
    ..\..\..\..\..\components\libraries\sha256\sha256.c 0x00000000   Number         0  sha256.o ABSOLUTE
    ..\..\..\..\..\components\libraries\slip\slip.c 0x00000000   Number         0  slip.o ABSOLUTE
    ..\..\..\..\..\components\libraries\strerror\nrf_strerror.c 0x00000000   Number         0  nrf_strerror.o ABSOLUTE
    ..\..\..\..\..\components\libraries\util\app_error_weak.c 0x00000000   Number         0  app_error_weak.o ABSOLUTE
    ..\..\..\..\..\components\libraries\util\app_util_platform.c 0x00000000   Number         0  app_util_platform.o ABSOLUTE
    ..\..\..\..\..\components\libraries\util\nrf_assert.c 0x00000000   Number         0  nrf_assert.o ABSOLUTE
    ..\..\..\..\..\external\fprintf\nrf_fprintf.c 0x00000000   Number         0  nrf_fprintf.o ABSOLUTE
    ..\..\..\..\..\external\fprintf\nrf_fprintf_format.c 0x00000000   Number         0  nrf_fprintf_format.o ABSOLUTE
    ..\..\..\..\..\external\nano-pb\pb_common.c 0x00000000   Number         0  pb_common.o ABSOLUTE
    ..\..\..\..\..\external\nano-pb\pb_decode.c 0x00000000   Number         0  pb_decode.o ABSOLUTE
    ..\..\..\..\..\integration\nrfx\legacy\nrf_drv_uart.c 0x00000000   Number         0  nrf_drv_uart.o ABSOLUTE
    ..\..\..\..\..\modules\nrfx\drivers\src\nrfx_uart.c 0x00000000   Number         0  nrfx_uart.o ABSOLUTE
    ..\..\..\..\..\modules\nrfx\drivers\src\nrfx_uarte.c 0x00000000   Number         0  nrfx_uarte.o ABSOLUTE
    ..\..\..\..\..\modules\nrfx\drivers\src\prs\nrfx_prs.c 0x00000000   Number         0  nrfx_prs.o ABSOLUTE
    ..\..\..\..\..\modules\nrfx\hal\nrf_nvmc.c 0x00000000   Number         0  nrf_nvmc.o ABSOLUTE
    ..\..\..\..\..\modules\nrfx\soc\nrfx_atomic.c 0x00000000   Number         0  nrfx_atomic.o ABSOLUTE
    ..\..\..\dfu_public_key.c                0x00000000   Number         0  dfu_public_key.o ABSOLUTE
    ..\..\main.c                             0x00000000   Number         0  main.o ABSOLUTE
    ..\\..\\..\\..\\..\\components\\boards\\boards.c 0x00000000   Number         0  boards.o ABSOLUTE
    ..\\..\\..\\..\\..\\components\\drivers_nrf\\nrf_soc_nosd\\nrf_nvic.c 0x00000000   Number         0  nrf_nvic.o ABSOLUTE
    ..\\..\\..\\..\\..\\components\\drivers_nrf\\nrf_soc_nosd\\nrf_soc.c 0x00000000   Number         0  nrf_soc.o ABSOLUTE
    ..\\..\\..\\..\\..\\components\\libraries\\atomic\\nrf_atomic.c 0x00000000   Number         0  nrf_atomic.o ABSOLUTE
    ..\\..\\..\\..\\..\\components\\libraries\\balloc\\nrf_balloc.c 0x00000000   Number         0  nrf_balloc.o ABSOLUTE
    ..\\..\\..\\..\\..\\components\\libraries\\bootloader\\dfu\\nrf_dfu.c 0x00000000   Number         0  nrf_dfu.o ABSOLUTE
    ..\\..\\..\\..\\..\\components\\libraries\\bootloader\\dfu\\nrf_dfu_flash.c 0x00000000   Number         0  nrf_dfu_flash.o ABSOLUTE
    ..\\..\\..\\..\\..\\components\\libraries\\bootloader\\dfu\\nrf_dfu_handling_error.c 0x00000000   Number         0  nrf_dfu_handling_error.o ABSOLUTE
    ..\\..\\..\\..\\..\\components\\libraries\\bootloader\\dfu\\nrf_dfu_mbr.c 0x00000000   Number         0  nrf_dfu_mbr.o ABSOLUTE
    ..\\..\\..\\..\\..\\components\\libraries\\bootloader\\dfu\\nrf_dfu_req_handler.c 0x00000000   Number         0  nrf_dfu_req_handler.o ABSOLUTE
    ..\\..\\..\\..\\..\\components\\libraries\\bootloader\\dfu\\nrf_dfu_settings.c 0x00000000   Number         0  nrf_dfu_settings.o ABSOLUTE
    ..\\..\\..\\..\\..\\components\\libraries\\bootloader\\dfu\\nrf_dfu_transport.c 0x00000000   Number         0  nrf_dfu_transport.o ABSOLUTE
    ..\\..\\..\\..\\..\\components\\libraries\\bootloader\\dfu\\nrf_dfu_utils.c 0x00000000   Number         0  nrf_dfu_utils.o ABSOLUTE
    ..\\..\\..\\..\\..\\components\\libraries\\bootloader\\dfu\\nrf_dfu_validation.c 0x00000000   Number         0  nrf_dfu_validation.o ABSOLUTE
    ..\\..\\..\\..\\..\\components\\libraries\\bootloader\\dfu\\nrf_dfu_ver_validation.c 0x00000000   Number         0  nrf_dfu_ver_validation.o ABSOLUTE
    ..\\..\\..\\..\\..\\components\\libraries\\bootloader\\nrf_bootloader.c 0x00000000   Number         0  nrf_bootloader.o ABSOLUTE
    ..\\..\\..\\..\\..\\components\\libraries\\bootloader\\nrf_bootloader_app_start.c 0x00000000   Number         0  nrf_bootloader_app_start.o ABSOLUTE
    ..\\..\\..\\..\\..\\components\\libraries\\bootloader\\nrf_bootloader_app_start_final.c 0x00000000   Number         0  nrf_bootloader_app_start_final.o ABSOLUTE
    ..\\..\\..\\..\\..\\components\\libraries\\bootloader\\nrf_bootloader_dfu_timers.c 0x00000000   Number         0  nrf_bootloader_dfu_timers.o ABSOLUTE
    ..\\..\\..\\..\\..\\components\\libraries\\bootloader\\nrf_bootloader_fw_activation.c 0x00000000   Number         0  nrf_bootloader_fw_activation.o ABSOLUTE
    ..\\..\\..\\..\\..\\components\\libraries\\bootloader\\nrf_bootloader_info.c 0x00000000   Number         0  nrf_bootloader_info.o ABSOLUTE
    ..\\..\\..\\..\\..\\components\\libraries\\bootloader\\nrf_bootloader_wdt.c 0x00000000   Number         0  nrf_bootloader_wdt.o ABSOLUTE
    ..\\..\\..\\..\\..\\components\\libraries\\bootloader\\serial_dfu\\nrf_dfu_serial.c 0x00000000   Number         0  nrf_dfu_serial.o ABSOLUTE
    ..\\..\\..\\..\\..\\components\\libraries\\bootloader\\serial_dfu\\nrf_dfu_serial_uart.c 0x00000000   Number         0  nrf_dfu_serial_uart.o ABSOLUTE
    ..\\..\\..\\..\\..\\components\\libraries\\crc32\\crc32.c 0x00000000   Number         0  crc32.o ABSOLUTE
    ..\\..\\..\\..\\..\\components\\libraries\\crypto\\backend\\micro_ecc\\micro_ecc_backend_ecc.c 0x00000000   Number         0  micro_ecc_backend_ecc.o ABSOLUTE
    ..\\..\\..\\..\\..\\components\\libraries\\crypto\\backend\\micro_ecc\\micro_ecc_backend_ecdh.c 0x00000000   Number         0  micro_ecc_backend_ecdh.o ABSOLUTE
    ..\\..\\..\\..\\..\\components\\libraries\\crypto\\backend\\micro_ecc\\micro_ecc_backend_ecdsa.c 0x00000000   Number         0  micro_ecc_backend_ecdsa.o ABSOLUTE
    ..\\..\\..\\..\\..\\components\\libraries\\crypto\\backend\\nrf_sw\\nrf_sw_backend_hash.c 0x00000000   Number         0  nrf_sw_backend_hash.o ABSOLUTE
    ..\\..\\..\\..\\..\\components\\libraries\\crypto\\backend\\oberon\\oberon_backend_chacha_poly_aead.c 0x00000000   Number         0  oberon_backend_chacha_poly_aead.o ABSOLUTE
    ..\\..\\..\\..\\..\\components\\libraries\\crypto\\backend\\oberon\\oberon_backend_hash.c 0x00000000   Number         0  oberon_backend_hash.o ABSOLUTE
    ..\\..\\..\\..\\..\\components\\libraries\\crypto\\backend\\oberon\\oberon_backend_hmac.c 0x00000000   Number         0  oberon_backend_hmac.o ABSOLUTE
    ..\\..\\..\\..\\..\\components\\libraries\\crypto\\nrf_crypto_ecc.c 0x00000000   Number         0  nrf_crypto_ecc.o ABSOLUTE
    ..\\..\\..\\..\\..\\components\\libraries\\crypto\\nrf_crypto_ecdsa.c 0x00000000   Number         0  nrf_crypto_ecdsa.o ABSOLUTE
    ..\\..\\..\\..\\..\\components\\libraries\\crypto\\nrf_crypto_hash.c 0x00000000   Number         0  nrf_crypto_hash.o ABSOLUTE
    ..\\..\\..\\..\\..\\components\\libraries\\crypto\\nrf_crypto_init.c 0x00000000   Number         0  nrf_crypto_init.o ABSOLUTE
    ..\\..\\..\\..\\..\\components\\libraries\\crypto\\nrf_crypto_shared.c 0x00000000   Number         0  nrf_crypto_shared.o ABSOLUTE
    ..\\..\\..\\..\\..\\components\\libraries\\fstorage\\nrf_fstorage.c 0x00000000   Number         0  nrf_fstorage.o ABSOLUTE
    ..\\..\\..\\..\\..\\components\\libraries\\fstorage\\nrf_fstorage_nvmc.c 0x00000000   Number         0  nrf_fstorage_nvmc.o ABSOLUTE
    ..\\..\\..\\..\\..\\components\\libraries\\log\\src\\nrf_log_frontend.c 0x00000000   Number         0  nrf_log_frontend.o ABSOLUTE
    ..\\..\\..\\..\\..\\components\\libraries\\log\\src\\nrf_log_str_formatter.c 0x00000000   Number         0  nrf_log_str_formatter.o ABSOLUTE
    ..\\..\\..\\..\\..\\components\\libraries\\mem_manager\\mem_manager.c 0x00000000   Number         0  mem_manager.o ABSOLUTE
    ..\\..\\..\\..\\..\\components\\libraries\\memobj\\nrf_memobj.c 0x00000000   Number         0  nrf_memobj.o ABSOLUTE
    ..\\..\\..\\..\\..\\components\\libraries\\queue\\nrf_queue.c 0x00000000   Number         0  nrf_queue.o ABSOLUTE
    ..\\..\\..\\..\\..\\components\\libraries\\ringbuf\\nrf_ringbuf.c 0x00000000   Number         0  nrf_ringbuf.o ABSOLUTE
    ..\\..\\..\\..\\..\\components\\libraries\\scheduler\\app_scheduler.c 0x00000000   Number         0  app_scheduler.o ABSOLUTE
    ..\\..\\..\\..\\..\\components\\libraries\\sha256\\sha256.c 0x00000000   Number         0  sha256.o ABSOLUTE
    ..\\..\\..\\..\\..\\components\\libraries\\slip\\slip.c 0x00000000   Number         0  slip.o ABSOLUTE
    ..\\..\\..\\..\\..\\components\\libraries\\strerror\\nrf_strerror.c 0x00000000   Number         0  nrf_strerror.o ABSOLUTE
    ..\\..\\..\\..\\..\\components\\libraries\\util\\app_error_weak.c 0x00000000   Number         0  app_error_weak.o ABSOLUTE
    ..\\..\\..\\..\\..\\components\\libraries\\util\\app_util_platform.c 0x00000000   Number         0  app_util_platform.o ABSOLUTE
    ..\\..\\..\\..\\..\\components\\libraries\\util\\nrf_assert.c 0x00000000   Number         0  nrf_assert.o ABSOLUTE
    ..\\..\\..\\..\\..\\external\\fprintf\\nrf_fprintf.c 0x00000000   Number         0  nrf_fprintf.o ABSOLUTE
    ..\\..\\..\\..\\..\\external\\fprintf\\nrf_fprintf_format.c 0x00000000   Number         0  nrf_fprintf_format.o ABSOLUTE
    ..\\..\\..\\..\\..\\integration\\nrfx\\legacy\\nrf_drv_uart.c 0x00000000   Number         0  nrf_drv_uart.o ABSOLUTE
    ..\\..\\..\\..\\..\\modules\\nrfx\\drivers\\src\\nrfx_uart.c 0x00000000   Number         0  nrfx_uart.o ABSOLUTE
    ..\\..\\..\\..\\..\\modules\\nrfx\\drivers\\src\\nrfx_uarte.c 0x00000000   Number         0  nrfx_uarte.o ABSOLUTE
    ..\\..\\..\\..\\..\\modules\\nrfx\\drivers\\src\\prs\\nrfx_prs.c 0x00000000   Number         0  nrfx_prs.o ABSOLUTE
    ..\\..\\..\\..\\..\\modules\\nrfx\\hal\\nrf_nvmc.c 0x00000000   Number         0  nrf_nvmc.o ABSOLUTE
    ..\\..\\..\\..\\..\\modules\\nrfx\\soc\\nrfx_atomic.c 0x00000000   Number         0  nrfx_atomic.o ABSOLUTE
    ..\\..\\main.c                           0x00000000   Number         0  main.o ABSOLUTE
    RTE\Device\nRF52820_xxAA\arm_startup_nrf52820.s 0x00000000   Number         0  arm_startup_nrf52820.o ABSOLUTE
    RTE\Device\nRF52820_xxAA\system_nrf52.c  0x00000000   Number         0  system_nrf52.o ABSOLUTE
    RTE\\Device\\nRF52820_xxAA\\system_nrf52.c 0x00000000   Number         0  system_nrf52.o ABSOLUTE
    dc.s                                     0x00000000   Number         0  dc.o ABSOLUTE
    handlers.s                               0x00000000   Number         0  handlers.o ABSOLUTE
    init.s                                   0x00000000   Number         0  init.o ABSOLUTE
    uECC.c                                   0x00000000   Number         0  uECC.c.o ABSOLUTE
    RESET                                    0x00038000   Section      512  arm_startup_nrf52820.o(RESET)
    .ARM.Collect$$$$00000000                 0x00038200   Section        0  entry.o(.ARM.Collect$$$$00000000)
    .ARM.Collect$$$$00000001                 0x00038200   Section        4  entry2.o(.ARM.Collect$$$$00000001)
    .ARM.Collect$$$$00000004                 0x00038204   Section        4  entry5.o(.ARM.Collect$$$$00000004)
    .ARM.Collect$$$$00000008                 0x00038208   Section        0  entry7b.o(.ARM.Collect$$$$00000008)
    .ARM.Collect$$$$0000000A                 0x00038208   Section        0  entry8b.o(.ARM.Collect$$$$0000000A)
    .ARM.Collect$$$$0000000B                 0x00038208   Section        8  entry9a.o(.ARM.Collect$$$$0000000B)
    .ARM.Collect$$$$0000000D                 0x00038210   Section        0  entry10a.o(.ARM.Collect$$$$0000000D)
    .ARM.Collect$$$$0000000F                 0x00038210   Section        0  entry11a.o(.ARM.Collect$$$$0000000F)
    .ARM.Collect$$$$00002712                 0x00038210   Section        4  entry2.o(.ARM.Collect$$$$00002712)
    __lit__00000000                          0x00038210   Data           4  entry2.o(.ARM.Collect$$$$00002712)
    .emb_text                                0x00038214   Section      226  nrf_atomic.o(.emb_text)
    .text                                    0x000382f8   Section       36  arm_startup_nrf52820.o(.text)
    .text                                    0x0003831c   Section        0  llshl.o(.text)
    .text                                    0x0003833a   Section        0  memcpya.o(.text)
    .text                                    0x0003835e   Section        0  memseta.o(.text)
    .text                                    0x00038382   Section        0  memcmp.o(.text)
    .text                                    0x0003839c   Section       36  init.o(.text)
    [Anonymous Symbol]                       0x000383c0   Section        0  uECC.c.o(.text.XYcZ_add)
    XYcZ_add                                 0x000383c1   Thumb Code   206  uECC.c.o(.text.XYcZ_add)
    [Anonymous Symbol]                       0x0003848e   Section        0  uECC.c.o(.text.apply_z)
    apply_z                                  0x0003848f   Thumb Code    62  uECC.c.o(.text.apply_z)
    [Anonymous Symbol]                       0x000384cc   Section        0  uECC.c.o(.text.bcopy)
    bcopy                                    0x000384cd   Thumb Code    20  uECC.c.o(.text.bcopy)
    [Anonymous Symbol]                       0x000384e0   Section        0  uECC.c.o(.text.bits2int)
    bits2int                                 0x000384e1   Thumb Code   142  uECC.c.o(.text.bits2int)
    [Anonymous Symbol]                       0x0003856e   Section        0  uECC.c.o(.text.double_jacobian_default)
    double_jacobian_default                  0x0003856f   Thumb Code   338  uECC.c.o(.text.double_jacobian_default)
    [Anonymous Symbol]                       0x000386c0   Section        0  uECC.c.o(.text.uECC_secp256r1)
    [Anonymous Symbol]                       0x000386c8   Section        0  uECC.c.o(.text.uECC_verify)
    [Anonymous Symbol]                       0x000389d0   Section        0  uECC.c.o(.text.uECC_vli_add)
    uECC_vli_add                             0x000389d1   Thumb Code    88  uECC.c.o(.text.uECC_vli_add)
    [Anonymous Symbol]                       0x00038a28   Section        0  uECC.c.o(.text.uECC_vli_clear)
    uECC_vli_clear                           0x00038a29   Thumb Code    22  uECC.c.o(.text.uECC_vli_clear)
    [Anonymous Symbol]                       0x00038a3e   Section        0  uECC.c.o(.text.uECC_vli_cmp_unsafe)
    uECC_vli_cmp_unsafe                      0x00038a3f   Thumb Code    42  uECC.c.o(.text.uECC_vli_cmp_unsafe)
    [Anonymous Symbol]                       0x00038a68   Section        0  uECC.c.o(.text.uECC_vli_isZero)
    uECC_vli_isZero                          0x00038a69   Thumb Code    30  uECC.c.o(.text.uECC_vli_isZero)
    [Anonymous Symbol]                       0x00038a86   Section        0  uECC.c.o(.text.uECC_vli_modAdd)
    uECC_vli_modAdd                          0x00038a87   Thumb Code    56  uECC.c.o(.text.uECC_vli_modAdd)
    [Anonymous Symbol]                       0x00038abe   Section        0  uECC.c.o(.text.uECC_vli_modInv)
    uECC_vli_modInv                          0x00038abf   Thumb Code   262  uECC.c.o(.text.uECC_vli_modInv)
    [Anonymous Symbol]                       0x00038bc4   Section        0  uECC.c.o(.text.uECC_vli_modMult)
    uECC_vli_modMult                         0x00038bc5   Thumb Code   316  uECC.c.o(.text.uECC_vli_modMult)
    [Anonymous Symbol]                       0x00038d00   Section        0  uECC.c.o(.text.uECC_vli_modMult_fast)
    uECC_vli_modMult_fast                    0x00038d01   Thumb Code    32  uECC.c.o(.text.uECC_vli_modMult_fast)
    [Anonymous Symbol]                       0x00038d20   Section        0  uECC.c.o(.text.uECC_vli_modSquare_fast)
    uECC_vli_modSquare_fast                  0x00038d21   Thumb Code     8  uECC.c.o(.text.uECC_vli_modSquare_fast)
    [Anonymous Symbol]                       0x00038d28   Section        0  uECC.c.o(.text.uECC_vli_modSub)
    uECC_vli_modSub                          0x00038d29   Thumb Code    40  uECC.c.o(.text.uECC_vli_modSub)
    [Anonymous Symbol]                       0x00038d50   Section        0  uECC.c.o(.text.uECC_vli_mult)
    uECC_vli_mult                            0x00038d51   Thumb Code   786  uECC.c.o(.text.uECC_vli_mult)
    [Anonymous Symbol]                       0x00039062   Section        0  uECC.c.o(.text.uECC_vli_numBits)
    uECC_vli_numBits                         0x00039063   Thumb Code    64  uECC.c.o(.text.uECC_vli_numBits)
    [Anonymous Symbol]                       0x000390a2   Section        0  uECC.c.o(.text.uECC_vli_rshift1)
    uECC_vli_rshift1                         0x000390a3   Thumb Code    26  uECC.c.o(.text.uECC_vli_rshift1)
    [Anonymous Symbol]                       0x000390bc   Section        0  uECC.c.o(.text.uECC_vli_set)
    uECC_vli_set                             0x000390bd   Thumb Code    24  uECC.c.o(.text.uECC_vli_set)
    [Anonymous Symbol]                       0x000390e0   Section        0  uECC.c.o(.text.uECC_vli_sub)
    uECC_vli_sub                             0x000390e1   Thumb Code    94  uECC.c.o(.text.uECC_vli_sub)
    [Anonymous Symbol]                       0x00039140   Section        0  uECC.c.o(.text.uECC_vli_testBit)
    uECC_vli_testBit                         0x00039141   Thumb Code    20  uECC.c.o(.text.uECC_vli_testBit)
    [Anonymous Symbol]                       0x00039154   Section        0  uECC.c.o(.text.vli_mmod_fast_secp256r1)
    vli_mmod_fast_secp256r1                  0x00039155   Thumb Code   432  uECC.c.o(.text.vli_mmod_fast_secp256r1)
    [Anonymous Symbol]                       0x00039304   Section        0  uECC.c.o(.text.vli_modInv_update)
    vli_modInv_update                        0x00039305   Thumb Code    56  uECC.c.o(.text.vli_modInv_update)
    [Anonymous Symbol]                       0x0003933c   Section        0  uECC.c.o(.text.x_side_default)
    x_side_default                           0x0003933d   Thumb Code    94  uECC.c.o(.text.x_side_default)
    i.RTC1_IRQHandler                        0x0003939c   Section        0  nrf_bootloader_dfu_timers.o(i.RTC1_IRQHandler)
    i.SystemInit                             0x00039410   Section        0  system_nrf52.o(i.SystemInit)
    i.UARTE0_UART0_IRQHandler                0x00039588   Section        0  nrfx_uarte.o(i.UARTE0_UART0_IRQHandler)
    i.WDT_IRQHandler                         0x00039598   Section        0  nrf_bootloader_wdt.o(i.WDT_IRQHandler)
    i.__scatterload_copy                     0x000395ac   Section       14  handlers.o(i.__scatterload_copy)
    i.__scatterload_null                     0x000395ba   Section        2  handlers.o(i.__scatterload_null)
    i.__scatterload_zeroinit                 0x000395bc   Section       14  handlers.o(i.__scatterload_zeroinit)
    i.addr_is_aligned32                      0x000395ca   Section        0  nrf_fstorage.o(i.addr_is_aligned32)
    addr_is_aligned32                        0x000395cb   Thumb Code    12  nrf_fstorage.o(i.addr_is_aligned32)
    i.addr_is_within_bounds                  0x000395d6   Section        0  nrf_fstorage.o(i.addr_is_within_bounds)
    addr_is_within_bounds                    0x000395d7   Thumb Code    24  nrf_fstorage.o(i.addr_is_within_bounds)
    i.app_activate                           0x000395f0   Section        0  nrf_bootloader_fw_activation.o(i.app_activate)
    app_activate                             0x000395f1   Thumb Code    66  nrf_bootloader_fw_activation.o(i.app_activate)
    i.app_error_handler_bare                 0x00039638   Section        0  main.o(i.app_error_handler_bare)
    i.app_sched_event_put                    0x0003963c   Section        0  app_scheduler.o(i.app_sched_event_put)
    i.app_sched_execute                      0x000396d8   Section        0  app_scheduler.o(i.app_sched_execute)
    i.app_sched_init                         0x00039718   Section        0  app_scheduler.o(i.app_sched_init)
    i.app_util_critical_region_enter         0x00039744   Section        0  app_util_platform.o(i.app_util_critical_region_enter)
    i.app_util_critical_region_exit          0x00039748   Section        0  app_util_platform.o(i.app_util_critical_region_exit)
    i.app_util_disable_irq                   0x0003974c   Section        0  app_util_platform.o(i.app_util_disable_irq)
    i.app_util_enable_irq                    0x0003975c   Section        0  app_util_platform.o(i.app_util_enable_irq)
    i.apply_config                           0x00039770   Section        0  nrfx_uarte.o(i.apply_config)
    apply_config                             0x00039771   Thumb Code   136  nrfx_uarte.o(i.apply_config)
    i.bl_activate                            0x000397f8   Section        0  nrf_bootloader_fw_activation.o(i.bl_activate)
    bl_activate                              0x000397f9   Thumb Code    66  nrf_bootloader_fw_activation.o(i.bl_activate)
    i.boot_validate                          0x00039844   Section        0  nrf_bootloader.o(i.boot_validate)
    boot_validate                            0x00039845   Thumb Code    16  nrf_bootloader.o(i.boot_validate)
    i.boot_validation_crc                    0x00039854   Section        0  nrf_dfu_settings.o(i.boot_validation_crc)
    boot_validation_crc                      0x00039855   Thumb Code    12  nrf_dfu_settings.o(i.boot_validation_crc)
    i.boot_validation_extract                0x00039860   Section        0  nrf_dfu_validation.o(i.boot_validation_extract)
    boot_validation_extract                  0x00039861   Thumb Code   146  nrf_dfu_validation.o(i.boot_validation_extract)
    i.bootloader_reset                       0x000398f8   Section        0  nrf_bootloader.o(i.bootloader_reset)
    bootloader_reset                         0x000398f9   Thumb Code    28  nrf_bootloader.o(i.bootloader_reset)
    i.bsp_board_init                         0x0003991c   Section        0  boards.o(i.bsp_board_init)
    i.bsp_board_led_off                      0x00039970   Section        0  boards.o(i.bsp_board_led_off)
    i.bsp_board_led_on                       0x00039980   Section        0  boards.o(i.bsp_board_led_on)
    i.bsp_board_leds_off                     0x00039990   Section        0  boards.o(i.bsp_board_leds_off)
    i.buf_read                               0x000399a2   Section        0  pb_decode.o(i.buf_read)
    buf_read                                 0x000399a3   Thumb Code    28  pb_decode.o(i.buf_read)
    i.cmd_response_offset_and_crc_set        0x000399c0   Section        0  nrf_dfu_req_handler.o(i.cmd_response_offset_and_crc_set)
    cmd_response_offset_and_crc_set          0x000399c1   Thumb Code    12  nrf_dfu_req_handler.o(i.cmd_response_offset_and_crc_set)
    i.crc32_compute                          0x000399d0   Section        0  crc32.o(i.crc32_compute)
    i.crc_ok                                 0x00039a0c   Section        0  nrf_dfu_settings.o(i.crc_ok)
    crc_ok                                   0x00039a0d   Thumb Code    30  nrf_dfu_settings.o(i.crc_ok)
    i.crypto_init                            0x00039a2c   Section        0  nrf_dfu_validation.o(i.crypto_init)
    crypto_init                              0x00039a2d   Thumb Code    46  nrf_dfu_validation.o(i.crypto_init)
    i.decode_callback_field                  0x00039a6c   Section        0  pb_decode.o(i.decode_callback_field)
    decode_callback_field                    0x00039a6d   Thumb Code   126  pb_decode.o(i.decode_callback_field)
    i.decode_field                           0x00039aea   Section        0  pb_decode.o(i.decode_field)
    decode_field                             0x00039aeb   Thumb Code    26  pb_decode.o(i.decode_field)
    i.decode_static_field                    0x00039b04   Section        0  pb_decode.o(i.decode_static_field)
    decode_static_field                      0x00039b05   Thumb Code   220  pb_decode.o(i.decode_static_field)
    i.dfu_enter_check                        0x00039be4   Section        0  nrf_bootloader.o(i.dfu_enter_check)
    dfu_enter_check                          0x00039be5   Thumb Code   140  nrf_bootloader.o(i.dfu_enter_check)
    i.dfu_fstorage_evt_handler               0x00039c84   Section        0  nrf_dfu_flash.o(i.dfu_fstorage_evt_handler)
    i.dfu_observer                           0x00039c90   Section        0  main.o(i.dfu_observer)
    dfu_observer                             0x00039c91   Thumb Code    64  main.o(i.dfu_observer)
    i.dfu_observer                           0x00039cd0   Section        0  nrf_bootloader.o(i.dfu_observer)
    dfu_observer                             0x00039cd1   Thumb Code    62  nrf_bootloader.o(i.dfu_observer)
    i.dfu_observer                           0x00039d18   Section        0  nrf_dfu.o(i.dfu_observer)
    dfu_observer                             0x00039d19   Thumb Code    36  nrf_dfu.o(i.dfu_observer)
    i.dfu_req_handler_rsp_clbk               0x00039d40   Section        0  nrf_dfu_serial.o(i.dfu_req_handler_rsp_clbk)
    i.do_reset                               0x00039d6c   Section        0  nrf_bootloader.o(i.do_reset)
    do_reset                                 0x00039d6d   Thumb Code    26  nrf_bootloader.o(i.do_reset)
    i.erase                                  0x00039d90   Section        0  nrf_fstorage_nvmc.o(i.erase)
    erase                                    0x00039d91   Thumb Code    68  nrf_fstorage_nvmc.o(i.erase)
    i.event_send                             0x00039dd8   Section        0  nrf_fstorage_nvmc.o(i.event_send)
    event_send                               0x00039dd9   Thumb Code    54  nrf_fstorage_nvmc.o(i.event_send)
    i.ext_err_code_handle                    0x00039e0e   Section        0  nrf_dfu_req_handler.o(i.ext_err_code_handle)
    ext_err_code_handle                      0x00039e0f   Thumb Code    14  nrf_dfu_req_handler.o(i.ext_err_code_handle)
    i.ext_error_get                          0x00039e1c   Section        0  nrf_dfu_handling_error.o(i.ext_error_get)
    i.ext_error_set                          0x00039e2c   Section        0  nrf_dfu_handling_error.o(i.ext_error_set)
    i.flash_write_callback                   0x00039e38   Section        0  nrf_bootloader.o(i.flash_write_callback)
    flash_write_callback                     0x00039e39   Thumb Code     8  nrf_bootloader.o(i.flash_write_callback)
    i.flash_write_callback                   0x00039e44   Section        0  nrf_bootloader_fw_activation.o(i.flash_write_callback)
    flash_write_callback                     0x00039e45   Thumb Code     8  nrf_bootloader_fw_activation.o(i.flash_write_callback)
    i.fw_hash_ok                             0x00039e50   Section        0  nrf_dfu_validation.o(i.fw_hash_ok)
    i.image_copy                             0x00039e58   Section        0  nrf_bootloader_fw_activation.o(i.image_copy)
    image_copy                               0x00039e59   Thumb Code   140  nrf_bootloader_fw_activation.o(i.image_copy)
    i.inactivity_timeout                     0x00039ee8   Section        0  nrf_bootloader.o(i.inactivity_timeout)
    inactivity_timeout                       0x00039ee9   Thumb Code     6  nrf_bootloader.o(i.inactivity_timeout)
    i.init                                   0x00039ef0   Section        0  nrf_fstorage_nvmc.o(i.init)
    init                                     0x00039ef1   Thumb Code     8  nrf_fstorage_nvmc.o(i.init)
    i.interrupts_enable                      0x00039efc   Section        0  nrfx_uarte.o(i.interrupts_enable)
    interrupts_enable                        0x00039efd   Thumb Code   132  nrfx_uarte.o(i.interrupts_enable)
    i.is_busy                                0x00039f84   Section        0  nrf_fstorage_nvmc.o(i.is_busy)
    is_busy                                  0x00039f85   Thumb Code    12  nrf_fstorage_nvmc.o(i.is_busy)
    i.is_major_softdevice_update             0x00039f94   Section        0  nrf_dfu_validation.o(i.is_major_softdevice_update)
    is_major_softdevice_update               0x00039f95   Thumb Code    88  nrf_dfu_validation.o(i.is_major_softdevice_update)
    i.iter_from_extension                    0x00039ff4   Section        0  pb_decode.o(i.iter_from_extension)
    iter_from_extension                      0x00039ff5   Thumb Code    46  pb_decode.o(i.iter_from_extension)
    i.led_test                               0x0003a024   Section        0  main.o(i.led_test)
    i.main                                   0x0003a040   Section        0  main.o(i.main)
    i.nrf_atomic_flag_clear                  0x0003a070   Section        0  nrf_atomic.o(i.nrf_atomic_flag_clear)
    i.nrf_atomic_flag_set_fetch              0x0003a076   Section        0  nrf_atomic.o(i.nrf_atomic_flag_set_fetch)
    i.nrf_atomic_u32_and                     0x0003a07c   Section        0  nrf_atomic.o(i.nrf_atomic_u32_and)
    i.nrf_atomic_u32_fetch_or                0x0003a088   Section        0  nrf_atomic.o(i.nrf_atomic_u32_fetch_or)
    i.nrf_balloc_alloc                       0x0003a092   Section        0  nrf_balloc.o(i.nrf_balloc_alloc)
    i.nrf_balloc_free                        0x0003a0d0   Section        0  nrf_balloc.o(i.nrf_balloc_free)
    i.nrf_balloc_init                        0x0003a0fa   Section        0  nrf_balloc.o(i.nrf_balloc_init)
    i.nrf_bootloader_app_start               0x0003a12a   Section        0  nrf_bootloader_app_start.o(i.nrf_bootloader_app_start)
    i.nrf_bootloader_app_start_final         0x0003a150   Section        0  nrf_bootloader_app_start_final.o(i.nrf_bootloader_app_start_final)
    i.nrf_bootloader_dfu_inactivity_timer_restart 0x0003a1b0   Section        0  nrf_bootloader_dfu_timers.o(i.nrf_bootloader_dfu_inactivity_timer_restart)
    i.nrf_bootloader_flash_protect           0x0003a1d8   Section        0  nrf_bootloader_app_start_final.o(i.nrf_bootloader_flash_protect)
    i.nrf_bootloader_fw_activate             0x0003a218   Section        0  nrf_bootloader_fw_activation.o(i.nrf_bootloader_fw_activate)
    i.nrf_bootloader_init                    0x0003a28c   Section        0  nrf_bootloader.o(i.nrf_bootloader_init)
    i.nrf_bootloader_mbr_addrs_populate      0x0003a36c   Section        0  nrf_bootloader_info.o(i.nrf_bootloader_mbr_addrs_populate)
    i.nrf_bootloader_wdt_feed                0x0003a39c   Section        0  nrf_bootloader_wdt.o(i.nrf_bootloader_wdt_feed)
    i.nrf_bootloader_wdt_feed_timer_start    0x0003a3b0   Section        0  nrf_bootloader_dfu_timers.o(i.nrf_bootloader_wdt_feed_timer_start)
    i.nrf_bootloader_wdt_init                0x0003a3c4   Section        0  nrf_bootloader_wdt.o(i.nrf_bootloader_wdt_init)
    i.nrf_crypto_backend_micro_ecc_curve_get 0x0003a40c   Section        0  micro_ecc_backend_ecc.o(i.nrf_crypto_backend_micro_ecc_curve_get)
    i.nrf_crypto_backend_micro_ecc_public_key_from_raw 0x0003a412   Section        0  micro_ecc_backend_ecc.o(i.nrf_crypto_backend_micro_ecc_public_key_from_raw)
    i.nrf_crypto_backend_micro_ecc_verify    0x0003a422   Section        0  micro_ecc_backend_ecdsa.o(i.nrf_crypto_backend_micro_ecc_verify)
    i.nrf_crypto_ecc_public_key_from_raw     0x0003a478   Section        0  nrf_crypto_ecc.o(i.nrf_crypto_ecc_public_key_from_raw)
    i.nrf_crypto_ecdsa_verify                0x0003a4ac   Section        0  nrf_crypto_ecdsa.o(i.nrf_crypto_ecdsa_verify)
    i.nrf_crypto_hash_calculate              0x0003a4f8   Section        0  nrf_crypto_hash.o(i.nrf_crypto_hash_calculate)
    i.nrf_crypto_hash_finalize               0x0003a52e   Section        0  nrf_crypto_hash.o(i.nrf_crypto_hash_finalize)
    i.nrf_crypto_hash_init                   0x0003a564   Section        0  nrf_crypto_hash.o(i.nrf_crypto_hash_init)
    i.nrf_crypto_hash_update                 0x0003a590   Section        0  nrf_crypto_hash.o(i.nrf_crypto_hash_update)
    i.nrf_crypto_init                        0x0003a5c0   Section        0  nrf_crypto_init.o(i.nrf_crypto_init)
    i.nrf_crypto_internal_double_swap_endian 0x0003a600   Section        0  nrf_crypto_shared.o(i.nrf_crypto_internal_double_swap_endian)
    i.nrf_crypto_internal_double_swap_endian_in_place 0x0003a61a   Section        0  nrf_crypto_shared.o(i.nrf_crypto_internal_double_swap_endian_in_place)
    i.nrf_crypto_internal_ecc_key_input_check 0x0003a630   Section        0  nrf_crypto_ecc.o(i.nrf_crypto_internal_ecc_key_input_check)
    i.nrf_crypto_internal_ecc_key_output_prepare 0x0003a648   Section        0  nrf_crypto_ecc.o(i.nrf_crypto_internal_ecc_key_output_prepare)
    i.nrf_crypto_internal_ecc_raw_input_check 0x0003a662   Section        0  nrf_crypto_ecc.o(i.nrf_crypto_internal_ecc_raw_input_check)
    i.nrf_crypto_internal_swap_endian        0x0003a678   Section        0  nrf_crypto_shared.o(i.nrf_crypto_internal_swap_endian)
    i.nrf_crypto_internal_swap_endian_in_place 0x0003a68e   Section        0  nrf_crypto_shared.o(i.nrf_crypto_internal_swap_endian_in_place)
    i.nrf_dfu_app_start_address              0x0003a6a6   Section        0  nrf_dfu_utils.o(i.nrf_dfu_app_start_address)
    i.nrf_dfu_bank0_start_addr               0x0003a6ac   Section        0  nrf_dfu_utils.o(i.nrf_dfu_bank0_start_addr)
    i.nrf_dfu_bank1_start_addr               0x0003a6d4   Section        0  nrf_dfu_utils.o(i.nrf_dfu_bank1_start_addr)
    i.nrf_dfu_bank_invalidate                0x0003a6f4   Section        0  nrf_dfu_utils.o(i.nrf_dfu_bank_invalidate)
    i.nrf_dfu_cache_prepare                  0x0003a708   Section        0  nrf_dfu_utils.o(i.nrf_dfu_cache_prepare)
    i.nrf_dfu_command_req                    0x0003a7ac   Section        0  nrf_dfu_req_handler.o(i.nrf_dfu_command_req)
    nrf_dfu_command_req                      0x0003a7ad   Thumb Code   142  nrf_dfu_req_handler.o(i.nrf_dfu_command_req)
    i.nrf_dfu_data_req                       0x0003a840   Section        0  nrf_dfu_req_handler.o(i.nrf_dfu_data_req)
    nrf_dfu_data_req                         0x0003a841   Thumb Code   108  nrf_dfu_req_handler.o(i.nrf_dfu_data_req)
    i.nrf_dfu_flash_erase                    0x0003a8b4   Section        0  nrf_dfu_flash.o(i.nrf_dfu_flash_erase)
    i.nrf_dfu_flash_init                     0x0003a8c4   Section        0  nrf_dfu_flash.o(i.nrf_dfu_flash_init)
    i.nrf_dfu_flash_store                    0x0003a8d8   Section        0  nrf_dfu_flash.o(i.nrf_dfu_flash_store)
    i.nrf_dfu_init                           0x0003a8f0   Section        0  nrf_dfu.o(i.nrf_dfu_init)
    i.nrf_dfu_init_user                      0x0003a91c   Section        0  nrf_bootloader.o(i.nrf_dfu_init_user)
    i.nrf_dfu_mbr_copy_bl                    0x0003a920   Section        0  nrf_dfu_mbr.o(i.nrf_dfu_mbr_copy_bl)
    i.nrf_dfu_mbr_irq_forward_address_set    0x0003a938   Section        0  nrf_dfu_mbr.o(i.nrf_dfu_mbr_irq_forward_address_set)
    i.nrf_dfu_req_handler_init               0x0003a964   Section        0  nrf_dfu_req_handler.o(i.nrf_dfu_req_handler_init)
    i.nrf_dfu_req_handler_on_req             0x0003a9a8   Section        0  nrf_dfu_req_handler.o(i.nrf_dfu_req_handler_on_req)
    i.nrf_dfu_req_handler_req                0x0003a9bc   Section        0  nrf_dfu_req_handler.o(i.nrf_dfu_req_handler_req)
    nrf_dfu_req_handler_req                  0x0003a9bd   Thumb Code     4  nrf_dfu_req_handler.o(i.nrf_dfu_req_handler_req)
    i.nrf_dfu_req_handler_req_process        0x0003a9c0   Section        0  nrf_dfu_req_handler.o(i.nrf_dfu_req_handler_req_process)
    nrf_dfu_req_handler_req_process          0x0003a9c1   Thumb Code   206  nrf_dfu_req_handler.o(i.nrf_dfu_req_handler_req_process)
    i.nrf_dfu_serial_on_packet_received      0x0003aa98   Section        0  nrf_dfu_serial.o(i.nrf_dfu_serial_on_packet_received)
    i.nrf_dfu_settings_additional_erase      0x0003ab2c   Section        0  nrf_dfu_settings.o(i.nrf_dfu_settings_additional_erase)
    i.nrf_dfu_settings_backup                0x0003ab30   Section        0  nrf_dfu_settings.o(i.nrf_dfu_settings_backup)
    i.nrf_dfu_settings_init                  0x0003ab3c   Section        0  nrf_dfu_settings.o(i.nrf_dfu_settings_init)
    i.nrf_dfu_settings_progress_reset        0x0003ab58   Section        0  nrf_dfu_settings.o(i.nrf_dfu_settings_progress_reset)
    i.nrf_dfu_settings_reinit                0x0003ab80   Section        0  nrf_dfu_settings.o(i.nrf_dfu_settings_reinit)
    i.nrf_dfu_settings_write                 0x0003ac54   Section        0  nrf_dfu_settings.o(i.nrf_dfu_settings_write)
    i.nrf_dfu_settings_write_and_backup      0x0003ac88   Section        0  nrf_dfu_settings.o(i.nrf_dfu_settings_write_and_backup)
    i.nrf_dfu_softdevice_invalidate          0x0003aca8   Section        0  nrf_dfu_utils.o(i.nrf_dfu_softdevice_invalidate)
    i.nrf_dfu_softdevice_start_address       0x0003acec   Section        0  nrf_dfu_utils.o(i.nrf_dfu_softdevice_start_address)
    i.nrf_dfu_transports_close               0x0003acf4   Section        0  nrf_dfu_transport.o(i.nrf_dfu_transports_close)
    i.nrf_dfu_transports_init                0x0003ad28   Section        0  nrf_dfu_transport.o(i.nrf_dfu_transports_init)
    i.nrf_dfu_validation_activation_prepare  0x0003ad5c   Section        0  nrf_dfu_validation.o(i.nrf_dfu_validation_activation_prepare)
    i.nrf_dfu_validation_boot_validate       0x0003ad62   Section        0  nrf_dfu_validation.o(i.nrf_dfu_validation_boot_validate)
    i.nrf_dfu_validation_hash_ok             0x0003adb4   Section        0  nrf_dfu_validation.o(i.nrf_dfu_validation_hash_ok)
    nrf_dfu_validation_hash_ok               0x0003adb5   Thumb Code    90  nrf_dfu_validation.o(i.nrf_dfu_validation_hash_ok)
    i.nrf_dfu_validation_init                0x0003ae18   Section        0  nrf_dfu_validation.o(i.nrf_dfu_validation_init)
    i.nrf_dfu_validation_init_cmd_append     0x0003ae3c   Section        0  nrf_dfu_validation.o(i.nrf_dfu_validation_init_cmd_append)
    i.nrf_dfu_validation_init_cmd_create     0x0003ae84   Section        0  nrf_dfu_validation.o(i.nrf_dfu_validation_init_cmd_create)
    i.nrf_dfu_validation_init_cmd_execute    0x0003aeb8   Section        0  nrf_dfu_validation.o(i.nrf_dfu_validation_init_cmd_execute)
    i.nrf_dfu_validation_init_cmd_present    0x0003af44   Section        0  nrf_dfu_validation.o(i.nrf_dfu_validation_init_cmd_present)
    i.nrf_dfu_validation_prevalidate         0x0003af50   Section        0  nrf_dfu_validation.o(i.nrf_dfu_validation_prevalidate)
    i.nrf_dfu_validation_signature_check     0x0003af98   Section        0  nrf_dfu_validation.o(i.nrf_dfu_validation_signature_check)
    nrf_dfu_validation_signature_check       0x0003af99   Thumb Code   140  nrf_dfu_validation.o(i.nrf_dfu_validation_signature_check)
    i.nrf_dfu_ver_validation_check           0x0003b02c   Section        0  nrf_dfu_ver_validation.o(i.nrf_dfu_ver_validation_check)
    i.nrf_drv_uart_init                      0x0003b0ac   Section        0  nrf_drv_uart.o(i.nrf_drv_uart_init)
    i.nrf_drv_uart_rx                        0x0003b0ec   Section        0  nrf_dfu_serial_uart.o(i.nrf_drv_uart_rx)
    nrf_drv_uart_rx                          0x0003b0ed   Thumb Code     6  nrf_dfu_serial_uart.o(i.nrf_drv_uart_rx)
    i.nrf_fstorage_erase                     0x0003b0f2   Section        0  nrf_fstorage.o(i.nrf_fstorage_erase)
    i.nrf_fstorage_init                      0x0003b11e   Section        0  nrf_fstorage.o(i.nrf_fstorage_init)
    i.nrf_fstorage_is_busy                   0x0003b128   Section        0  nrf_fstorage.o(i.nrf_fstorage_is_busy)
    i.nrf_fstorage_write                     0x0003b178   Section        0  nrf_fstorage.o(i.nrf_fstorage_write)
    i.nrf_gpio_cfg                           0x0003b1b6   Section        0  boards.o(i.nrf_gpio_cfg)
    nrf_gpio_cfg                             0x0003b1b7   Thumb Code    36  boards.o(i.nrf_gpio_cfg)
    i.nrf_gpio_cfg                           0x0003b1da   Section        0  nrfx_uarte.o(i.nrf_gpio_cfg)
    nrf_gpio_cfg                             0x0003b1db   Thumb Code    36  nrfx_uarte.o(i.nrf_gpio_cfg)
    i.nrf_gpio_cfg_default                   0x0003b1fe   Section        0  nrfx_uarte.o(i.nrf_gpio_cfg_default)
    nrf_gpio_cfg_default                     0x0003b1ff   Thumb Code    18  nrfx_uarte.o(i.nrf_gpio_cfg_default)
    i.nrf_gpio_cfg_input                     0x0003b210   Section        0  nrfx_uarte.o(i.nrf_gpio_cfg_input)
    nrf_gpio_cfg_input                       0x0003b211   Thumb Code    18  nrfx_uarte.o(i.nrf_gpio_cfg_input)
    i.nrf_gpio_cfg_output                    0x0003b222   Section        0  nrfx_uarte.o(i.nrf_gpio_cfg_output)
    nrf_gpio_cfg_output                      0x0003b223   Thumb Code    20  nrfx_uarte.o(i.nrf_gpio_cfg_output)
    i.nrf_gpio_pin_write                     0x0003b236   Section        0  boards.o(i.nrf_gpio_pin_write)
    nrf_gpio_pin_write                       0x0003b237   Thumb Code    22  boards.o(i.nrf_gpio_pin_write)
    i.nrf_nvmc_page_erase                    0x0003b24c   Section        0  nrf_nvmc.o(i.nrf_nvmc_page_erase)
    i.nrf_nvmc_write_word                    0x0003b27c   Section        0  nrf_nvmc.o(i.nrf_nvmc_write_word)
    i.nrf_nvmc_write_words                   0x0003b2ac   Section        0  nrf_nvmc.o(i.nrf_nvmc_write_words)
    i.nrf_rtc_event_clear                    0x0003b2f0   Section        0  nrf_bootloader_dfu_timers.o(i.nrf_rtc_event_clear)
    nrf_rtc_event_clear                      0x0003b2f1   Thumb Code    12  nrf_bootloader_dfu_timers.o(i.nrf_rtc_event_clear)
    i.nrf_sw_backend_hash_sha256_finalize    0x0003b2fc   Section        0  nrf_sw_backend_hash.o(i.nrf_sw_backend_hash_sha256_finalize)
    nrf_sw_backend_hash_sha256_finalize      0x0003b2fd   Thumb Code    36  nrf_sw_backend_hash.o(i.nrf_sw_backend_hash_sha256_finalize)
    i.nrf_sw_backend_hash_sha256_init        0x0003b320   Section        0  nrf_sw_backend_hash.o(i.nrf_sw_backend_hash_sha256_init)
    nrf_sw_backend_hash_sha256_init          0x0003b321   Thumb Code     6  nrf_sw_backend_hash.o(i.nrf_sw_backend_hash_sha256_init)
    i.nrf_sw_backend_hash_sha256_update      0x0003b326   Section        0  nrf_sw_backend_hash.o(i.nrf_sw_backend_hash_sha256_update)
    nrf_sw_backend_hash_sha256_update        0x0003b327   Thumb Code     6  nrf_sw_backend_hash.o(i.nrf_sw_backend_hash_sha256_update)
    i.nrf_uarte_event_check                  0x0003b32c   Section        0  nrfx_uarte.o(i.nrf_uarte_event_check)
    nrf_uarte_event_check                    0x0003b32d   Thumb Code    10  nrfx_uarte.o(i.nrf_uarte_event_check)
    i.nrf_uarte_event_clear                  0x0003b336   Section        0  nrfx_uarte.o(i.nrf_uarte_event_clear)
    nrf_uarte_event_clear                    0x0003b337   Thumb Code    12  nrfx_uarte.o(i.nrf_uarte_event_clear)
    i.nrf_wdt_started                        0x0003b344   Section        0  nrf_bootloader_wdt.o(i.nrf_wdt_started)
    nrf_wdt_started                          0x0003b345   Thumb Code    12  nrf_bootloader_wdt.o(i.nrf_wdt_started)
    i.nrfx_is_in_ram                         0x0003b354   Section        0  nrfx_uarte.o(i.nrfx_is_in_ram)
    nrfx_is_in_ram                           0x0003b355   Thumb Code    16  nrfx_uarte.o(i.nrfx_is_in_ram)
    i.nrfx_prs_acquire                       0x0003b364   Section        0  nrfx_prs.o(i.nrfx_prs_acquire)
    i.nrfx_prs_release                       0x0003b368   Section        0  nrfx_prs.o(i.nrfx_prs_release)
    i.nrfx_uarte_init                        0x0003b36c   Section        0  nrfx_uarte.o(i.nrfx_uarte_init)
    i.nrfx_uarte_rx                          0x0003b3d8   Section        0  nrfx_uarte.o(i.nrfx_uarte_rx)
    i.nrfx_uarte_tx                          0x0003b4dc   Section        0  nrfx_uarte.o(i.nrfx_uarte_tx)
    i.nrfx_uarte_tx_in_progress              0x0003b588   Section        0  nrfx_uarte.o(i.nrfx_uarte_tx_in_progress)
    i.nrfx_uarte_uninit                      0x0003b5a4   Section        0  nrfx_uarte.o(i.nrfx_uarte_uninit)
    i.nvmc_config                            0x0003b6ac   Section        0  system_nrf52.o(i.nvmc_config)
    i.on_data_obj_create_request             0x0003b6c4   Section        0  nrf_dfu_req_handler.o(i.on_data_obj_create_request)
    on_data_obj_create_request               0x0003b6c5   Thumb Code   108  nrf_dfu_req_handler.o(i.on_data_obj_create_request)
    i.on_data_obj_execute_request_sched      0x0003b738   Section        0  nrf_dfu_req_handler.o(i.on_data_obj_execute_request_sched)
    on_data_obj_execute_request_sched        0x0003b739   Thumb Code   100  nrf_dfu_req_handler.o(i.on_data_obj_execute_request_sched)
    i.on_data_obj_write_request              0x0003b7b0   Section        0  nrf_dfu_req_handler.o(i.on_data_obj_write_request)
    on_data_obj_write_request                0x0003b7b1   Thumb Code   118  nrf_dfu_req_handler.o(i.on_data_obj_write_request)
    i.on_dfu_complete                        0x0003b830   Section        0  nrf_dfu_req_handler.o(i.on_dfu_complete)
    on_dfu_complete                          0x0003b831   Thumb Code     8  nrf_dfu_req_handler.o(i.on_dfu_complete)
    i.on_error                               0x0003b83c   Section        0  main.o(i.on_error)
    on_error                                 0x0003b83d   Thumb Code    26  main.o(i.on_error)
    i.on_fw_version_request                  0x0003b860   Section        0  nrf_dfu_req_handler.o(i.on_fw_version_request)
    on_fw_version_request                    0x0003b861   Thumb Code   138  nrf_dfu_req_handler.o(i.on_fw_version_request)
    i.payload_free                           0x0003b8f8   Section        0  nrf_dfu_serial_uart.o(i.payload_free)
    payload_free                             0x0003b8f9   Thumb Code     8  nrf_dfu_serial_uart.o(i.payload_free)
    i.pb_dec_bytes                           0x0003b904   Section        0  pb_decode.o(i.pb_dec_bytes)
    pb_dec_bytes                             0x0003b905   Thumb Code    64  pb_decode.o(i.pb_dec_bytes)
    i.pb_dec_fixed32                         0x0003b944   Section        0  pb_decode.o(i.pb_dec_fixed32)
    pb_dec_fixed32                           0x0003b945   Thumb Code     6  pb_decode.o(i.pb_dec_fixed32)
    i.pb_dec_fixed64                         0x0003b94a   Section        0  pb_decode.o(i.pb_dec_fixed64)
    pb_dec_fixed64                           0x0003b94b   Thumb Code     6  pb_decode.o(i.pb_dec_fixed64)
    i.pb_dec_string                          0x0003b950   Section        0  pb_decode.o(i.pb_dec_string)
    pb_dec_string                            0x0003b951   Thumb Code    62  pb_decode.o(i.pb_dec_string)
    i.pb_dec_submessage                      0x0003b98e   Section        0  pb_decode.o(i.pb_dec_submessage)
    pb_dec_submessage                        0x0003b98f   Thumb Code    64  pb_decode.o(i.pb_dec_submessage)
    i.pb_dec_svarint                         0x0003b9ce   Section        0  pb_decode.o(i.pb_dec_svarint)
    pb_dec_svarint                           0x0003b9cf   Thumb Code    88  pb_decode.o(i.pb_dec_svarint)
    i.pb_dec_uvarint                         0x0003ba26   Section        0  pb_decode.o(i.pb_dec_uvarint)
    pb_dec_uvarint                           0x0003ba27   Thumb Code    88  pb_decode.o(i.pb_dec_uvarint)
    i.pb_dec_varint                          0x0003ba7e   Section        0  pb_decode.o(i.pb_dec_varint)
    pb_dec_varint                            0x0003ba7f   Thumb Code    90  pb_decode.o(i.pb_dec_varint)
    i.pb_decode                              0x0003bad8   Section        0  pb_decode.o(i.pb_decode)
    i.pb_decode_fixed32                      0x0003baf6   Section        0  pb_decode.o(i.pb_decode_fixed32)
    i.pb_decode_fixed64                      0x0003bb16   Section        0  pb_decode.o(i.pb_decode_fixed64)
    i.pb_decode_noinit                       0x0003bb74   Section        0  pb_decode.o(i.pb_decode_noinit)
    i.pb_decode_svarint                      0x0003bcfa   Section        0  pb_decode.o(i.pb_decode_svarint)
    i.pb_decode_tag                          0x0003bd34   Section        0  pb_decode.o(i.pb_decode_tag)
    i.pb_decode_varint                       0x0003bd70   Section        0  pb_decode.o(i.pb_decode_varint)
    i.pb_decode_varint32                     0x0003bdba   Section        0  pb_decode.o(i.pb_decode_varint32)
    pb_decode_varint32                       0x0003bdbb   Thumb Code    76  pb_decode.o(i.pb_decode_varint32)
    i.pb_decoding_callback                   0x0003be08   Section        0  nrf_dfu_validation.o(i.pb_decoding_callback)
    pb_decoding_callback                     0x0003be09   Thumb Code    52  nrf_dfu_validation.o(i.pb_decoding_callback)
    i.pb_field_iter_begin                    0x0003be44   Section        0  pb_common.o(i.pb_field_iter_begin)
    i.pb_field_iter_find                     0x0003be66   Section        0  pb_common.o(i.pb_field_iter_find)
    i.pb_field_iter_next                     0x0003be94   Section        0  pb_common.o(i.pb_field_iter_next)
    i.pb_field_set_to_default                0x0003bf12   Section        0  pb_decode.o(i.pb_field_set_to_default)
    pb_field_set_to_default                  0x0003bf13   Thumb Code   164  pb_decode.o(i.pb_field_set_to_default)
    i.pb_istream_from_buffer                 0x0003bfb8   Section        0  pb_decode.o(i.pb_istream_from_buffer)
    i.pb_make_string_substream               0x0003bfcc   Section        0  pb_decode.o(i.pb_make_string_substream)
    i.pb_message_set_to_defaults             0x0003c002   Section        0  pb_decode.o(i.pb_message_set_to_defaults)
    pb_message_set_to_defaults               0x0003c003   Thumb Code    38  pb_decode.o(i.pb_message_set_to_defaults)
    i.pb_read                                0x0003c028   Section        0  pb_decode.o(i.pb_read)
    i.pb_readbyte                            0x0003c080   Section        0  pb_decode.o(i.pb_readbyte)
    pb_readbyte                              0x0003c081   Thumb Code    32  pb_decode.o(i.pb_readbyte)
    i.pb_skip_field                          0x0003c0a0   Section        0  pb_decode.o(i.pb_skip_field)
    i.postvalidate                           0x0003c0fc   Section        0  nrf_dfu_validation.o(i.postvalidate)
    i.postvalidate_sd_bl                     0x0003c1ec   Section        0  nrf_dfu_validation.o(i.postvalidate_sd_bl)
    postvalidate_sd_bl                       0x0003c1ed   Thumb Code   266  nrf_dfu_validation.o(i.postvalidate_sd_bl)
    i.read                                   0x0003c304   Section        0  nrf_fstorage_nvmc.o(i.read)
    read                                     0x0003c305   Thumb Code    14  nrf_fstorage_nvmc.o(i.read)
    i.read_raw_value                         0x0003c312   Section        0  pb_decode.o(i.read_raw_value)
    read_raw_value                           0x0003c313   Thumb Code    98  pb_decode.o(i.read_raw_value)
    i.response_send                          0x0003c374   Section        0  nrf_dfu_serial.o(i.response_send)
    response_send                            0x0003c375   Thumb Code   238  nrf_dfu_serial.o(i.response_send)
    i.rmap                                   0x0003c462   Section        0  nrf_fstorage_nvmc.o(i.rmap)
    rmap                                     0x0003c463   Thumb Code     4  nrf_fstorage_nvmc.o(i.rmap)
    i.rsp_send                               0x0003c468   Section        0  nrf_dfu_serial_uart.o(i.rsp_send)
    rsp_send                                 0x0003c469   Thumb Code    28  nrf_dfu_serial_uart.o(i.rsp_send)
    i.rx_done_event                          0x0003c48c   Section        0  nrfx_uarte.o(i.rx_done_event)
    rx_done_event                            0x0003c48d   Thumb Code    22  nrfx_uarte.o(i.rx_done_event)
    i.sd_activate                            0x0003c4a4   Section        0  nrf_bootloader_fw_activation.o(i.sd_activate)
    sd_activate                              0x0003c4a5   Thumb Code    74  nrf_bootloader_fw_activation.o(i.sd_activate)
    i.sd_req_check                           0x0003c4f8   Section        0  nrf_dfu_ver_validation.o(i.sd_req_check)
    sd_req_check                             0x0003c4f9   Thumb Code    64  nrf_dfu_ver_validation.o(i.sd_req_check)
    i.sd_req_ok                              0x0003c53c   Section        0  nrf_dfu_ver_validation.o(i.sd_req_ok)
    sd_req_ok                                0x0003c53d   Thumb Code    88  nrf_dfu_ver_validation.o(i.sd_req_ok)
    i.settings_backup                        0x0003c598   Section        0  nrf_dfu_settings.o(i.settings_backup)
    i.settings_crc_get                       0x0003c5ac   Section        0  nrf_dfu_settings.o(i.settings_crc_get)
    settings_crc_get                         0x0003c5ad   Thumb Code    10  nrf_dfu_settings.o(i.settings_crc_get)
    i.settings_write                         0x0003c5b6   Section        0  nrf_dfu_settings.o(i.settings_write)
    settings_write                           0x0003c5b7   Thumb Code    80  nrf_dfu_settings.o(i.settings_write)
    i.sha256_final                           0x0003c606   Section        0  sha256.o(i.sha256_final)
    i.sha256_init                            0x0003c718   Section        0  sha256.o(i.sha256_init)
    i.sha256_transform                       0x0003c76c   Section        0  sha256.o(i.sha256_transform)
    i.sha256_update                          0x0003c898   Section        0  sha256.o(i.sha256_update)
    i.slip_decode_add_byte                   0x0003c8ec   Section        0  slip.o(i.slip_decode_add_byte)
    i.slip_encode                            0x0003c95a   Section        0  slip.o(i.slip_encode)
    i.stored_init_cmd_decode                 0x0003c9b0   Section        0  nrf_dfu_validation.o(i.stored_init_cmd_decode)
    stored_init_cmd_decode                   0x0003c9b1   Thumb Code   172  nrf_dfu_validation.o(i.stored_init_cmd_decode)
    i.timer_activate                         0x0003ca78   Section        0  nrf_bootloader_dfu_timers.o(i.timer_activate)
    timer_activate                           0x0003ca79   Thumb Code    86  nrf_bootloader_dfu_timers.o(i.timer_activate)
    i.timer_init                             0x0003cad8   Section        0  nrf_bootloader_dfu_timers.o(i.timer_init)
    timer_init                               0x0003cad9   Thumb Code    98  nrf_bootloader_dfu_timers.o(i.timer_init)
    i.timer_start                            0x0003cb50   Section        0  nrf_bootloader_dfu_timers.o(i.timer_start)
    timer_start                              0x0003cb51   Thumb Code    26  nrf_bootloader_dfu_timers.o(i.timer_start)
    i.timer_stop                             0x0003cb6c   Section        0  nrf_bootloader_dfu_timers.o(i.timer_stop)
    timer_stop                               0x0003cb6d   Thumb Code    16  nrf_bootloader_dfu_timers.o(i.timer_stop)
    i.tx_done_event                          0x0003cb80   Section        0  nrfx_uarte.o(i.tx_done_event)
    tx_done_event                            0x0003cb81   Thumb Code    26  nrfx_uarte.o(i.tx_done_event)
    i.uart_dfu_transport_close               0x0003cb9c   Section        0  nrf_dfu_serial_uart.o(i.uart_dfu_transport_close)
    uart_dfu_transport_close                 0x0003cb9d   Thumb Code    30  nrf_dfu_serial_uart.o(i.uart_dfu_transport_close)
    i.uart_dfu_transport_init                0x0003cbc4   Section        0  nrf_dfu_serial_uart.o(i.uart_dfu_transport_init)
    uart_dfu_transport_init                  0x0003cbc5   Thumb Code   152  nrf_dfu_serial_uart.o(i.uart_dfu_transport_init)
    i.uart_event_handler                     0x0003cc7c   Section        0  nrf_dfu_serial_uart.o(i.uart_event_handler)
    uart_event_handler                       0x0003cc7d   Thumb Code    92  nrf_dfu_serial_uart.o(i.uart_event_handler)
    i.uarte_evt_handler                      0x0003cce4   Section        0  nrf_drv_uart.o(i.uarte_evt_handler)
    uarte_evt_handler                        0x0003cce5   Thumb Code    42  nrf_drv_uart.o(i.uarte_evt_handler)
    i.uarte_irq_handler                      0x0003cd14   Section        0  nrfx_uarte.o(i.uarte_irq_handler)
    uarte_irq_handler                        0x0003cd15   Thumb Code   274  nrfx_uarte.o(i.uarte_irq_handler)
    i.uint32_encode                          0x0003ce26   Section        0  nrf_dfu_serial.o(i.uint32_encode)
    uint32_encode                            0x0003ce27   Thumb Code    18  nrf_dfu_serial.o(i.uint32_encode)
    i.uninit                                 0x0003ce38   Section        0  nrf_fstorage_nvmc.o(i.uninit)
    uninit                                   0x0003ce39   Thumb Code    12  nrf_fstorage_nvmc.o(i.uninit)
    i.update_data_size_get                   0x0003ce48   Section        0  nrf_dfu_validation.o(i.update_data_size_get)
    update_data_size_get                     0x0003ce49   Thumb Code    84  nrf_dfu_validation.o(i.update_data_size_get)
    i.update_requires_softdevice             0x0003cea0   Section        0  nrf_dfu_validation.o(i.update_requires_softdevice)
    update_requires_softdevice               0x0003cea1   Thumb Code    16  nrf_dfu_validation.o(i.update_requires_softdevice)
    i.verify_context                         0x0003ceb0   Section        0  nrf_crypto_hash.o(i.verify_context)
    verify_context                           0x0003ceb1   Thumb Code    26  nrf_crypto_hash.o(i.verify_context)
    i.wdt_feed                               0x0003ced0   Section        0  nrf_bootloader_wdt.o(i.wdt_feed)
    wdt_feed                                 0x0003ced1   Thumb Code    48  nrf_bootloader_wdt.o(i.wdt_feed)
    i.wdt_feed_timer_handler                 0x0003cf0c   Section        0  nrf_bootloader_wdt.o(i.wdt_feed_timer_handler)
    wdt_feed_timer_handler                   0x0003cf0d   Thumb Code     4  nrf_bootloader_wdt.o(i.wdt_feed_timer_handler)
    i.wmap                                   0x0003cf10   Section        0  nrf_fstorage_nvmc.o(i.wmap)
    wmap                                     0x0003cf11   Thumb Code     4  nrf_fstorage_nvmc.o(i.wmap)
    i.write                                  0x0003cf14   Section        0  nrf_fstorage_nvmc.o(i.write)
    write                                    0x0003cf15   Thumb Code    64  nrf_fstorage_nvmc.o(i.write)
    .constdata                               0x0003cf58   Section       64  dfu_public_key.o(.constdata)
    .constdata                               0x0003cf98   Section        8  boards.o(.constdata)
    m_board_led_list                         0x0003cf98   Data           4  boards.o(.constdata)
    m_board_btn_list                         0x0003cf9c   Data           4  boards.o(.constdata)
    .constdata                               0x0003cfa0   Section        6  nrf_bootloader_dfu_timers.o(.constdata)
    delay_machine_code                       0x0003cfa0   Data           6  nrf_bootloader_dfu_timers.o(.constdata)
    .constdata                               0x0003cfa8   Section       24  nrf_sw_backend_hash.o(.constdata)
    .constdata                               0x0003cfc0   Section       12  micro_ecc_backend_ecc.o(.constdata)
    .constdata                               0x0003cfcc   Section        1  dfu-cc.pb.o(.constdata)
    .constdata                               0x0003cfd0   Section       48  dfu-cc.pb.o(.constdata)
    .constdata                               0x0003d000   Section       48  dfu-cc.pb.o(.constdata)
    .constdata                               0x0003d030   Section      176  dfu-cc.pb.o(.constdata)
    .constdata                               0x0003d0e0   Section       48  dfu-cc.pb.o(.constdata)
    .constdata                               0x0003d110   Section       64  dfu-cc.pb.o(.constdata)
    .constdata                               0x0003d150   Section       48  dfu-cc.pb.o(.constdata)
    .constdata                               0x0003d180   Section       32  nrf_dfu_mbr.o(.constdata)
    .constdata                               0x0003d1a0   Section       48  nrf_dfu_req_handler.o(.constdata)
    .constdata                               0x0003d1d0   Section       32  nrf_dfu_serial_uart.o(.constdata)
    .constdata                               0x0003d1f0   Section        4  nrf_dfu_utils.o(.constdata)
    all_zero                                 0x0003d1f0   Data           4  nrf_dfu_utils.o(.constdata)
    .constdata                               0x0003d1f4   Section        4  nrfx_uarte.o(.constdata)
    irq_handlers                             0x0003d1f4   Data           4  nrfx_uarte.o(.constdata)
    .constdata                               0x0003d1f8   Section       12  nrf_fstorage_nvmc.o(.constdata)
    m_flash_info                             0x0003d1f8   Data          12  nrf_fstorage_nvmc.o(.constdata)
    .constdata                               0x0003d204   Section       32  nrf_fstorage_nvmc.o(.constdata)
    .constdata                               0x0003d224   Section      256  sha256.o(.constdata)
    k                                        0x0003d224   Data         256  sha256.o(.constdata)
    .constdata                               0x0003d324   Section       24  nrf_dfu_serial.o(.constdata)
    .constdata                               0x0003d33c   Section       36  pb_decode.o(.constdata)
    PB_DECODERS                              0x0003d33c   Data          36  pb_decode.o(.constdata)
    [Anonymous Symbol]                       0x0003d360   Section        0  uECC.c.o(.rodata.curve_secp256r1)
    curve_secp256r1                          0x0003d360   Data         176  uECC.c.o(.rodata.curve_secp256r1)
    dfu_trans                                0x0003d430   Section        8  nrf_dfu_serial_uart.o(dfu_trans)
    __tagsym$$used                           0x0003d430   Number         0  nrf_dfu_serial_uart.o(dfu_trans)
    nrf_balloc                               0x0003d438   Section       20  nrf_dfu_serial_uart.o(nrf_balloc)
    __tagsym$$used                           0x0003d438   Number         0  nrf_dfu_serial_uart.o(nrf_balloc)
    .ARM.__AT_0x0003E000                     0x0003e000   Section     4096  nrf_dfu_settings.o(.ARM.__AT_0x0003E000)
    __tagsym$$used                           0x0003e000   Number         0  nrf_dfu_settings.o(.ARM.__AT_0x0003E000)
    .ARM.__AT_0x0003F000                     0x0003f000   Section     4096  nrf_dfu_settings.o(.ARM.__AT_0x0003F000)
    __tagsym$$used                           0x0003f000   Number         0  nrf_dfu_settings.o(.ARM.__AT_0x0003F000)
    .ARM.__AT_0x10001014                     0x10001014   Section        4  nrf_bootloader_info.o(.ARM.__AT_0x10001014)
    .ARM.__AT_0x10001018                     0x10001018   Section        4  nrf_dfu_settings.o(.ARM.__AT_0x10001018)
    .data                                    0x20000008   Section        8  nrf_bootloader.o(.data)
    m_flash_write_done                       0x20000008   Data           1  nrf_bootloader.o(.data)
    m_user_observer                          0x2000000c   Data           4  nrf_bootloader.o(.data)
    .data                                    0x20000010   Section        4  nrf_bootloader_app_start_final.o(.data)
    acl_instance                             0x20000010   Data           4  nrf_bootloader_app_start_final.o(.data)
    .data                                    0x20000014   Section       48  nrf_bootloader_dfu_timers.o(.data)
    m_timer_initialized                      0x20000014   Data           1  nrf_bootloader_dfu_timers.o(.data)
    .data                                    0x20000044   Section        1  nrf_bootloader_fw_activation.o(.data)
    m_flash_write_done                       0x20000044   Data           1  nrf_bootloader_fw_activation.o(.data)
    .data                                    0x20000045   Section        1  nrf_bootloader_wdt.o(.data)
    initialized                              0x20000045   Data           1  nrf_bootloader_wdt.o(.data)
    .data                                    0x20000046   Section        1  nrf_crypto_init.o(.data)
    m_state                                  0x20000046   Data           1  nrf_crypto_init.o(.data)
    .data                                    0x20000048   Section        4  nrf_dfu.o(.data)
    m_user_observer                          0x20000048   Data           4  nrf_dfu.o(.data)
    .data                                    0x2000004c   Section        1  nrf_dfu_handling_error.o(.data)
    m_last_error                             0x2000004c   Data           1  nrf_dfu_handling_error.o(.data)
    .data                                    0x20000050   Section       16  nrf_dfu_req_handler.o(.data)
    current_object                           0x20000050   Data           1  nrf_dfu_req_handler.o(.data)
    m_firmware_start_addr                    0x20000054   Data           4  nrf_dfu_req_handler.o(.data)
    m_firmware_size_req                      0x20000058   Data           4  nrf_dfu_req_handler.o(.data)
    m_observer                               0x2000005c   Data           4  nrf_dfu_req_handler.o(.data)
    .data                                    0x20000060   Section       20  nrf_dfu_serial_uart.o(.data)
    m_rx_byte                                0x20000060   Data           1  nrf_dfu_serial_uart.o(.data)
    m_active                                 0x20000061   Data           1  nrf_dfu_serial_uart.o(.data)
    m_observer                               0x20000064   Data           4  nrf_dfu_serial_uart.o(.data)
    m_uart                                   0x20000068   Data          12  nrf_dfu_serial_uart.o(.data)
    .data                                    0x20000074   Section        3  nrf_dfu_serial_uart.o(.data)
    m_payload_pool_nrf_balloc_pool_stack     0x20000074   Data           3  nrf_dfu_serial_uart.o(.data)
    .data                                    0x20000078   Section        8  nrf_dfu_serial_uart.o(.data)
    m_payload_pool_nrf_balloc_cb             0x20000078   Data           8  nrf_dfu_serial_uart.o(.data)
    .data                                    0x20000080   Section        4  nrf_dfu_settings.o(.data)
    .data                                    0x20000084   Section       16  nrf_dfu_validation.o(.data)
    m_valid_init_cmd_present                 0x20000084   Data           1  nrf_dfu_validation.o(.data)
    m_crypto_initialized                     0x20000085   Data           1  nrf_dfu_validation.o(.data)
    m_init_packet_valid                      0x20000086   Data           1  nrf_dfu_validation.o(.data)
    m_init_packet_data_ptr                   0x20000088   Data           4  nrf_dfu_validation.o(.data)
    m_init_packet_data_len                   0x2000008c   Data           4  nrf_dfu_validation.o(.data)
    mp_init                                  0x20000090   Data           4  nrf_dfu_validation.o(.data)
    .data                                    0x20000094   Section        8  nrf_drv_uart.o(.data)
    m_handlers                               0x20000094   Data           4  nrf_drv_uart.o(.data)
    m_contexts                               0x20000098   Data           4  nrf_drv_uart.o(.data)
    .data                                    0x2000009c   Section       16  app_scheduler.o(.data)
    m_queue_start_index                      0x2000009c   Data           1  app_scheduler.o(.data)
    m_queue_end_index                        0x2000009d   Data           1  app_scheduler.o(.data)
    m_queue_event_size                       0x2000009e   Data           2  app_scheduler.o(.data)
    m_queue_size                             0x200000a0   Data           2  app_scheduler.o(.data)
    m_queue_event_headers                    0x200000a4   Data           4  app_scheduler.o(.data)
    m_queue_event_data                       0x200000a8   Data           4  app_scheduler.o(.data)
    .data                                    0x200000ac   Section        4  app_util_platform.o(.data)
    m_in_critical_region                     0x200000ac   Data           4  app_util_platform.o(.data)
    .data                                    0x200000b0   Section        4  nrf_fstorage_nvmc.o(.data)
    m_flash_operation_ongoing                0x200000b0   Data           4  nrf_fstorage_nvmc.o(.data)
    .data                                    0x200000b4   Section        4  system_nrf52.o(.data)
    __tagsym$$used                           0x200000b4   Number         0  system_nrf52.o(.data)
    fs_data                                  0x200000b8   Section       20  nrf_dfu_flash.o(fs_data)
    __tagsym$$used                           0x200000b8   Number         0  nrf_dfu_flash.o(fs_data)
    .bss                                     0x200000cc   Section     1056  nrf_bootloader.o(.bss)
    APP_SCHED_BUF                            0x200000cc   Data        1056  nrf_bootloader.o(.bss)
    .bss                                     0x200004ec   Section      396  nrf_dfu_serial_uart.o(.bss)
    m_payload_pool_nrf_balloc_pool_mem       0x200004ec   Data         396  nrf_dfu_serial_uart.o(.bss)
    .bss                                     0x20000678   Section       89  nrf_dfu_serial_uart.o(.bss)
    m_serial                                 0x20000678   Data          24  nrf_dfu_serial_uart.o(.bss)
    m_slip                                   0x20000690   Data          16  nrf_dfu_serial_uart.o(.bss)
    m_rsp_buf                                0x200006a0   Data          49  nrf_dfu_serial_uart.o(.bss)
    .bss                                     0x200006d4   Section     2688  nrf_dfu_settings.o(.bss)
    dfu_settings_buffer                      0x200006d4   Data         896  nrf_dfu_settings.o(.bss)
    dfu_settings_buffer                      0x20000a54   Data         896  nrf_dfu_settings.o(.bss)
    .bss                                     0x20001154   Section     1012  nrf_dfu_validation.o(.bss)
    m_packet                                 0x20001154   Data         796  nrf_dfu_validation.o(.bss)
    m_pb_stream                              0x20001470   Data          16  nrf_dfu_validation.o(.bss)
    m_public_key                             0x20001480   Data          72  nrf_dfu_validation.o(.bss)
    m_signature                              0x200014c8   Data          64  nrf_dfu_validation.o(.bss)
    m_sig_hash                               0x20001508   Data          32  nrf_dfu_validation.o(.bss)
    m_fw_hash                                0x20001528   Data          32  nrf_dfu_validation.o(.bss)
    .bss                                     0x20001548   Section       36  nrfx_uarte.o(.bss)
    m_cb                                     0x20001548   Data          36  nrfx_uarte.o(.bss)
    STACK                                    0x20001570   Section     2048  arm_startup_nrf52820.o(STACK)

    Global Symbols

    Symbol Name                              Value     Ov Type        Size  Object(Section)

    BuildAttributes$$THM_ISAv4$E$P$D$K$B$S$7EM$VFPi3$EXTD16$VFPS$VFMA$PE$A:L22UL41UL21$X:L11$S22US41US21$IEEE1$IW$USESV6$~STKCKD$USESV7$~SHL$OSPACE$IEEEX$EBA8$MICROLIB$REQ8$EABIv2 0x00000000   Number         0  anon$$obj.o ABSOLUTE
    __ARM_use_no_argv                        0x00000000   Number         0  main.o ABSOLUTE
    __cpp_initialize__aeabi_                  - Undefined Weak Reference
    __cxa_finalize                            - Undefined Weak Reference
    __decompress                              - Undefined Weak Reference
    _clock_init                               - Undefined Weak Reference
    _microlib_exit                            - Undefined Weak Reference
    crypto_data$$Base                         - Undefined Reference
    crypto_data$$Limit                        - Undefined Reference
    __Vectors_Size                           0x00000200   Number         0  arm_startup_nrf52820.o ABSOLUTE
    Load$$LR$$LR_IROM1$$Base                 0x00038000   Number         0  anon$$obj.o ABSOLUTE
    __Vectors                                0x00038000   Data           4  arm_startup_nrf52820.o(RESET)
    __Vectors_End                            0x00038200   Data           0  arm_startup_nrf52820.o(RESET)
    __main                                   0x00038201   Thumb Code     0  entry.o(.ARM.Collect$$$$00000000)
    _main_stk                                0x00038201   Thumb Code     0  entry2.o(.ARM.Collect$$$$00000001)
    _main_scatterload                        0x00038205   Thumb Code     0  entry5.o(.ARM.Collect$$$$00000004)
    __main_after_scatterload                 0x00038209   Thumb Code     0  entry5.o(.ARM.Collect$$$$00000004)
    _main_clock                              0x00038209   Thumb Code     0  entry7b.o(.ARM.Collect$$$$00000008)
    _main_cpp_init                           0x00038209   Thumb Code     0  entry8b.o(.ARM.Collect$$$$0000000A)
    _main_init                               0x00038209   Thumb Code     0  entry9a.o(.ARM.Collect$$$$0000000B)
    __rt_final_cpp                           0x00038211   Thumb Code     0  entry10a.o(.ARM.Collect$$$$0000000D)
    __rt_final_exit                          0x00038211   Thumb Code     0  entry11a.o(.ARM.Collect$$$$0000000F)
    __asm___12_nrf_atomic_c_85ca2469__nrf_atomic_internal_mov 0x00038215   Thumb Code    24  nrf_atomic.o(.emb_text)
    __asm___12_nrf_atomic_c_85ca2469__nrf_atomic_internal_orr 0x0003822d   Thumb Code    26  nrf_atomic.o(.emb_text)
    __asm___12_nrf_atomic_c_85ca2469__nrf_atomic_internal_and 0x00038247   Thumb Code    26  nrf_atomic.o(.emb_text)
    __asm___12_nrf_atomic_c_85ca2469__nrf_atomic_internal_eor 0x00038261   Thumb Code    26  nrf_atomic.o(.emb_text)
    __asm___12_nrf_atomic_c_85ca2469__nrf_atomic_internal_add 0x0003827b   Thumb Code    26  nrf_atomic.o(.emb_text)
    __asm___12_nrf_atomic_c_85ca2469__nrf_atomic_internal_sub 0x00038295   Thumb Code    26  nrf_atomic.o(.emb_text)
    __asm___12_nrf_atomic_c_85ca2469__nrf_atomic_internal_cmp_exch 0x000382af   Thumb Code    42  nrf_atomic.o(.emb_text)
    __asm___12_nrf_atomic_c_85ca2469__nrf_atomic_internal_sub_hs 0x000382d9   Thumb Code    30  nrf_atomic.o(.emb_text)
    Reset_Handler                            0x000382f9   Thumb Code     8  arm_startup_nrf52820.o(.text)
    NMI_Handler                              0x00038301   Thumb Code     2  arm_startup_nrf52820.o(.text)
    HardFault_Handler                        0x00038303   Thumb Code     2  arm_startup_nrf52820.o(.text)
    MemoryManagement_Handler                 0x00038305   Thumb Code     2  arm_startup_nrf52820.o(.text)
    BusFault_Handler                         0x00038307   Thumb Code     2  arm_startup_nrf52820.o(.text)
    UsageFault_Handler                       0x00038309   Thumb Code     2  arm_startup_nrf52820.o(.text)
    SVC_Handler                              0x0003830b   Thumb Code     2  arm_startup_nrf52820.o(.text)
    DebugMon_Handler                         0x0003830d   Thumb Code     2  arm_startup_nrf52820.o(.text)
    PendSV_Handler                           0x0003830f   Thumb Code     2  arm_startup_nrf52820.o(.text)
    SysTick_Handler                          0x00038311   Thumb Code     2  arm_startup_nrf52820.o(.text)
    CCM_AAR_IRQHandler                       0x00038313   Thumb Code     0  arm_startup_nrf52820.o(.text)
    COMP_IRQHandler                          0x00038313   Thumb Code     0  arm_startup_nrf52820.o(.text)
    ECB_IRQHandler                           0x00038313   Thumb Code     0  arm_startup_nrf52820.o(.text)
    GPIOTE_IRQHandler                        0x00038313   Thumb Code     0  arm_startup_nrf52820.o(.text)
    POWER_CLOCK_IRQHandler                   0x00038313   Thumb Code     0  arm_startup_nrf52820.o(.text)
    QDEC_IRQHandler                          0x00038313   Thumb Code     0  arm_startup_nrf52820.o(.text)
    RADIO_IRQHandler                         0x00038313   Thumb Code     0  arm_startup_nrf52820.o(.text)
    RNG_IRQHandler                           0x00038313   Thumb Code     0  arm_startup_nrf52820.o(.text)
    RTC0_IRQHandler                          0x00038313   Thumb Code     0  arm_startup_nrf52820.o(.text)
    SPIM0_SPIS0_TWIM0_TWIS0_SPI0_TWI0_IRQHandler 0x00038313   Thumb Code     0  arm_startup_nrf52820.o(.text)
    SPIM1_SPIS1_TWIM1_TWIS1_SPI1_TWI1_IRQHandler 0x00038313   Thumb Code     0  arm_startup_nrf52820.o(.text)
    SWI0_EGU0_IRQHandler                     0x00038313   Thumb Code     0  arm_startup_nrf52820.o(.text)
    SWI1_EGU1_IRQHandler                     0x00038313   Thumb Code     0  arm_startup_nrf52820.o(.text)
    SWI2_EGU2_IRQHandler                     0x00038313   Thumb Code     0  arm_startup_nrf52820.o(.text)
    SWI3_EGU3_IRQHandler                     0x00038313   Thumb Code     0  arm_startup_nrf52820.o(.text)
    SWI4_EGU4_IRQHandler                     0x00038313   Thumb Code     0  arm_startup_nrf52820.o(.text)
    SWI5_EGU5_IRQHandler                     0x00038313   Thumb Code     0  arm_startup_nrf52820.o(.text)
    TEMP_IRQHandler                          0x00038313   Thumb Code     0  arm_startup_nrf52820.o(.text)
    TIMER0_IRQHandler                        0x00038313   Thumb Code     0  arm_startup_nrf52820.o(.text)
    TIMER1_IRQHandler                        0x00038313   Thumb Code     0  arm_startup_nrf52820.o(.text)
    TIMER2_IRQHandler                        0x00038313   Thumb Code     0  arm_startup_nrf52820.o(.text)
    TIMER3_IRQHandler                        0x00038313   Thumb Code     0  arm_startup_nrf52820.o(.text)
    USBD_IRQHandler                          0x00038313   Thumb Code     0  arm_startup_nrf52820.o(.text)
    __aeabi_llsl                             0x0003831d   Thumb Code    30  llshl.o(.text)
    _ll_shift_l                              0x0003831d   Thumb Code     0  llshl.o(.text)
    __aeabi_memcpy                           0x0003833b   Thumb Code    36  memcpya.o(.text)
    __aeabi_memcpy4                          0x0003833b   Thumb Code     0  memcpya.o(.text)
    __aeabi_memcpy8                          0x0003833b   Thumb Code     0  memcpya.o(.text)
    __aeabi_memset                           0x0003835f   Thumb Code    14  memseta.o(.text)
    __aeabi_memset4                          0x0003835f   Thumb Code     0  memseta.o(.text)
    __aeabi_memset8                          0x0003835f   Thumb Code     0  memseta.o(.text)
    __aeabi_memclr                           0x0003836d   Thumb Code     4  memseta.o(.text)
    __aeabi_memclr4                          0x0003836d   Thumb Code     0  memseta.o(.text)
    __aeabi_memclr8                          0x0003836d   Thumb Code     0  memseta.o(.text)
    memset                                   0x00038371   Thumb Code    18  memseta.o(.text)
    memcmp                                   0x00038383   Thumb Code    26  memcmp.o(.text)
    __scatterload                            0x0003839d   Thumb Code    28  init.o(.text)
    __scatterload_rt2                        0x0003839d   Thumb Code     0  init.o(.text)
    uECC_secp256r1                           0x000386c1   Thumb Code     8  uECC.c.o(.text.uECC_secp256r1)
    uECC_verify                              0x000386c9   Thumb Code   764  uECC.c.o(.text.uECC_verify)
    RTC1_IRQHandler                          0x0003939d   Thumb Code   106  nrf_bootloader_dfu_timers.o(i.RTC1_IRQHandler)
    SystemInit                               0x00039411   Thumb Code   338  system_nrf52.o(i.SystemInit)
    UARTE0_UART0_IRQHandler                  0x00039589   Thumb Code     8  nrfx_uarte.o(i.UARTE0_UART0_IRQHandler)
    WDT_IRQHandler                           0x00039599   Thumb Code    14  nrf_bootloader_wdt.o(i.WDT_IRQHandler)
    __scatterload_copy                       0x000395ad   Thumb Code    14  handlers.o(i.__scatterload_copy)
    __scatterload_null                       0x000395bb   Thumb Code     2  handlers.o(i.__scatterload_null)
    __scatterload_zeroinit                   0x000395bd   Thumb Code    14  handlers.o(i.__scatterload_zeroinit)
    app_error_handler_bare                   0x00039639   Thumb Code     4  main.o(i.app_error_handler_bare)
    app_sched_event_put                      0x0003963d   Thumb Code   150  app_scheduler.o(i.app_sched_event_put)
    app_sched_execute                        0x000396d9   Thumb Code    58  app_scheduler.o(i.app_sched_execute)
    app_sched_init                           0x00039719   Thumb Code    40  app_scheduler.o(i.app_sched_init)
    app_util_critical_region_enter           0x00039745   Thumb Code     4  app_util_platform.o(i.app_util_critical_region_enter)
    app_util_critical_region_exit            0x00039749   Thumb Code     4  app_util_platform.o(i.app_util_critical_region_exit)
    app_util_disable_irq                     0x0003974d   Thumb Code    12  app_util_platform.o(i.app_util_disable_irq)
    app_util_enable_irq                      0x0003975d   Thumb Code    14  app_util_platform.o(i.app_util_enable_irq)
    bsp_board_init                           0x0003991d   Thumb Code    80  boards.o(i.bsp_board_init)
    bsp_board_led_off                        0x00039971   Thumb Code    10  boards.o(i.bsp_board_led_off)
    bsp_board_led_on                         0x00039981   Thumb Code    10  boards.o(i.bsp_board_led_on)
    bsp_board_leds_off                       0x00039991   Thumb Code    18  boards.o(i.bsp_board_leds_off)
    crc32_compute                            0x000399d1   Thumb Code    54  crc32.o(i.crc32_compute)
    dfu_fstorage_evt_handler                 0x00039c85   Thumb Code    12  nrf_dfu_flash.o(i.dfu_fstorage_evt_handler)
    dfu_req_handler_rsp_clbk                 0x00039d41   Thumb Code    42  nrf_dfu_serial.o(i.dfu_req_handler_rsp_clbk)
    ext_error_get                            0x00039e1d   Thumb Code    10  nrf_dfu_handling_error.o(i.ext_error_get)
    ext_error_set                            0x00039e2d   Thumb Code     8  nrf_dfu_handling_error.o(i.ext_error_set)
    fw_hash_ok                               0x00039e51   Thumb Code     8  nrf_dfu_validation.o(i.fw_hash_ok)
    led_test                                 0x0003a025   Thumb Code    22  main.o(i.led_test)
    main                                     0x0003a041   Thumb Code    38  main.o(i.main)
    nrf_atomic_flag_clear                    0x0003a071   Thumb Code     6  nrf_atomic.o(i.nrf_atomic_flag_clear)
    nrf_atomic_flag_set_fetch                0x0003a077   Thumb Code     6  nrf_atomic.o(i.nrf_atomic_flag_set_fetch)
    nrf_atomic_u32_and                       0x0003a07d   Thumb Code    12  nrf_atomic.o(i.nrf_atomic_u32_and)
    nrf_atomic_u32_fetch_or                  0x0003a089   Thumb Code    10  nrf_atomic.o(i.nrf_atomic_u32_fetch_or)
    nrf_balloc_alloc                         0x0003a093   Thumb Code    62  nrf_balloc.o(i.nrf_balloc_alloc)
    nrf_balloc_free                          0x0003a0d1   Thumb Code    42  nrf_balloc.o(i.nrf_balloc_free)
    nrf_balloc_init                          0x0003a0fb   Thumb Code    48  nrf_balloc.o(i.nrf_balloc_init)
    nrf_bootloader_app_start                 0x0003a12b   Thumb Code    36  nrf_bootloader_app_start.o(i.nrf_bootloader_app_start)
    nrf_bootloader_app_start_final           0x0003a151   Thumb Code    88  nrf_bootloader_app_start_final.o(i.nrf_bootloader_app_start_final)
    nrf_bootloader_dfu_inactivity_timer_restart 0x0003a1b1   Thumb Code    34  nrf_bootloader_dfu_timers.o(i.nrf_bootloader_dfu_inactivity_timer_restart)
    nrf_bootloader_flash_protect             0x0003a1d9   Thumb Code    56  nrf_bootloader_app_start_final.o(i.nrf_bootloader_flash_protect)
    nrf_bootloader_fw_activate               0x0003a219   Thumb Code   102  nrf_bootloader_fw_activation.o(i.nrf_bootloader_fw_activate)
    nrf_bootloader_init                      0x0003a28d   Thumb Code   188  nrf_bootloader.o(i.nrf_bootloader_init)
    nrf_bootloader_mbr_addrs_populate        0x0003a36d   Thumb Code    42  nrf_bootloader_info.o(i.nrf_bootloader_mbr_addrs_populate)
    nrf_bootloader_wdt_feed                  0x0003a39d   Thumb Code    20  nrf_bootloader_wdt.o(i.nrf_bootloader_wdt_feed)
    nrf_bootloader_wdt_feed_timer_start      0x0003a3b1   Thumb Code    16  nrf_bootloader_dfu_timers.o(i.nrf_bootloader_wdt_feed_timer_start)
    nrf_bootloader_wdt_init                  0x0003a3c5   Thumb Code    60  nrf_bootloader_wdt.o(i.nrf_bootloader_wdt_init)
    nrf_crypto_backend_micro_ecc_curve_get   0x0003a40d   Thumb Code     6  micro_ecc_backend_ecc.o(i.nrf_crypto_backend_micro_ecc_curve_get)
    nrf_crypto_backend_micro_ecc_public_key_from_raw 0x0003a413   Thumb Code    16  micro_ecc_backend_ecc.o(i.nrf_crypto_backend_micro_ecc_public_key_from_raw)
    nrf_crypto_backend_micro_ecc_verify      0x0003a423   Thumb Code    86  micro_ecc_backend_ecdsa.o(i.nrf_crypto_backend_micro_ecc_verify)
    nrf_crypto_ecc_public_key_from_raw       0x0003a479   Thumb Code    48  nrf_crypto_ecc.o(i.nrf_crypto_ecc_public_key_from_raw)
    nrf_crypto_ecdsa_verify                  0x0003a4ad   Thumb Code    72  nrf_crypto_ecdsa.o(i.nrf_crypto_ecdsa_verify)
    nrf_crypto_hash_calculate                0x0003a4f9   Thumb Code    54  nrf_crypto_hash.o(i.nrf_crypto_hash_calculate)
    nrf_crypto_hash_finalize                 0x0003a52f   Thumb Code    54  nrf_crypto_hash.o(i.nrf_crypto_hash_finalize)
    nrf_crypto_hash_init                     0x0003a565   Thumb Code    38  nrf_crypto_hash.o(i.nrf_crypto_hash_init)
    nrf_crypto_hash_update                   0x0003a591   Thumb Code    46  nrf_crypto_hash.o(i.nrf_crypto_hash_update)
    nrf_crypto_init                          0x0003a5c1   Thumb Code    50  nrf_crypto_init.o(i.nrf_crypto_init)
    nrf_crypto_internal_double_swap_endian   0x0003a601   Thumb Code    26  nrf_crypto_shared.o(i.nrf_crypto_internal_double_swap_endian)
    nrf_crypto_internal_double_swap_endian_in_place 0x0003a61b   Thumb Code    22  nrf_crypto_shared.o(i.nrf_crypto_internal_double_swap_endian_in_place)
    nrf_crypto_internal_ecc_key_input_check  0x0003a631   Thumb Code    24  nrf_crypto_ecc.o(i.nrf_crypto_internal_ecc_key_input_check)
    nrf_crypto_internal_ecc_key_output_prepare 0x0003a649   Thumb Code    26  nrf_crypto_ecc.o(i.nrf_crypto_internal_ecc_key_output_prepare)
    nrf_crypto_internal_ecc_raw_input_check  0x0003a663   Thumb Code    22  nrf_crypto_ecc.o(i.nrf_crypto_internal_ecc_raw_input_check)
    nrf_crypto_internal_swap_endian          0x0003a679   Thumb Code    22  nrf_crypto_shared.o(i.nrf_crypto_internal_swap_endian)
    nrf_crypto_internal_swap_endian_in_place 0x0003a68f   Thumb Code    24  nrf_crypto_shared.o(i.nrf_crypto_internal_swap_endian_in_place)
    nrf_dfu_app_start_address                0x0003a6a7   Thumb Code     4  nrf_dfu_utils.o(i.nrf_dfu_app_start_address)
    nrf_dfu_bank0_start_addr                 0x0003a6ad   Thumb Code    34  nrf_dfu_utils.o(i.nrf_dfu_bank0_start_addr)
    nrf_dfu_bank1_start_addr                 0x0003a6d5   Thumb Code    28  nrf_dfu_utils.o(i.nrf_dfu_bank1_start_addr)
    nrf_dfu_bank_invalidate                  0x0003a6f5   Thumb Code    14  nrf_dfu_utils.o(i.nrf_dfu_bank_invalidate)
    nrf_dfu_cache_prepare                    0x0003a709   Thumb Code   150  nrf_dfu_utils.o(i.nrf_dfu_cache_prepare)
    nrf_dfu_flash_erase                      0x0003a8b5   Thumb Code    12  nrf_dfu_flash.o(i.nrf_dfu_flash_erase)
    nrf_dfu_flash_init                       0x0003a8c5   Thumb Code    10  nrf_dfu_flash.o(i.nrf_dfu_flash_init)
    nrf_dfu_flash_store                      0x0003a8d9   Thumb Code    18  nrf_dfu_flash.o(i.nrf_dfu_flash_store)
    nrf_dfu_init                             0x0003a8f1   Thumb Code    34  nrf_dfu.o(i.nrf_dfu_init)
    nrf_dfu_init_user                        0x0003a91d   Thumb Code     4  nrf_bootloader.o(i.nrf_dfu_init_user)
    nrf_dfu_mbr_copy_bl                      0x0003a921   Thumb Code    22  nrf_dfu_mbr.o(i.nrf_dfu_mbr_copy_bl)
    nrf_dfu_mbr_irq_forward_address_set      0x0003a939   Thumb Code    40  nrf_dfu_mbr.o(i.nrf_dfu_mbr_irq_forward_address_set)
    nrf_dfu_req_handler_init                 0x0003a965   Thumb Code    62  nrf_dfu_req_handler.o(i.nrf_dfu_req_handler_init)
    nrf_dfu_req_handler_on_req               0x0003a9a9   Thumb Code    16  nrf_dfu_req_handler.o(i.nrf_dfu_req_handler_on_req)
    nrf_dfu_serial_on_packet_received        0x0003aa99   Thumb Code   142  nrf_dfu_serial.o(i.nrf_dfu_serial_on_packet_received)
    nrf_dfu_settings_additional_erase        0x0003ab2d   Thumb Code     4  nrf_dfu_settings.o(i.nrf_dfu_settings_additional_erase)
    nrf_dfu_settings_backup                  0x0003ab31   Thumb Code     6  nrf_dfu_settings.o(i.nrf_dfu_settings_backup)
    nrf_dfu_settings_init                    0x0003ab3d   Thumb Code    26  nrf_dfu_settings.o(i.nrf_dfu_settings_init)
    nrf_dfu_settings_progress_reset          0x0003ab59   Thumb Code    34  nrf_dfu_settings.o(i.nrf_dfu_settings_progress_reset)
    nrf_dfu_settings_reinit                  0x0003ab81   Thumb Code   190  nrf_dfu_settings.o(i.nrf_dfu_settings_reinit)
    nrf_dfu_settings_write                   0x0003ac55   Thumb Code    42  nrf_dfu_settings.o(i.nrf_dfu_settings_write)
    nrf_dfu_settings_write_and_backup        0x0003ac89   Thumb Code    26  nrf_dfu_settings.o(i.nrf_dfu_settings_write_and_backup)
    nrf_dfu_softdevice_invalidate            0x0003aca9   Thumb Code    56  nrf_dfu_utils.o(i.nrf_dfu_softdevice_invalidate)
    nrf_dfu_softdevice_start_address         0x0003aced   Thumb Code     6  nrf_dfu_utils.o(i.nrf_dfu_softdevice_start_address)
    nrf_dfu_transports_close                 0x0003acf5   Thumb Code    44  nrf_dfu_transport.o(i.nrf_dfu_transports_close)
    nrf_dfu_transports_init                  0x0003ad29   Thumb Code    42  nrf_dfu_transport.o(i.nrf_dfu_transports_init)
    nrf_dfu_validation_activation_prepare    0x0003ad5d   Thumb Code     6  nrf_dfu_validation.o(i.nrf_dfu_validation_activation_prepare)
    nrf_dfu_validation_boot_validate         0x0003ad63   Thumb Code    82  nrf_dfu_validation.o(i.nrf_dfu_validation_boot_validate)
    nrf_dfu_validation_init                  0x0003ae19   Thumb Code    26  nrf_dfu_validation.o(i.nrf_dfu_validation_init)
    nrf_dfu_validation_init_cmd_append       0x0003ae3d   Thumb Code    66  nrf_dfu_validation.o(i.nrf_dfu_validation_init_cmd_append)
    nrf_dfu_validation_init_cmd_create       0x0003ae85   Thumb Code    42  nrf_dfu_validation.o(i.nrf_dfu_validation_init_cmd_create)
    nrf_dfu_validation_init_cmd_execute      0x0003aeb9   Thumb Code   132  nrf_dfu_validation.o(i.nrf_dfu_validation_init_cmd_execute)
    nrf_dfu_validation_init_cmd_present      0x0003af45   Thumb Code     6  nrf_dfu_validation.o(i.nrf_dfu_validation_init_cmd_present)
    nrf_dfu_validation_prevalidate           0x0003af51   Thumb Code    64  nrf_dfu_validation.o(i.nrf_dfu_validation_prevalidate)
    nrf_dfu_ver_validation_check             0x0003b02d   Thumb Code   122  nrf_dfu_ver_validation.o(i.nrf_dfu_ver_validation_check)
    nrf_drv_uart_init                        0x0003b0ad   Thumb Code    56  nrf_drv_uart.o(i.nrf_drv_uart_init)
    nrf_fstorage_erase                       0x0003b0f3   Thumb Code    44  nrf_fstorage.o(i.nrf_fstorage_erase)
    nrf_fstorage_init                        0x0003b11f   Thumb Code     8  nrf_fstorage.o(i.nrf_fstorage_init)
    nrf_fstorage_is_busy                     0x0003b129   Thumb Code    70  nrf_fstorage.o(i.nrf_fstorage_is_busy)
    nrf_fstorage_write                       0x0003b179   Thumb Code    62  nrf_fstorage.o(i.nrf_fstorage_write)
    nrf_nvmc_page_erase                      0x0003b24d   Thumb Code    40  nrf_nvmc.o(i.nrf_nvmc_page_erase)
    nrf_nvmc_write_word                      0x0003b27d   Thumb Code    38  nrf_nvmc.o(i.nrf_nvmc_write_word)
    nrf_nvmc_write_words                     0x0003b2ad   Thumb Code    58  nrf_nvmc.o(i.nrf_nvmc_write_words)
    nrfx_prs_acquire                         0x0003b365   Thumb Code     4  nrfx_prs.o(i.nrfx_prs_acquire)
    nrfx_prs_release                         0x0003b369   Thumb Code     2  nrfx_prs.o(i.nrfx_prs_release)
    nrfx_uarte_init                          0x0003b36d   Thumb Code   100  nrfx_uarte.o(i.nrfx_uarte_init)
    nrfx_uarte_rx                            0x0003b3d9   Thumb Code   256  nrfx_uarte.o(i.nrfx_uarte_rx)
    nrfx_uarte_tx                            0x0003b4dd   Thumb Code   166  nrfx_uarte.o(i.nrfx_uarte_tx)
    nrfx_uarte_tx_in_progress                0x0003b589   Thumb Code    22  nrfx_uarte.o(i.nrfx_uarte_tx_in_progress)
    nrfx_uarte_uninit                        0x0003b5a5   Thumb Code   254  nrfx_uarte.o(i.nrfx_uarte_uninit)
    nvmc_config                              0x0003b6ad   Thumb Code    14  system_nrf52.o(i.nvmc_config)
    pb_decode                                0x0003bad9   Thumb Code    30  pb_decode.o(i.pb_decode)
    pb_decode_fixed32                        0x0003baf7   Thumb Code    32  pb_decode.o(i.pb_decode_fixed32)
    pb_decode_fixed64                        0x0003bb17   Thumb Code    92  pb_decode.o(i.pb_decode_fixed64)
    pb_decode_noinit                         0x0003bb75   Thumb Code   390  pb_decode.o(i.pb_decode_noinit)
    pb_decode_svarint                        0x0003bcfb   Thumb Code    58  pb_decode.o(i.pb_decode_svarint)
    pb_decode_tag                            0x0003bd35   Thumb Code    60  pb_decode.o(i.pb_decode_tag)
    pb_decode_varint                         0x0003bd71   Thumb Code    74  pb_decode.o(i.pb_decode_varint)
    pb_field_iter_begin                      0x0003be45   Thumb Code    34  pb_common.o(i.pb_field_iter_begin)
    pb_field_iter_find                       0x0003be67   Thumb Code    46  pb_common.o(i.pb_field_iter_find)
    pb_field_iter_next                       0x0003be95   Thumb Code   126  pb_common.o(i.pb_field_iter_next)
    pb_istream_from_buffer                   0x0003bfb9   Thumb Code    14  pb_decode.o(i.pb_istream_from_buffer)
    pb_make_string_substream                 0x0003bfcd   Thumb Code    54  pb_decode.o(i.pb_make_string_substream)
    pb_read                                  0x0003c029   Thumb Code    84  pb_decode.o(i.pb_read)
    pb_skip_field                            0x0003c0a1   Thumb Code    90  pb_decode.o(i.pb_skip_field)
    postvalidate                             0x0003c0fd   Thumb Code   226  nrf_dfu_validation.o(i.postvalidate)
    settings_backup                          0x0003c599   Thumb Code    12  nrf_dfu_settings.o(i.settings_backup)
    sha256_final                             0x0003c607   Thumb Code   272  sha256.o(i.sha256_final)
    sha256_init                              0x0003c719   Thumb Code    50  sha256.o(i.sha256_init)
    sha256_transform                         0x0003c76d   Thumb Code   294  sha256.o(i.sha256_transform)
    sha256_update                            0x0003c899   Thumb Code    84  sha256.o(i.sha256_update)
    slip_decode_add_byte                     0x0003c8ed   Thumb Code   110  slip.o(i.slip_decode_add_byte)
    slip_encode                              0x0003c95b   Thumb Code    86  slip.o(i.slip_encode)
    pk                                       0x0003cf58   Data          64  dfu_public_key.o(.constdata)
    g_nrf_crypto_hash_sha256_info            0x0003cfa8   Data          24  nrf_sw_backend_hash.o(.constdata)
    g_nrf_crypto_ecc_secp256r1_curve_info    0x0003cfc0   Data          12  micro_ecc_backend_ecc.o(.constdata)
    dfu_init_command_is_debug_default        0x0003cfcc   Data           1  dfu-cc.pb.o(.constdata)
    dfu_hash_fields                          0x0003cfd0   Data          48  dfu-cc.pb.o(.constdata)
    dfu_boot_validation_fields               0x0003d000   Data          48  dfu-cc.pb.o(.constdata)
    dfu_init_command_fields                  0x0003d030   Data         176  dfu-cc.pb.o(.constdata)
    dfu_command_fields                       0x0003d0e0   Data          48  dfu-cc.pb.o(.constdata)
    dfu_signed_command_fields                0x0003d110   Data          64  dfu-cc.pb.o(.constdata)
    dfu_packet_fields                        0x0003d150   Data          48  dfu-cc.pb.o(.constdata)
    nrf_fstorage_nvmc                        0x0003d204   Data          32  nrf_fstorage_nvmc.o(.constdata)
    Region$$Table$$Base                      0x0003d410   Number         0  anon$$obj.o(Region$$Table)
    Region$$Table$$Limit                     0x0003d430   Number         0  anon$$obj.o(Region$$Table)
    dfu_trans$$Base                          0x0003d430   Number         0  nrf_dfu_serial_uart.o(dfu_trans)
    uart_dfu_transport                       0x0003d430   Data           8  nrf_dfu_serial_uart.o(dfu_trans)
    dfu_trans$$Limit                         0x0003d438   Number         0  nrf_dfu_serial_uart.o(dfu_trans)
    m_payload_pool                           0x0003d438   Data          20  nrf_dfu_serial_uart.o(nrf_balloc)
    m_mbr_params_page                        0x0003e000   Data        4096  nrf_dfu_settings.o(.ARM.__AT_0x0003E000)
    m_dfu_settings_buffer                    0x0003f000   Data        4096  nrf_dfu_settings.o(.ARM.__AT_0x0003F000)
    m_uicr_bootloader_start_address          0x10001014   Data           4  nrf_bootloader_info.o(.ARM.__AT_0x10001014)
    m_uicr_mbr_params_page_address           0x10001018   Data           4  nrf_dfu_settings.o(.ARM.__AT_0x10001018)
    mp_inactivity                            0x20000018   Data           4  nrf_bootloader_dfu_timers.o(.data)
    mp_wdt_feed                              0x2000001c   Data           4  nrf_bootloader_dfu_timers.o(.data)
    m_counter_loops                          0x20000020   Data           4  nrf_bootloader_dfu_timers.o(.data)
    m_timers                                 0x20000024   Data          32  nrf_bootloader_dfu_timers.o(.data)
    mp_dfu_settings_backup_buffer            0x20000080   Data           4  nrf_dfu_settings.o(.data)
    SystemCoreClock                          0x200000b4   Data           4  system_nrf52.o(.data)
    fs_data$$Base                            0x200000b8   Number         0  nrf_dfu_flash.o(fs_data)
    m_fs                                     0x200000b8   Data          20  nrf_dfu_flash.o(fs_data)
    fs_data$$Limit                           0x200000cc   Number         0  nrf_dfu_flash.o(fs_data)
    s_dfu_settings                           0x20000dd4   Data         896  nrf_dfu_settings.o(.bss)
    __initial_sp                             0x20001d70   Data           0  arm_startup_nrf52820.o(STACK)



==============================================================================

Memory Map of the image

  Image Entry point : 0x00038201

  Load Region LR_IROM1 (Base: 0x00038000, Size: 0x00005510, Max: 0x00006000, ABSOLUTE)

    Execution Region ER_IROM1 (Base: 0x00038000, Size: 0x0000544c, Max: 0x00006000, ABSOLUTE)

    Base Addr    Size         Type   Attr      Idx    E Section Name        Object

    0x00038000   0x00000200   Data   RO         4355    RESET               arm_startup_nrf52820.o
    0x00038200   0x00000000   Code   RO         4492  * .ARM.Collect$$$$00000000  mc_w.l(entry.o)
    0x00038200   0x00000004   Code   RO         4509    .ARM.Collect$$$$00000001  mc_w.l(entry2.o)
    0x00038204   0x00000004   Code   RO         4512    .ARM.Collect$$$$00000004  mc_w.l(entry5.o)
    0x00038208   0x00000000   Code   RO         4514    .ARM.Collect$$$$00000008  mc_w.l(entry7b.o)
    0x00038208   0x00000000   Code   RO         4516    .ARM.Collect$$$$0000000A  mc_w.l(entry8b.o)
    0x00038208   0x00000008   Code   RO         4517    .ARM.Collect$$$$0000000B  mc_w.l(entry9a.o)
    0x00038210   0x00000000   Code   RO         4519    .ARM.Collect$$$$0000000D  mc_w.l(entry10a.o)
    0x00038210   0x00000000   Code   RO         4521    .ARM.Collect$$$$0000000F  mc_w.l(entry11a.o)
    0x00038210   0x00000004   Code   RO         4510    .ARM.Collect$$$$00002712  mc_w.l(entry2.o)
    0x00038214   0x000000e2   Code   RO         3378    .emb_text           nrf_atomic.o
    0x000382f6   0x00000002   PAD
    0x000382f8   0x00000024   Code   RO         4356    .text               arm_startup_nrf52820.o
    0x0003831c   0x0000001e   Code   RO         4495    .text               mc_w.l(llshl.o)
    0x0003833a   0x00000024   Code   RO         4497    .text               mc_w.l(memcpya.o)
    0x0003835e   0x00000024   Code   RO         4501    .text               mc_w.l(memseta.o)
    0x00038382   0x0000001a   Code   RO         4505    .text               mc_w.l(memcmp.o)
    0x0003839c   0x00000024   Code   RO         4523    .text               mc_w.l(init.o)
    0x000383c0   0x000000ce   Code   RO         4446    .text.XYcZ_add      micro_ecc_lib_nrf52.lib(uECC.c.o)
    0x0003848e   0x0000003e   Code   RO         4445    .text.apply_z       micro_ecc_lib_nrf52.lib(uECC.c.o)
    0x000384cc   0x00000014   Code   RO         4418    .text.bcopy         micro_ecc_lib_nrf52.lib(uECC.c.o)
    0x000384e0   0x0000008e   Code   RO         4450    .text.bits2int      micro_ecc_lib_nrf52.lib(uECC.c.o)
    0x0003856e   0x00000152   Code   RO         4435    .text.double_jacobian_default  micro_ecc_lib_nrf52.lib(uECC.c.o)
    0x000386c0   0x00000008   Code   RO         4468    .text.uECC_secp256r1  micro_ecc_lib_nrf52.lib(uECC.c.o)
    0x000386c8   0x000002fc   Code   RO         4477    .text.uECC_verify   micro_ecc_lib_nrf52.lib(uECC.c.o)
    0x000389c4   0x0000000c   PAD
    0x000389d0   0x00000058   Code   RO         4419    .text.uECC_vli_add  micro_ecc_lib_nrf52.lib(uECC.c.o)
    0x00038a28   0x00000016   Code   RO         4422    .text.uECC_vli_clear  micro_ecc_lib_nrf52.lib(uECC.c.o)
    0x00038a3e   0x0000002a   Code   RO         4427    .text.uECC_vli_cmp_unsafe  micro_ecc_lib_nrf52.lib(uECC.c.o)
    0x00038a68   0x0000001e   Code   RO         4423    .text.uECC_vli_isZero  micro_ecc_lib_nrf52.lib(uECC.c.o)
    0x00038a86   0x00000038   Code   RO         4430    .text.uECC_vli_modAdd  micro_ecc_lib_nrf52.lib(uECC.c.o)
    0x00038abe   0x00000106   Code   RO         4456    .text.uECC_vli_modInv  micro_ecc_lib_nrf52.lib(uECC.c.o)
    0x00038bc4   0x0000013c   Code   RO         4432    .text.uECC_vli_modMult  micro_ecc_lib_nrf52.lib(uECC.c.o)
    0x00038d00   0x00000020   Code   RO         4433    .text.uECC_vli_modMult_fast  micro_ecc_lib_nrf52.lib(uECC.c.o)
    0x00038d20   0x00000008   Code   RO         4434    .text.uECC_vli_modSquare_fast  micro_ecc_lib_nrf52.lib(uECC.c.o)
    0x00038d28   0x00000028   Code   RO         4431    .text.uECC_vli_modSub  micro_ecc_lib_nrf52.lib(uECC.c.o)
    0x00038d50   0x00000312   Code   RO         4421    .text.uECC_vli_mult  micro_ecc_lib_nrf52.lib(uECC.c.o)
    0x00039062   0x00000040   Code   RO         4425    .text.uECC_vli_numBits  micro_ecc_lib_nrf52.lib(uECC.c.o)
    0x000390a2   0x0000001a   Code   RO         4429    .text.uECC_vli_rshift1  micro_ecc_lib_nrf52.lib(uECC.c.o)
    0x000390bc   0x00000018   Code   RO         4426    .text.uECC_vli_set  micro_ecc_lib_nrf52.lib(uECC.c.o)
    0x000390d4   0x0000000c   PAD
    0x000390e0   0x00000060   Code   RO         4420    .text.uECC_vli_sub  micro_ecc_lib_nrf52.lib(uECC.c.o)
    0x00039140   0x00000014   Code   RO         4424    .text.uECC_vli_testBit  micro_ecc_lib_nrf52.lib(uECC.c.o)
    0x00039154   0x000001b0   Code   RO         4441    .text.vli_mmod_fast_secp256r1  micro_ecc_lib_nrf52.lib(uECC.c.o)
    0x00039304   0x00000038   Code   RO         4455    .text.vli_modInv_update  micro_ecc_lib_nrf52.lib(uECC.c.o)
    0x0003933c   0x0000005e   Code   RO         4436    .text.x_side_default  micro_ecc_lib_nrf52.lib(uECC.c.o)
    0x0003939a   0x00000002   PAD
    0x0003939c   0x00000074   Code   RO          590    i.RTC1_IRQHandler   nrf_bootloader_dfu_timers.o
    0x00039410   0x00000178   Code   RO         4364    i.SystemInit        system_nrf52.o
    0x00039588   0x00000010   Code   RO         2932    i.UARTE0_UART0_IRQHandler  nrfx_uarte.o
    0x00039598   0x00000014   Code   RO          769    i.WDT_IRQHandler    nrf_bootloader_wdt.o
    0x000395ac   0x0000000e   Code   RO         4527    i.__scatterload_copy  mc_w.l(handlers.o)
    0x000395ba   0x00000002   Code   RO         4528    i.__scatterload_null  mc_w.l(handlers.o)
    0x000395bc   0x0000000e   Code   RO         4529    i.__scatterload_zeroinit  mc_w.l(handlers.o)
    0x000395ca   0x0000000c   Code   RO         3633    i.addr_is_aligned32  nrf_fstorage.o
    0x000395d6   0x00000018   Code   RO         3634    i.addr_is_within_bounds  nrf_fstorage.o
    0x000395ee   0x00000002   PAD
    0x000395f0   0x00000048   Code   RO          674    i.app_activate      nrf_bootloader_fw_activation.o
    0x00039638   0x00000004   Code   RO           23    i.app_error_handler_bare  main.o
    0x0003963c   0x0000009c   Code   RO         3126    i.app_sched_event_put  app_scheduler.o
    0x000396d8   0x00000040   Code   RO         3127    i.app_sched_execute  app_scheduler.o
    0x00039718   0x0000002c   Code   RO         3128    i.app_sched_init    app_scheduler.o
    0x00039744   0x00000004   Code   RO         3181    i.app_util_critical_region_enter  app_util_platform.o
    0x00039748   0x00000004   Code   RO         3182    i.app_util_critical_region_exit  app_util_platform.o
    0x0003974c   0x00000010   Code   RO         3183    i.app_util_disable_irq  app_util_platform.o
    0x0003975c   0x00000014   Code   RO         3184    i.app_util_enable_irq  app_util_platform.o
    0x00039770   0x00000088   Code   RO         2933    i.apply_config      nrfx_uarte.o
    0x000397f8   0x0000004c   Code   RO          675    i.bl_activate       nrf_bootloader_fw_activation.o
    0x00039844   0x00000010   Code   RO          404    i.boot_validate     nrf_bootloader.o
    0x00039854   0x0000000c   Code   RO         2108    i.boot_validation_crc  nrf_dfu_settings.o
    0x00039860   0x00000098   Code   RO         2320    i.boot_validation_extract  nrf_dfu_validation.o
    0x000398f8   0x00000024   Code   RO          405    i.bootloader_reset  nrf_bootloader.o
    0x0003991c   0x00000054   Code   RO          299    i.bsp_board_init    boards.o
    0x00039970   0x00000010   Code   RO          302    i.bsp_board_led_off  boards.o
    0x00039980   0x00000010   Code   RO          303    i.bsp_board_led_on  boards.o
    0x00039990   0x00000012   Code   RO          305    i.bsp_board_leds_off  boards.o
    0x000399a2   0x0000001c   Code   RO         4171    i.buf_read          pb_decode.o
    0x000399be   0x00000002   PAD
    0x000399c0   0x00000010   Code   RO         1749    i.cmd_response_offset_and_crc_set  nrf_dfu_req_handler.o
    0x000399d0   0x0000003c   Code   RO         3243    i.crc32_compute     crc32.o
    0x00039a0c   0x0000001e   Code   RO         2109    i.crc_ok            nrf_dfu_settings.o
    0x00039a2a   0x00000002   PAD
    0x00039a2c   0x00000040   Code   RO         2321    i.crypto_init       nrf_dfu_validation.o
    0x00039a6c   0x0000007e   Code   RO         4172    i.decode_callback_field  pb_decode.o
    0x00039aea   0x0000001a   Code   RO         4173    i.decode_field      pb_decode.o
    0x00039b04   0x000000e0   Code   RO         4174    i.decode_static_field  pb_decode.o
    0x00039be4   0x000000a0   Code   RO          406    i.dfu_enter_check   nrf_bootloader.o
    0x00039c84   0x0000000c   Code   RO         1613    i.dfu_fstorage_evt_handler  nrf_dfu_flash.o
    0x00039c90   0x00000040   Code   RO           24    i.dfu_observer      main.o
    0x00039cd0   0x00000048   Code   RO          407    i.dfu_observer      nrf_bootloader.o
    0x00039d18   0x00000028   Code   RO         1579    i.dfu_observer      nrf_dfu.o
    0x00039d40   0x0000002a   Code   RO         4095    i.dfu_req_handler_rsp_clbk  nrf_dfu_serial.o
    0x00039d6a   0x00000002   PAD
    0x00039d6c   0x00000024   Code   RO          408    i.do_reset          nrf_bootloader.o
    0x00039d90   0x00000048   Code   RO         3719    i.erase             nrf_fstorage_nvmc.o
    0x00039dd8   0x00000036   Code   RO         3720    i.event_send        nrf_fstorage_nvmc.o
    0x00039e0e   0x0000000e   Code   RO         1750    i.ext_err_code_handle  nrf_dfu_req_handler.o
    0x00039e1c   0x00000010   Code   RO         1674    i.ext_error_get     nrf_dfu_handling_error.o
    0x00039e2c   0x0000000c   Code   RO         1675    i.ext_error_set     nrf_dfu_handling_error.o
    0x00039e38   0x0000000c   Code   RO          409    i.flash_write_callback  nrf_bootloader.o
    0x00039e44   0x0000000c   Code   RO          676    i.flash_write_callback  nrf_bootloader_fw_activation.o
    0x00039e50   0x00000008   Code   RO         2322    i.fw_hash_ok        nrf_dfu_validation.o
    0x00039e58   0x00000090   Code   RO          677    i.image_copy        nrf_bootloader_fw_activation.o
    0x00039ee8   0x00000006   Code   RO          410    i.inactivity_timeout  nrf_bootloader.o
    0x00039eee   0x00000002   PAD
    0x00039ef0   0x0000000c   Code   RO         3721    i.init              nrf_fstorage_nvmc.o
    0x00039efc   0x00000088   Code   RO         2934    i.interrupts_enable  nrfx_uarte.o
    0x00039f84   0x00000010   Code   RO         3722    i.is_busy           nrf_fstorage_nvmc.o
    0x00039f94   0x00000060   Code   RO         2323    i.is_major_softdevice_update  nrf_dfu_validation.o
    0x00039ff4   0x0000002e   Code   RO         4175    i.iter_from_extension  pb_decode.o
    0x0003a022   0x00000002   PAD
    0x0003a024   0x0000001c   Code   RO           25    i.led_test          main.o
    0x0003a040   0x00000030   Code   RO           26    i.main              main.o
    0x0003a070   0x00000006   Code   RO         3379    i.nrf_atomic_flag_clear  nrf_atomic.o
    0x0003a076   0x00000006   Code   RO         3382    i.nrf_atomic_flag_set_fetch  nrf_atomic.o
    0x0003a07c   0x0000000c   Code   RO         3384    i.nrf_atomic_u32_and  nrf_atomic.o
    0x0003a088   0x0000000a   Code   RO         3388    i.nrf_atomic_u32_fetch_or  nrf_atomic.o
    0x0003a092   0x0000003e   Code   RO         3517    i.nrf_balloc_alloc  nrf_balloc.o
    0x0003a0d0   0x0000002a   Code   RO         3518    i.nrf_balloc_free   nrf_balloc.o
    0x0003a0fa   0x00000030   Code   RO         3519    i.nrf_balloc_init   nrf_balloc.o
    0x0003a12a   0x00000024   Code   RO          523    i.nrf_bootloader_app_start  nrf_bootloader_app_start.o
    0x0003a14e   0x00000002   PAD
    0x0003a150   0x00000060   Code   RO          551    i.nrf_bootloader_app_start_final  nrf_bootloader_app_start_final.o
    0x0003a1b0   0x00000028   Code   RO          591    i.nrf_bootloader_dfu_inactivity_timer_restart  nrf_bootloader_dfu_timers.o
    0x0003a1d8   0x00000040   Code   RO          552    i.nrf_bootloader_flash_protect  nrf_bootloader_app_start_final.o
    0x0003a218   0x00000074   Code   RO          678    i.nrf_bootloader_fw_activate  nrf_bootloader_fw_activation.o
    0x0003a28c   0x000000e0   Code   RO          411    i.nrf_bootloader_init  nrf_bootloader.o
    0x0003a36c   0x00000030   Code   RO          730    i.nrf_bootloader_mbr_addrs_populate  nrf_bootloader_info.o
    0x0003a39c   0x00000014   Code   RO          770    i.nrf_bootloader_wdt_feed  nrf_bootloader_wdt.o
    0x0003a3b0   0x00000014   Code   RO          593    i.nrf_bootloader_wdt_feed_timer_start  nrf_bootloader_dfu_timers.o
    0x0003a3c4   0x00000048   Code   RO          771    i.nrf_bootloader_wdt_init  nrf_bootloader_wdt.o
    0x0003a40c   0x00000006   Code   RO         1371    i.nrf_crypto_backend_micro_ecc_curve_get  micro_ecc_backend_ecc.o
    0x0003a412   0x00000010   Code   RO         1376    i.nrf_crypto_backend_micro_ecc_public_key_from_raw  micro_ecc_backend_ecc.o
    0x0003a422   0x00000056   Code   RO         1529    i.nrf_crypto_backend_micro_ecc_verify  micro_ecc_backend_ecdsa.o
    0x0003a478   0x00000034   Code   RO          840    i.nrf_crypto_ecc_public_key_from_raw  nrf_crypto_ecc.o
    0x0003a4ac   0x0000004c   Code   RO          997    i.nrf_crypto_ecdsa_verify  nrf_crypto_ecdsa.o
    0x0003a4f8   0x00000036   Code   RO         1072    i.nrf_crypto_hash_calculate  nrf_crypto_hash.o
    0x0003a52e   0x00000036   Code   RO         1073    i.nrf_crypto_hash_finalize  nrf_crypto_hash.o
    0x0003a564   0x0000002c   Code   RO         1074    i.nrf_crypto_hash_init  nrf_crypto_hash.o
    0x0003a590   0x0000002e   Code   RO         1075    i.nrf_crypto_hash_update  nrf_crypto_hash.o
    0x0003a5be   0x00000002   PAD
    0x0003a5c0   0x00000040   Code   RO         1150    i.nrf_crypto_init   nrf_crypto_init.o
    0x0003a600   0x0000001a   Code   RO         1201    i.nrf_crypto_internal_double_swap_endian  nrf_crypto_shared.o
    0x0003a61a   0x00000016   Code   RO         1202    i.nrf_crypto_internal_double_swap_endian_in_place  nrf_crypto_shared.o
    0x0003a630   0x00000018   Code   RO          842    i.nrf_crypto_internal_ecc_key_input_check  nrf_crypto_ecc.o
    0x0003a648   0x0000001a   Code   RO          843    i.nrf_crypto_internal_ecc_key_output_prepare  nrf_crypto_ecc.o
    0x0003a662   0x00000016   Code   RO          844    i.nrf_crypto_internal_ecc_raw_input_check  nrf_crypto_ecc.o
    0x0003a678   0x00000016   Code   RO         1203    i.nrf_crypto_internal_swap_endian  nrf_crypto_shared.o
    0x0003a68e   0x00000018   Code   RO         1204    i.nrf_crypto_internal_swap_endian_in_place  nrf_crypto_shared.o
    0x0003a6a6   0x00000004   Code   RO         2241    i.nrf_dfu_app_start_address  nrf_dfu_utils.o
    0x0003a6aa   0x00000002   PAD
    0x0003a6ac   0x00000028   Code   RO         2242    i.nrf_dfu_bank0_start_addr  nrf_dfu_utils.o
    0x0003a6d4   0x00000020   Code   RO         2243    i.nrf_dfu_bank1_start_addr  nrf_dfu_utils.o
    0x0003a6f4   0x00000014   Code   RO         2244    i.nrf_dfu_bank_invalidate  nrf_dfu_utils.o
    0x0003a708   0x000000a4   Code   RO         2245    i.nrf_dfu_cache_prepare  nrf_dfu_utils.o
    0x0003a7ac   0x00000094   Code   RO         1751    i.nrf_dfu_command_req  nrf_dfu_req_handler.o
    0x0003a840   0x00000074   Code   RO         1752    i.nrf_dfu_data_req  nrf_dfu_req_handler.o
    0x0003a8b4   0x00000010   Code   RO         1614    i.nrf_dfu_flash_erase  nrf_dfu_flash.o
    0x0003a8c4   0x00000014   Code   RO         1615    i.nrf_dfu_flash_init  nrf_dfu_flash.o
    0x0003a8d8   0x00000018   Code   RO         1616    i.nrf_dfu_flash_store  nrf_dfu_flash.o
    0x0003a8f0   0x0000002c   Code   RO         1580    i.nrf_dfu_init      nrf_dfu.o
    0x0003a91c   0x00000004   Code   RO          413    i.nrf_dfu_init_user  nrf_bootloader.o
    0x0003a920   0x00000016   Code   RO         1706    i.nrf_dfu_mbr_copy_bl  nrf_dfu_mbr.o
    0x0003a936   0x00000002   PAD
    0x0003a938   0x0000002c   Code   RO         1708    i.nrf_dfu_mbr_irq_forward_address_set  nrf_dfu_mbr.o
    0x0003a964   0x00000044   Code   RO         1753    i.nrf_dfu_req_handler_init  nrf_dfu_req_handler.o
    0x0003a9a8   0x00000014   Code   RO         1754    i.nrf_dfu_req_handler_on_req  nrf_dfu_req_handler.o
    0x0003a9bc   0x00000004   Code   RO         1755    i.nrf_dfu_req_handler_req  nrf_dfu_req_handler.o
    0x0003a9c0   0x000000d8   Code   RO         1756    i.nrf_dfu_req_handler_req_process  nrf_dfu_req_handler.o
    0x0003aa98   0x00000094   Code   RO         4096    i.nrf_dfu_serial_on_packet_received  nrf_dfu_serial.o
    0x0003ab2c   0x00000004   Code   RO         2110    i.nrf_dfu_settings_additional_erase  nrf_dfu_settings.o
    0x0003ab30   0x0000000c   Code   RO         2111    i.nrf_dfu_settings_backup  nrf_dfu_settings.o
    0x0003ab3c   0x0000001a   Code   RO         2112    i.nrf_dfu_settings_init  nrf_dfu_settings.o
    0x0003ab56   0x00000002   PAD
    0x0003ab58   0x00000028   Code   RO         2113    i.nrf_dfu_settings_progress_reset  nrf_dfu_settings.o
    0x0003ab80   0x000000d4   Code   RO         2114    i.nrf_dfu_settings_reinit  nrf_dfu_settings.o
    0x0003ac54   0x00000034   Code   RO         2115    i.nrf_dfu_settings_write  nrf_dfu_settings.o
    0x0003ac88   0x00000020   Code   RO         2116    i.nrf_dfu_settings_write_and_backup  nrf_dfu_settings.o
    0x0003aca8   0x00000044   Code   RO         2246    i.nrf_dfu_softdevice_invalidate  nrf_dfu_utils.o
    0x0003acec   0x00000006   Code   RO         2247    i.nrf_dfu_softdevice_start_address  nrf_dfu_utils.o
    0x0003acf2   0x00000002   PAD
    0x0003acf4   0x00000034   Code   RO         2210    i.nrf_dfu_transports_close  nrf_dfu_transport.o
    0x0003ad28   0x00000034   Code   RO         2211    i.nrf_dfu_transports_init  nrf_dfu_transport.o
    0x0003ad5c   0x00000006   Code   RO         2324    i.nrf_dfu_validation_activation_prepare  nrf_dfu_validation.o
    0x0003ad62   0x00000052   Code   RO         2325    i.nrf_dfu_validation_boot_validate  nrf_dfu_validation.o
    0x0003adb4   0x00000064   Code   RO         2326    i.nrf_dfu_validation_hash_ok  nrf_dfu_validation.o
    0x0003ae18   0x00000024   Code   RO         2327    i.nrf_dfu_validation_init  nrf_dfu_validation.o
    0x0003ae3c   0x00000048   Code   RO         2328    i.nrf_dfu_validation_init_cmd_append  nrf_dfu_validation.o
    0x0003ae84   0x00000034   Code   RO         2329    i.nrf_dfu_validation_init_cmd_create  nrf_dfu_validation.o
    0x0003aeb8   0x0000008c   Code   RO         2330    i.nrf_dfu_validation_init_cmd_execute  nrf_dfu_validation.o
    0x0003af44   0x0000000c   Code   RO         2331    i.nrf_dfu_validation_init_cmd_present  nrf_dfu_validation.o
    0x0003af50   0x00000048   Code   RO         2334    i.nrf_dfu_validation_prevalidate  nrf_dfu_validation.o
    0x0003af98   0x00000094   Code   RO         2335    i.nrf_dfu_validation_signature_check  nrf_dfu_validation.o
    0x0003b02c   0x00000080   Code   RO         2485    i.nrf_dfu_ver_validation_check  nrf_dfu_ver_validation.o
    0x0003b0ac   0x00000040   Code   RO         2527    i.nrf_drv_uart_init  nrf_drv_uart.o
    0x0003b0ec   0x00000006   Code   RO         2015    i.nrf_drv_uart_rx   nrf_dfu_serial_uart.o
    0x0003b0f2   0x0000002c   Code   RO         3635    i.nrf_fstorage_erase  nrf_fstorage.o
    0x0003b11e   0x00000008   Code   RO         3636    i.nrf_fstorage_init  nrf_fstorage.o
    0x0003b126   0x00000002   PAD
    0x0003b128   0x00000050   Code   RO         3637    i.nrf_fstorage_is_busy  nrf_fstorage.o
    0x0003b178   0x0000003e   Code   RO         3642    i.nrf_fstorage_write  nrf_fstorage.o
    0x0003b1b6   0x00000024   Code   RO          309    i.nrf_gpio_cfg      boards.o
    0x0003b1da   0x00000024   Code   RO         2935    i.nrf_gpio_cfg      nrfx_uarte.o
    0x0003b1fe   0x00000012   Code   RO         2936    i.nrf_gpio_cfg_default  nrfx_uarte.o
    0x0003b210   0x00000012   Code   RO         2937    i.nrf_gpio_cfg_input  nrfx_uarte.o
    0x0003b222   0x00000014   Code   RO         2938    i.nrf_gpio_cfg_output  nrfx_uarte.o
    0x0003b236   0x00000016   Code   RO          310    i.nrf_gpio_pin_write  boards.o
    0x0003b24c   0x00000030   Code   RO         2656    i.nrf_nvmc_page_erase  nrf_nvmc.o
    0x0003b27c   0x00000030   Code   RO         2659    i.nrf_nvmc_write_word  nrf_nvmc.o
    0x0003b2ac   0x00000044   Code   RO         2660    i.nrf_nvmc_write_words  nrf_nvmc.o
    0x0003b2f0   0x0000000c   Code   RO          594    i.nrf_rtc_event_clear  nrf_bootloader_dfu_timers.o
    0x0003b2fc   0x00000024   Code   RO         1326    i.nrf_sw_backend_hash_sha256_finalize  nrf_sw_backend_hash.o
    0x0003b320   0x00000006   Code   RO         1327    i.nrf_sw_backend_hash_sha256_init  nrf_sw_backend_hash.o
    0x0003b326   0x00000006   Code   RO         1328    i.nrf_sw_backend_hash_sha256_update  nrf_sw_backend_hash.o
    0x0003b32c   0x0000000a   Code   RO         2939    i.nrf_uarte_event_check  nrfx_uarte.o
    0x0003b336   0x0000000c   Code   RO         2940    i.nrf_uarte_event_clear  nrfx_uarte.o
    0x0003b342   0x00000002   PAD
    0x0003b344   0x00000010   Code   RO          772    i.nrf_wdt_started   nrf_bootloader_wdt.o
    0x0003b354   0x00000010   Code   RO         2941    i.nrfx_is_in_ram    nrfx_uarte.o
    0x0003b364   0x00000004   Code   RO         2870    i.nrfx_prs_acquire  nrfx_prs.o
    0x0003b368   0x00000002   Code   RO         2871    i.nrfx_prs_release  nrfx_prs.o
    0x0003b36a   0x00000002   PAD
    0x0003b36c   0x0000006c   Code   RO         2943    i.nrfx_uarte_init   nrfx_uarte.o
    0x0003b3d8   0x00000104   Code   RO         2944    i.nrfx_uarte_rx     nrfx_uarte.o
    0x0003b4dc   0x000000ac   Code   RO         2947    i.nrfx_uarte_tx     nrfx_uarte.o
    0x0003b588   0x0000001c   Code   RO         2949    i.nrfx_uarte_tx_in_progress  nrfx_uarte.o
    0x0003b5a4   0x00000108   Code   RO         2950    i.nrfx_uarte_uninit  nrfx_uarte.o
    0x0003b6ac   0x00000018   Code   RO         4365    i.nvmc_config       system_nrf52.o
    0x0003b6c4   0x00000074   Code   RO         1757    i.on_data_obj_create_request  nrf_dfu_req_handler.o
    0x0003b738   0x00000078   Code   RO         1758    i.on_data_obj_execute_request_sched  nrf_dfu_req_handler.o
    0x0003b7b0   0x00000080   Code   RO         1759    i.on_data_obj_write_request  nrf_dfu_req_handler.o
    0x0003b830   0x0000000c   Code   RO         1760    i.on_dfu_complete   nrf_dfu_req_handler.o
    0x0003b83c   0x00000024   Code   RO           27    i.on_error          main.o
    0x0003b860   0x00000098   Code   RO         1761    i.on_fw_version_request  nrf_dfu_req_handler.o
    0x0003b8f8   0x0000000c   Code   RO         2016    i.payload_free      nrf_dfu_serial_uart.o
    0x0003b904   0x00000040   Code   RO         4177    i.pb_dec_bytes      pb_decode.o
    0x0003b944   0x00000006   Code   RO         4178    i.pb_dec_fixed32    pb_decode.o
    0x0003b94a   0x00000006   Code   RO         4179    i.pb_dec_fixed64    pb_decode.o
    0x0003b950   0x0000003e   Code   RO         4180    i.pb_dec_string     pb_decode.o
    0x0003b98e   0x00000040   Code   RO         4181    i.pb_dec_submessage  pb_decode.o
    0x0003b9ce   0x00000058   Code   RO         4182    i.pb_dec_svarint    pb_decode.o
    0x0003ba26   0x00000058   Code   RO         4183    i.pb_dec_uvarint    pb_decode.o
    0x0003ba7e   0x0000005a   Code   RO         4184    i.pb_dec_varint     pb_decode.o
    0x0003bad8   0x0000001e   Code   RO         4185    i.pb_decode         pb_decode.o
    0x0003baf6   0x00000020   Code   RO         4187    i.pb_decode_fixed32  pb_decode.o
    0x0003bb16   0x0000005c   Code   RO         4188    i.pb_decode_fixed64  pb_decode.o
    0x0003bb72   0x00000002   PAD
    0x0003bb74   0x00000186   Code   RO         4189    i.pb_decode_noinit  pb_decode.o
    0x0003bcfa   0x0000003a   Code   RO         4190    i.pb_decode_svarint  pb_decode.o
    0x0003bd34   0x0000003c   Code   RO         4191    i.pb_decode_tag     pb_decode.o
    0x0003bd70   0x0000004a   Code   RO         4192    i.pb_decode_varint  pb_decode.o
    0x0003bdba   0x0000004c   Code   RO         4193    i.pb_decode_varint32  pb_decode.o
    0x0003be06   0x00000002   PAD
    0x0003be08   0x0000003c   Code   RO         2337    i.pb_decoding_callback  nrf_dfu_validation.o
    0x0003be44   0x00000022   Code   RO         4144    i.pb_field_iter_begin  pb_common.o
    0x0003be66   0x0000002e   Code   RO         4145    i.pb_field_iter_find  pb_common.o
    0x0003be94   0x0000007e   Code   RO         4146    i.pb_field_iter_next  pb_common.o
    0x0003bf12   0x000000a4   Code   RO         4194    i.pb_field_set_to_default  pb_decode.o
    0x0003bfb6   0x00000002   PAD
    0x0003bfb8   0x00000014   Code   RO         4195    i.pb_istream_from_buffer  pb_decode.o
    0x0003bfcc   0x00000036   Code   RO         4196    i.pb_make_string_substream  pb_decode.o
    0x0003c002   0x00000026   Code   RO         4197    i.pb_message_set_to_defaults  pb_decode.o
    0x0003c028   0x00000058   Code   RO         4198    i.pb_read           pb_decode.o
    0x0003c080   0x00000020   Code   RO         4199    i.pb_readbyte       pb_decode.o
    0x0003c0a0   0x0000005a   Code   RO         4200    i.pb_skip_field     pb_decode.o
    0x0003c0fa   0x00000002   PAD
    0x0003c0fc   0x000000f0   Code   RO         2338    i.postvalidate      nrf_dfu_validation.o
    0x0003c1ec   0x00000118   Code   RO         2339    i.postvalidate_sd_bl  nrf_dfu_validation.o
    0x0003c304   0x0000000e   Code   RO         3723    i.read              nrf_fstorage_nvmc.o
    0x0003c312   0x00000062   Code   RO         4201    i.read_raw_value    pb_decode.o
    0x0003c374   0x000000ee   Code   RO         4097    i.response_send     nrf_dfu_serial.o
    0x0003c462   0x00000004   Code   RO         3724    i.rmap              nrf_fstorage_nvmc.o
    0x0003c466   0x00000002   PAD
    0x0003c468   0x00000024   Code   RO         2017    i.rsp_send          nrf_dfu_serial_uart.o
    0x0003c48c   0x00000016   Code   RO         2951    i.rx_done_event     nrfx_uarte.o
    0x0003c4a2   0x00000002   PAD
    0x0003c4a4   0x00000054   Code   RO          679    i.sd_activate       nrf_bootloader_fw_activation.o
    0x0003c4f8   0x00000044   Code   RO         2486    i.sd_req_check      nrf_dfu_ver_validation.o
    0x0003c53c   0x0000005c   Code   RO         2487    i.sd_req_ok         nrf_dfu_ver_validation.o
    0x0003c598   0x00000014   Code   RO         2117    i.settings_backup   nrf_dfu_settings.o
    0x0003c5ac   0x0000000a   Code   RO         2118    i.settings_crc_get  nrf_dfu_settings.o
    0x0003c5b6   0x00000050   Code   RO         2119    i.settings_write    nrf_dfu_settings.o
    0x0003c606   0x00000110   Code   RO         3985    i.sha256_final      sha256.o
    0x0003c716   0x00000002   PAD
    0x0003c718   0x00000054   Code   RO         3986    i.sha256_init       sha256.o
    0x0003c76c   0x0000012c   Code   RO         3987    i.sha256_transform  sha256.o
    0x0003c898   0x00000054   Code   RO         3988    i.sha256_update     sha256.o
    0x0003c8ec   0x0000006e   Code   RO         4029    i.slip_decode_add_byte  slip.o
    0x0003c95a   0x00000056   Code   RO         4030    i.slip_encode       slip.o
    0x0003c9b0   0x000000c8   Code   RO         2340    i.stored_init_cmd_decode  nrf_dfu_validation.o
    0x0003ca78   0x00000060   Code   RO          595    i.timer_activate    nrf_bootloader_dfu_timers.o
    0x0003cad8   0x00000078   Code   RO          596    i.timer_init        nrf_bootloader_dfu_timers.o
    0x0003cb50   0x0000001a   Code   RO          597    i.timer_start       nrf_bootloader_dfu_timers.o
    0x0003cb6a   0x00000002   PAD
    0x0003cb6c   0x00000014   Code   RO          598    i.timer_stop        nrf_bootloader_dfu_timers.o
    0x0003cb80   0x0000001a   Code   RO         2952    i.tx_done_event     nrfx_uarte.o
    0x0003cb9a   0x00000002   PAD
    0x0003cb9c   0x00000028   Code   RO         2018    i.uart_dfu_transport_close  nrf_dfu_serial_uart.o
    0x0003cbc4   0x000000b8   Code   RO         2019    i.uart_dfu_transport_init  nrf_dfu_serial_uart.o
    0x0003cc7c   0x00000068   Code   RO         2020    i.uart_event_handler  nrf_dfu_serial_uart.o
    0x0003cce4   0x00000030   Code   RO         2528    i.uarte_evt_handler  nrf_drv_uart.o
    0x0003cd14   0x00000112   Code   RO         2953    i.uarte_irq_handler  nrfx_uarte.o
    0x0003ce26   0x00000012   Code   RO         4098    i.uint32_encode     nrf_dfu_serial.o
    0x0003ce38   0x00000010   Code   RO         3725    i.uninit            nrf_fstorage_nvmc.o
    0x0003ce48   0x00000058   Code   RO         2341    i.update_data_size_get  nrf_dfu_validation.o
    0x0003cea0   0x00000010   Code   RO         2342    i.update_requires_softdevice  nrf_dfu_validation.o
    0x0003ceb0   0x00000020   Code   RO         1076    i.verify_context    nrf_crypto_hash.o
    0x0003ced0   0x0000003c   Code   RO          773    i.wdt_feed          nrf_bootloader_wdt.o
    0x0003cf0c   0x00000004   Code   RO          774    i.wdt_feed_timer_handler  nrf_bootloader_wdt.o
    0x0003cf10   0x00000004   Code   RO         3726    i.wmap              nrf_fstorage_nvmc.o
    0x0003cf14   0x00000044   Code   RO         3727    i.write             nrf_fstorage_nvmc.o
    0x0003cf58   0x00000040   Data   RO            1    .constdata          dfu_public_key.o
    0x0003cf98   0x00000008   Data   RO          311    .constdata          boards.o
    0x0003cfa0   0x00000006   Data   RO          599    .constdata          nrf_bootloader_dfu_timers.o
    0x0003cfa6   0x00000002   PAD
    0x0003cfa8   0x00000018   Data   RO         1329    .constdata          nrf_sw_backend_hash.o
    0x0003cfc0   0x0000000c   Data   RO         1379    .constdata          micro_ecc_backend_ecc.o
    0x0003cfcc   0x00000001   Data   RO         1558    .constdata          dfu-cc.pb.o
    0x0003cfcd   0x00000003   PAD
    0x0003cfd0   0x00000030   Data   RO         1559    .constdata          dfu-cc.pb.o
    0x0003d000   0x00000030   Data   RO         1560    .constdata          dfu-cc.pb.o
    0x0003d030   0x000000b0   Data   RO         1561    .constdata          dfu-cc.pb.o
    0x0003d0e0   0x00000030   Data   RO         1562    .constdata          dfu-cc.pb.o
    0x0003d110   0x00000040   Data   RO         1563    .constdata          dfu-cc.pb.o
    0x0003d150   0x00000030   Data   RO         1564    .constdata          dfu-cc.pb.o
    0x0003d180   0x00000020   Data   RO         1709    .constdata          nrf_dfu_mbr.o
    0x0003d1a0   0x00000030   Data   RO         1762    .constdata          nrf_dfu_req_handler.o
    0x0003d1d0   0x00000020   Data   RO         2023    .constdata          nrf_dfu_serial_uart.o
    0x0003d1f0   0x00000004   Data   RO         2248    .constdata          nrf_dfu_utils.o
    0x0003d1f4   0x00000004   Data   RO         2956    .constdata          nrfx_uarte.o
    0x0003d1f8   0x0000000c   Data   RO         3728    .constdata          nrf_fstorage_nvmc.o
    0x0003d204   0x00000020   Data   RO         3729    .constdata          nrf_fstorage_nvmc.o
    0x0003d224   0x00000100   Data   RO         3989    .constdata          sha256.o
    0x0003d324   0x00000018   Data   RO         4099    .constdata          nrf_dfu_serial.o
    0x0003d33c   0x00000024   Data   RO         4202    .constdata          pb_decode.o
    0x0003d360   0x000000b0   Data   RO         4483    .rodata.curve_secp256r1  micro_ecc_lib_nrf52.lib(uECC.c.o)
    0x0003d410   0x00000020   Data   RO         4525    Region$$Table       anon$$obj.o
    0x0003d430   0x00000008   Data   RO         2027    dfu_trans           nrf_dfu_serial_uart.o
    0x0003d438   0x00000014   Data   RO         2028    nrf_balloc          nrf_dfu_serial_uart.o


    Execution Region RW_IRAM1 (Base: 0x20000008, Size: 0x00001d68, Max: 0x00005ff8, ABSOLUTE)

    Base Addr    Size         Type   Attr      Idx    E Section Name        Object

    0x20000008   0x00000008   Data   RW          416    .data               nrf_bootloader.o
    0x20000010   0x00000004   Data   RW          553    .data               nrf_bootloader_app_start_final.o
    0x20000014   0x00000030   Data   RW          600    .data               nrf_bootloader_dfu_timers.o
    0x20000044   0x00000001   Data   RW          680    .data               nrf_bootloader_fw_activation.o
    0x20000045   0x00000001   Data   RW          775    .data               nrf_bootloader_wdt.o
    0x20000046   0x00000001   Data   RW         1154    .data               nrf_crypto_init.o
    0x20000047   0x00000001   PAD
    0x20000048   0x00000004   Data   RW         1581    .data               nrf_dfu.o
    0x2000004c   0x00000001   Data   RW         1676    .data               nrf_dfu_handling_error.o
    0x2000004d   0x00000003   PAD
    0x20000050   0x00000010   Data   RW         1763    .data               nrf_dfu_req_handler.o
    0x20000060   0x00000014   Data   RW         2024    .data               nrf_dfu_serial_uart.o
    0x20000074   0x00000003   Data   RW         2025    .data               nrf_dfu_serial_uart.o
    0x20000077   0x00000001   PAD
    0x20000078   0x00000008   Data   RW         2026    .data               nrf_dfu_serial_uart.o
    0x20000080   0x00000004   Data   RW         2124    .data               nrf_dfu_settings.o
    0x20000084   0x00000010   Data   RW         2344    .data               nrf_dfu_validation.o
    0x20000094   0x00000008   Data   RW         2529    .data               nrf_drv_uart.o
    0x2000009c   0x00000010   Data   RW         3130    .data               app_scheduler.o
    0x200000ac   0x00000004   Data   RW         3187    .data               app_util_platform.o
    0x200000b0   0x00000004   Data   RW         3730    .data               nrf_fstorage_nvmc.o
    0x200000b4   0x00000004   Data   RW         4367    .data               system_nrf52.o
    0x200000b8   0x00000014   Data   RW         1618    fs_data             nrf_dfu_flash.o
    0x200000cc   0x00000420   Zero   RW          414    .bss                nrf_bootloader.o
    0x200004ec   0x0000018c   Zero   RW         2021    .bss                nrf_dfu_serial_uart.o
    0x20000678   0x00000059   Zero   RW         2022    .bss                nrf_dfu_serial_uart.o
    0x200006d1   0x00000003   PAD
    0x200006d4   0x00000a80   Zero   RW         2123    .bss                nrf_dfu_settings.o
    0x20001154   0x000003f4   Zero   RW         2343    .bss                nrf_dfu_validation.o
    0x20001548   0x00000024   Zero   RW         2954    .bss                nrfx_uarte.o
    0x2000156c   0x00000004   PAD
    0x20001570   0x00000800   Zero   RW         4353    STACK               arm_startup_nrf52820.o



  Load Region LR$$.ARM.__AT_0x0003E000 (Base: 0x0003e000, Size: 0x00000000, Max: 0x00001000, ABSOLUTE)

    Execution Region ER$$.ARM.__AT_0x0003E000 (Base: 0x0003e000, Size: 0x00001000, Max: 0x00001000, ABSOLUTE, UNINIT)

    Base Addr    Size         Type   Attr      Idx    E Section Name        Object

    0x0003e000   0x00001000   Zero   RW         2120    .ARM.__AT_0x0003E000  nrf_dfu_settings.o



  Load Region LR$$.ARM.__AT_0x0003F000 (Base: 0x0003f000, Size: 0x00000000, Max: 0x00001000, ABSOLUTE)

    Execution Region ER$$.ARM.__AT_0x0003F000 (Base: 0x0003f000, Size: 0x00001000, Max: 0x00001000, ABSOLUTE, UNINIT)

    Base Addr    Size         Type   Attr      Idx    E Section Name        Object

    0x0003f000   0x00001000   Zero   RW         2121    .ARM.__AT_0x0003F000  nrf_dfu_settings.o



  Load Region LR$$.ARM.__AT_0x10001014 (Base: 0x10001014, Size: 0x00000004, Max: 0x00000004, ABSOLUTE)

    Execution Region ER$$.ARM.__AT_0x10001014 (Base: 0x10001014, Size: 0x00000004, Max: 0x00000004, ABSOLUTE, UNINIT)

    Base Addr    Size         Type   Attr      Idx    E Section Name        Object

    0x10001014   0x00000004   Data   RW          731    .ARM.__AT_0x10001014  nrf_bootloader_info.o



  Load Region LR$$.ARM.__AT_0x10001018 (Base: 0x10001018, Size: 0x00000004, Max: 0x00000004, ABSOLUTE)

    Execution Region ER$$.ARM.__AT_0x10001018 (Base: 0x10001018, Size: 0x00000004, Max: 0x00000004, ABSOLUTE, UNINIT)

    Base Addr    Size         Type   Attr      Idx    E Section Name        Object

    0x10001018   0x00000004   Data   RO         2122    .ARM.__AT_0x10001018  nrf_dfu_settings.o


==============================================================================

Image component sizes


      Code (inc. data)   RO Data    RW Data    ZI Data      Debug   Object Name

       264         16          0         16          0      41641   app_scheduler.o
        44         10          0          4          0       3008   app_util_platform.o
        36          8        512          0       2048        868   arm_startup_nrf52820.o
       192         16          8          0          0       8789   boards.o
        60          6          0          0          0       1432   crc32.o
         0          0        433          0          0       1446   dfu-cc.pb.o
         0          0         64          0          0       5313   dfu_public_key.o
       180         34          0          0          0      79666   main.o
        22          0         12          0          0      25445   micro_ecc_backend_ecc.o
        86          0          0          0          0       2278   micro_ecc_backend_ecdsa.o
       260          0          0          0          0       5144   nrf_atomic.o
       152          0          0          0          0       3316   nrf_balloc.o
       566         94          0          8       1056      30694   nrf_bootloader.o
        36          0          0          0          0        687   nrf_bootloader_app_start.o
       160         16          0          4          0       8795   nrf_bootloader_app_start_final.o
       450         56          6         48          0      46718   nrf_bootloader_dfu_timers.o
       504         48          0          1          0       6429   nrf_bootloader_fw_activation.o
        48          6          0          4          0       1034   nrf_bootloader_info.o
       192         34          0          1          0      36008   nrf_bootloader_wdt.o
       124          4          0          0          0      30184   nrf_crypto_ecc.o
        76          4          0          0          0      37685   nrf_crypto_ecdsa.o
       230         12          0          0          0      10017   nrf_crypto_hash.o
        64         14          0          1          0       3001   nrf_crypto_init.o
        94          0          0          0          0       3690   nrf_crypto_shared.o
        84         14          0          4          0       3039   nrf_dfu.o
        72         20          0         20          0       5579   nrf_dfu_flash.o
        28         10          0          1          0       1540   nrf_dfu_handling_error.o
        66          4         32          0          0       7256   nrf_dfu_mbr.o
      1130        128         48         16          0      53452   nrf_dfu_req_handler.o
       446         30         24          0          0      45137   nrf_dfu_serial.o
       382         66         60         31        485      25128   nrf_dfu_serial_uart.o
       530         58          4          4      10880      11509   nrf_dfu_settings.o
       104         18          0          0          0       2564   nrf_dfu_transport.o
       334         42          4          0          0       5931   nrf_dfu_utils.o
      1924        166          0         16       1012      24079   nrf_dfu_validation.o
       288         14          0          0          0      10045   nrf_dfu_ver_validation.o
       112         14          0          8          0      13300   nrf_drv_uart.o
       230         10          0          0          0       5768   nrf_fstorage.o
       260         20         44          4          0       9148   nrf_fstorage_nvmc.o
         0          0          0          0          0       1512   nrf_nvic.o
       164         28          0          0          0       2495   nrf_nvmc.o
        48          0         24          0          0       5340   nrf_sw_backend_hash.o
         6          0          0          0          0       2394   nrfx_prs.o
      1572         46          4          0         36      63551   nrfx_uarte.o
       206          0          0          0          0       3264   pb_common.o
      2314         14         36          0          0      34682   pb_decode.o
       740         40        256          0          0       4940   sha256.o
       196          0          0          0          0       2401   slip.o
       400         48          0          4          0      29557   system_nrf52.o

    ----------------------------------------------------------------------
     15526       1168       1608        200      15524     766899   Object Totals
         0          0         32          0          0          0   (incl. Generated)
        50          0          5          5          7          0   (incl. Padding)

    ----------------------------------------------------------------------

      Code (inc. data)   RO Data    RW Data    ZI Data      Debug   Library Member Name

         0          0          0          0          0          0   entry.o
         0          0          0          0          0          0   entry10a.o
         0          0          0          0          0          0   entry11a.o
         8          4          0          0          0          0   entry2.o
         4          0          0          0          0          0   entry5.o
         0          0          0          0          0          0   entry7b.o
         0          0          0          0          0          0   entry8b.o
         8          4          0          0          0          0   entry9a.o
        30          0          0          0          0          0   handlers.o
        36          8          0          0          0         68   init.o
        30          0          0          0          0         68   llshl.o
        26          0          0          0          0         80   memcmp.o
        36          0          0          0          0         68   memcpya.o
        36          0          0          0          0        108   memseta.o
      4034          8        176          0          0      50043   uECC.c.o

    ----------------------------------------------------------------------
      4274         24        176          0          0      50435   Library Totals
        26          0          0          0          0          0   (incl. Padding)

    ----------------------------------------------------------------------

      Code (inc. data)   RO Data    RW Data    ZI Data      Debug   Library Name

       214         16          0          0          0        392   mc_w.l
      4034          8        176          0          0      50043   micro_ecc_lib_nrf52.lib

    ----------------------------------------------------------------------
      4274         24        176          0          0      50435   Library Totals

    ----------------------------------------------------------------------

==============================================================================


      Code (inc. data)   RO Data    RW Data    ZI Data      Debug   

     19800       1192       1784        200      15524     805318   Grand Totals
     19800       1192       1784        200      15524     805318   ELF Image Totals
     19800       1192       1784        200          0          0   ROM Totals

==============================================================================

    Total RO  Size (Code + RO Data)                21584 (  21.08kB)
    Total RW  Size (RW Data + ZI Data)             15724 (  15.36kB)
    Total ROM Size (Code + RO Data + RW Data)      21784 (  21.27kB)

==============================================================================

